:100000000C9407080C9438080C9438080C943808A1
:100010000C9438080C9438080C9438080C94380860
:100020000C9438080C9438080C9438080C94380850
:100030000C9438080C94677C0C9438080C9438089D
:100040000C9438080C9438080C9438080C94380830
:100050000C9438080C9438080C9438080C942A85B1
:100060000C9438080C940B450C94E2440C9438081A
:100070000C943808FDC70000FBC70000F9C700005A
:10008000F7C70000F5C70000F3C70000F1C7000084
:100090000C94B8440C948F44EBC700000C947A7D08
:1000A000E7C70000E5C70000E3C70000E1C70000A4
:1000B000DFC70000DDC70000DBC70000D9C70000B4
:1000C000D7C70000D5C70000D3C700000C94654413
:1000D0000C943C44CDC700000C9412440C94E943AA
:1000E000C7C70000B9309B30C030C030C030C0300E
:1000F000C030C030C030C030C030C030401E55218C
:100100005D212123D823F424A726A3271B283028E8
:100110003428C03047285328C029952BAF2BCF2C2B
:100120002E2D0A2E862E8D2E762FC030C030C03058
:10013000C030C030C030C030C030C030C030B12F4F
:10014000C030C030C030C030C030C030EE30D97E9A
:10015000BC7F5C807A808F80A480B980D780EC805F
:1001600001811F81348143815881B683B983A8837B
:10017000AC83B283F083BD83C183C783CB83CF833A
:10018000D583D983DD83F083E383E783EB83084A58
:10019000D73B3BCE016E84BCBFFDC12F3D6C74319B
:1001A0009ABD56833DDA3D00C77F11BED9E4BB4CF2
:1001B0003E916BAAAABE000000803F07634236B79B
:1001C0009BD8A71A39685618AEBAAB558C1D3CB7E8
:1001D000CC5763BD6DEDFD753EF6177231BF000063
:1001E00000803F08000000BE922449123EABAAAA3C
:1001F0002ABECDCCCC4C3E00000080BEABAAAAAA41
:100200003E00000000BF000000803F000000000032
:10021000084178D3BB4387D1133D190E3CC3BD427F
:1002200082AD2B3E68EC8276BED98FE1A93E4C8030
:10023000EFFFBE01C4FF7F3F0000000000004E4101
:100240004E494E495459494E46CDCCCC3D0AD72350
:100250003C17B7D13877CC2B329595E6241FB14F98
:100260000A000020410000C84200401C4620BCBEDD
:100270004CCA1B0E5AAEC59D7400407A10F35A004A
:10028000A0724E18090010A5D4E80000E8764817BF
:100290000000E40B54020000CA9A3B000000E1F5A4
:1002A00005000080969800000040420F000000A06A
:1002B0008601000000102700000000E80300000095
:1002C000006400000000000A0000000000010000BF
:1002D0000000002C76D888DC674F0823DFC1DFAE32
:1002E00059E1B1B796E5E3E453C63AE651997696FB
:1002F000E8E6C28426EB898C9B62ED407C6FFCEFC4
:10030000BC9C9F40F2BAA56FA5F490055A2AF75CF1
:10031000936B6CF9676DC11BFCE0E40D47FEF520A3
:10032000E6B500D0ED902E0300943577050080846B
:100330001E080000204E0A000000C80C333333337F
:100340000F986E12831141EF8D2114893BE65516EB
:10035000CFFEE6DB18D1844B381BF77C1D901DA423
:10036000BBE424203284725E228100C9F124ECA116
:10037000E53D27696E7075742044535463616C6960
:1003800062726174653A0020766F6C746167653DD6
:1003900000235475726269646974792055707065C0
:1003A00072204C696D69743A200020766F6C74611C
:1003B00067653D0023547572626964697479204CE5
:1003C0006F776572204C696D69743A20002354750B
:1003D00072626964697479204C6F776572204C6928
:1003E0006D69742056696E663A200023434F3220AF
:1003F0004D415820766F6C7420280023434F3220E3
:100400007A65726F20766F6C74202800234F32203B
:1004100063616C6962726174696F6E3A2000235483
:100420007572626964697479204C6F776572204CCB
:10043000696D69742056313A200057694669204930
:10044000503A004D6F74696F6E004D6F74696F6E36
:1004500000555620496E742E00555620496E74651D
:100460006E73697479004F3220436F6E6300434F9F
:100470003220436F6E630053656E736F7220657236
:10048000726F722100234E6F2073656E736F72213D
:1004900000434F3220436F6E63004D656173757288
:1004A000696E6700234E6F2073656E736F722066EE
:1004B0006F7220504D21004E6F2073656E736F7206
:1004C0002100206E672F4C00504D313A322E353AC4
:1004D0003130004D6561737572696E672E2E002391
:1004E0004E6F2054422073656E736F723F00234E2F
:1004F0006F2073656E736F722100536F756E642089
:100500004C6576656C004D6561737572696E672E1A
:100510002E00234E6F2073656E736F722100536F30
:10052000756E64204C6576656C00234E6F20736594
:100530006E736F7220666F722074656D7020262056
:1005400068756D696469747921004E6F2053656E1A
:10055000736F72210020666F722074656D702026A3
:100560002068756D696469747921002353656E7321
:100570006F72204572726F72200053656E736F72D6
:10058000204572726F7221002357726F6E6720735D
:10059000656E736F7220666F722074656D702026B1
:1005A0002068756D6964697479210057726F6E6790
:1005B0002053656E736F72210054656D702048750D
:1005C0006D6964697479004C6967687420496E7458
:1005D000656E7369747900466C616D6520495200DF
:1005E000482D6669656C64005365617263682044D8
:1005F0006972656374696F6E00234E6F20704820C6
:1006000073656E736F72210070482076616C75653A
:1006100000496E76616C6964206B657921002372F4
:1006200065706C6965733D0067657453656C6654ED
:1006300065737442697428293A20006973496E749D
:10064000657272757074456E61626C6564283129DB
:100650003A2000676574496E746572727570744DE6
:10066000617070696E672831293A200067657449A6
:100670006E74657272757074536F7572636528312C
:10068000293A2000676574496E74657272757074DA
:10069000536F7572636528293A200067657452614B
:1006A000746528293A20332E31343135393F0061C1
:1006B0006363656C2E69734C6F77506F7765722832
:1006C000293A2000616363656C2E697341736C6520
:1006D000657028293A2000616363656C2E69735444
:1006E0006170536F757263654F6E5A28293A200006
:1006F000616363656C2E6973546170536F757263C7
:10070000654F6E5928293A2000616363656C2E6934
:1007100073546170536F757263654F6E5828293A30
:100720002000616363656C2E697341637469766947
:100730007479536F757263654F6E5A28293A200099
:10074000616363656C2E697341637469766974795A
:10075000536F757263654F6E5928293A200069738B
:100760004163746976697479536F757263654F6E0E
:100770005828293A20006973546170446574656390
:1007800074696F6E4F6E5A28293B2066616C7365E1
:100790003F20006973546170446574656374696FC8
:1007A0006E4F6E5A28293B20747275653F20006990
:1007B00073546170446574656374696F6E4F6E59EC
:1007C00028293B2066616C73653F20006973546182
:1007D00070446574656374696F6E4F6E5928293B68
:1007E00020747275653F20006973546170446574AC
:1007F000656374696F6E4F6E5828293B2066616C83
:1008000073653F2000697354617044657465637457
:10081000696F6E4F6E5828293B20747275653F20B2
:1008200000676574537570707265737342697428DC
:10083000293B2066616C73653F20006765745375C2
:1008400070707265737342697428293B20747275E5
:10085000653F200069734163746976697479416307
:1008600028293A20006973496E6163746976697456
:10087000795A456E61626C656428293A2000697373
:10088000496E616374697669747959456E61626C09
:10089000656428293A20006973496E61637469763A
:1008A00069747958456E61626C656428293A200044
:1008B000697341637469766974795A456E61626CD3
:1008C000656428293A200069734163746976697404
:1008D0007959456E61626C656428293A2000697314
:1008E000416374697669747958456E61626C6564B8
:1008F00028293A20006765744672656546616C6C0C
:100900004475726174696F6E28293A2000676574B6
:100910004672656546616C6C5468726573686F6C8D
:100920006428293A200067657454696D65496E61D1
:100930006374697669747928293A20006765744977
:100940006E61637469766974795468726573686FEF
:100950006C64282920006765744163746976697442
:10096000795468726573686F6C6428292000676524
:1009700074446F75626C6554617057696E646F770B
:1009800028292000676574446F75626C6554617036
:100990004C6174656E637928293A20006765745448
:1009A00061704475726174696F6E28293A2000671E
:1009B0006574417869734F66667365742826782C70
:1009C0002026792C20267A293A2000676574546104
:1009D000705468726573686F6C6428293A200058F7
:1009E000595A2047733A200058595A20434F554EC0
:1009F00054533A2000736574206761696E735B5DC0
:100A00003A006761696E735F6F7269675B5D3A0098
:100A100043616C6962726174696F6E2050726573B4
:100A2000737572653D00536561206C6576656C2059
:100A3000502863616C63293D00234572726F723ADE
:100A4000707265737375726520424D503038352C65
:100A500020636865636B20776972696E672100495E
:100A6000522054656D702073656E736F7220666FCF
:100A7000756E6400504D322E352073656E736F7243
:100A8000206C696B656C7920666F756E64005769C0
:100A900046692049503A00456455484B2053455318
:100AA0004C6F676765720053656E736F7220736C6D
:100AB0006F7420616E6420747970653A0057656CBC
:100AC000636F6D6520746F20456455484B00005E70
:100AD000BCE2613FDD83C29C7E20A3FD1F41009DDF
:100AE00023BE46DB65F88C11AF32CA57E9744F66F6
:100AF00066206169722D636F6E64210049742773EB
:100B000020746F6F20636F6F6C210054656D7020CF
:100B100069732066696E6521004973206169722DD1
:100B2000636F6E64206F6E3F004974277320717588
:100B300069746520686F7421004974277320766595
:100B4000727920686F742120004F66662061697297
:100B50002D636F6E6421004974277320746F6F20BA
:100B6000636F6F6C210054656D7020697320666936
:100B70006E6521004973206169722D636F6E642078
:100B80006F6E3F0049742773207175697465206822
:100B90006F74210049742773207665727920686F1D
:100BA00074210054656D702048756D6964697479AD
:100BB0000020202020202020202020202020202055
:100BC0002000202020202020202020202020202045
:100BD00020200023616E6F7468657220495220697D
:100BE0006E7075743D00236B65793D00416E676CD6
:100BF00065732F003E6128782C792C7A292F673A6B
:100C0000004E6F2073656E736F722100495220543D
:100C1000656D7065726174757265004D656173759F
:100C200072696E672E2E004E6F2073656E736F7241
:100C30003F0049522054656D70657261747572652C
:100C4000004D6561737572696E672E2E00232D2D20
:100C50002D2D2D2D2D2D2D2D2D2D2D2D2D2D2D2DC4
:100C60002D2D2D2D2D2D2D2D2D2D2D2D2D2D2D2DB4
:100C70002D2D00235265736F6C7574696F6E3A2069
:100C8000202000234D696E2056616C75653A202046
:100C9000202000234D61782056616C75653A202034
:100CA00020200023556E697175652049443A202043
:100CB00020200023447269766572205665723A20BE
:100CC0002020002353656E736F723A20202020206D
:100CD000202000232D2D2D2D204D61676E65746918
:100CE000632053656E736F72202D2D2D2D2D2D2DAC
:100CF0002D2D2D2D2D2D2D2D2D2D2D2D2D00482D36
:100D00006669656C643A202800202020202020207D
:100D100020202020202020202000202020202020F3
:100D200020202020202020202020002020202020E3
:100D300020202020202020202020002020202020D3
:100D400020202020202020202020004E6F205365CE
:100D50006E736F7221004E6F204453205468657289
:100D60006D6F6D657465722100445320546865721F
:100D70006D2E00233A53686F772F48696465204CC5
:100D80004344002A3A546869732048656C700044F3
:100D9000433A436C656172204C43440044423A52EA
:100DA00065736574204C6F676765720044363A441A
:100DB000532054656D700044353A555620496E7481
:100DC000656E736974790044343A4F3220636F6EF4
:100DD000632E0044333A434F3220636F6E632E001C
:100DE00044323A504D28313A322E353A31302900CA
:100DF00044323A504D28313A322E353A3130292A90
:100E00000044313A547572626964697479004430FF
:100E10003A566F6C7461676500393A6F72203344DB
:100E200020616363656C2E00393A496E636C2E2035
:100E3000616E672E00383A70482076616C756500E7
:100E4000373A49522054656D7000373A4952205460
:100E5000656D702A00363A4D61676E65746963206E
:100E60006669656C6400353A476173204C65766548
:100E70006C00343A495220466C616D6500333A4C3F
:100E80006967687420496E742E00323A616E64207E
:100E900048656967687400323A54656D7020507215
:100EA00065737375726500313A54656D70204875CD
:100EB0006D696469747900303A536F756E64204CC3
:100EC0006576656C00303A536F756E64204C6576BC
:100ED000656C2A0054696D65206C617073653A0019
:100EE000576946692049503A000000210024002734
:100EF000002A002D0030003300010100000401072A
:100F0000010A0100002200250028002B002E0031DC
:100F100000340002010000050108010B010000205F
:100F2000002300260029002C002F003200000100C1
:100F30000003010601090105050505070508080864
:100F400008020202020A0A0808040404040101015A
:100F50000101010101030303030303030304070762
:100F6000070C0C0C0C0C0C0C0C0202020206060600
:100F700006060606060B0B0B0B0B0B0B0B010210E8
:100F800020200808102040102040800201020108A3
:100F90000402010102040810204080804020100853
:100FA00004020180040201804020100804020108AC
:100FB000040201010204081020408001020408100C
:100FC00020408000000A0B02090C0D0E08070304E4
:100FD0000100000000000000000000000000000010
:100FE00000000000000000000000000000000012EF
:100FF00011100000000000000000000000000000D0
:1010000000000000000000000000408E98901124B5
:101010001FBECFEFD1E2DEBFCDBF00E00CBF1BE0B3
:10102000A0E0B2E0ECEDF9E301E00BBF02C00790F5
:101030000D92A43EB107D9F722E1A4EEBBE001C0B6
:101040001D92A739B207E1F718E0C6E0D8E000E04A
:1010500006C021970109802FFE010E94389AC530F1
:10106000D10780E00807A9F70E94B9850C94DD9CA0
:101070000C9400002F923F924F925F926F927F925A
:101080008F929F92AF92BF92CF92DF92EF92FF9298
:101090000F931F93CF93DF93CDB7DEB7EA970FB6C9
:1010A000F894DEBF0FBECDBF10918712112321F03F
:1010B000109287120C948E1D8091461190914711C9
:1010C000019709F050C060E070E082E491E10E9475
:1010D0002341082E000C990B0E947C9C892B09F45B
:1010E00042C06BE675E0CE0183960E94B142BE011C
:1010F0006D5D7F4F82E491E10E946054811127C0B1
:1011000060E779E0CE0145960E94B142BE016B5E78
:101110007F4F82E491E10E946054811114C06BEB17
:101120007AE0CE0101960E94B142BE016F5F7F4F0F
:1011300082E491E10E94605411E0811110E0CE013F
:1011400001960E946D42CE0145960E946D42CE01ED
:1011500083960E946D42112331F062E471E186E3CF
:1011600091E10E9458428091461190914711049755
:1011700008F041C062EB77E0CE0101960E94B142D7
:10118000BE016F5F7F4F82E491E10E946054182F8F
:10119000CE0101960E946D42112369F161E070E079
:1011A00082E491E10E94234180330CF484516AE28D
:1011B00070E0681B710987FD7395CE0101960E944E
:1011C000BB58BE016F5F7F4F82E491E10E943441C2
:1011D000CE0101960E946D4262E471E186E391E1E5
:1011E0000E94584282E491E10E94B840CB010E94E3
:1011F000A71D0C948E1D6DE675E0CE0145960E94EC
:10120000B142BE016B5E7F4F82E491E10E94605467
:10121000811116C061E775E0CE0101960E94B142CE
:10122000BE016F5F7F4F82E491E10E94605411E044
:10123000811101C010E0CE0101960E946D4201C0F3
:1012400011E0CE0145960E946D42112309F453C36B
:1012500065E775E0CE0101960E94B142CE0101968C
:101260000E947258CE0101960E946D4261E875E0BD
:10127000CE0101960E94B1426FE172E1CE0101966A
:101280000E94D941BC01CE0145960E94A942CE01DF
:1012900045960E947258CE0145960E946D42CE013D
:1012A00001960E946D4260916F047091700480916C
:1012B0007104909172040E945A9520E030E048EC4D
:1012C00052E40E94AA97AB01BC0122E0CE014596F0
:1012D0000E94724267E975E0CE0101960E94B14218
:1012E000BE016B5E7F4FCE0101960E94D94168EF2F
:1012F00076E00E94C241BC01CE0183960E94A942C1
:10130000CE0183960E947258CE0183960E946D4250
:10131000CE0101960E946D42CE0145960E946D421B
:1013200040916B0450916C0460916D0470916E0457
:1013300024E0CE0145960E9472426CEA75E0CE012F
:1013400001960E94B142BE016B5E7F4FCE010196B5
:101350000E94D941BC01CE0183960E94A942CE01D0
:1013600083960E947258CE0183960E946D42CE01F0
:1013700001960E946D42CE0145960E946D424091B9
:101380005F0450916004609161047091620422E0F6
:10139000CE018F960E94724240915704509158049A
:1013A0006091590470915A0423E0CE0189960E94FD
:1013B000724240916304509164046091650470919D
:1013C000660422E0CE0183960E94724240915B0443
:1013D00050915C0460915D0470915E0423E0CE0145
:1013E00045960E94724269EC75E0CE0101960E941A
:1013F000B142BE016B5E7F4FCE0101960E94D94182
:101400006EED75E00E94C241BE016D5D7F4F0E948E
:10141000D94161EE75E00E94C241BE01675D7F4F18
:101420000E94D9416EED75E00E94C241BE01615D2E
:101430007F4F0E94D94167EE75E00E94C241BC0116
:10144000CE01C5960E94A942CE01C5960E9472584F
:10145000CE01C5960E946D42CE0101960E946D425A
:10146000CE0145960E946D42CE0183960E946D4248
:10147000CE0189960E946D42CE018F960E946D42E8
:101480004091BA045091BB046091BC047091BD04BA
:1014900023E0CE0183960E94724220915304309142
:1014A0005404409155045091560460E070E080E28D
:1014B00091E40E945899AB01BC0121E0CE01459610
:1014C0000E9472426CEE75E0CE0101960E94B1421C
:1014D000BE016B5E7F4FCE0101960E94D9416FEF36
:1014E00075E00E94C241BE016D5D7F4F0E94D941EF
:1014F00065E076E00E94C241BC01CE0189960E945F
:10150000A942CE0189960E947258CE0189960E9406
:101510006D42CE0101960E946D42CE0145960E9419
:101520006D42CE0183960E946D424091B604509167
:10153000B7046091B8047091B90423E0CE0183969A
:101540000E94724220914F04309150044091510406
:101550005091520460E070E080E291E40E9458995A
:10156000AB01BC0121E0CE0145960E94724268E0C9
:1015700076E0CE0101960E94B142BE016B5E7F4FC4
:10158000CE0101960E94D9416FEF75E00E94C241E1
:10159000BE016D5D7F4F0E94D94165E076E00E94FB
:1015A000C241BC01CE0189960E94A942CE01899612
:1015B0000E947258CE0189960E946D42CE0101961A
:1015C0000E946D42CE0145960E946D42CE018396E7
:1015D0000E946D4240914B0450914C0460914D0427
:1015E00070914E0422E0CE0145960E9472426BE15A
:1015F00076E0CE0101960E94B142BE016B5E7F4F44
:10160000CE0101960E94D94161E376E00E94C24179
:10161000BC01CE0183960E94A942CE0183960E940E
:101620007258CE0183960E946D42CE0101960E94AF
:101630006D42CE0145960E946D4240914704509103
:1016400048046091490470914A0422E0CE01459615
:101650000E94724268E376E0CE0101960E94B14298
:10166000BE016B5E7F4FCE0101960E94D94165E0BD
:1016700076E00E94C241BC01CE0183960E94A9423D
:10168000CE0183960E947258CE0183960E946D42CD
:10169000CE0101960E946D42CE0145960E946D4298
:1016A00095E3C92E94E0D92E01E010E027E1E22E67
:1016B0008091330490913404801791070CF44DC04D
:1016C000D601AD90BD906D01B501CE0183960E940B
:1016D000BB58B801CE0145960E94BB586BE476E03A
:1016E000CE0101960E94B142BE016B5E7F4FCE01DA
:1016F00001960E94D94168E176E00E94C241BE0194
:101700006D5D7F4F0E94D94163E576E00E94C24142
:10171000EA9CB001EB9C700D1124655E7D4F0E9428
:10172000C241BC01CE0189960E94A942CE01899690
:101730000E947258CE0189960E946D42CE01019698
:101740000E946D42CE0145960E946D42CE01839665
:101750000E946D420F5F1F4FABCF8091220D909181
:10176000230D892B71F469E576E0CE0101960E9484
:10177000B142CE0101960E947258CE0101960E949C
:101780006D428091220D9091230D019771F468E6CE
:1017900076E0CE0101960E94B142CE0101960E94F0
:1017A0007258CE0101960E946D428091220D909157
:1017B000230D029771F462E776E0CE0101960E9454
:1017C000B142CE0101960E947258CE0101960E944C
:1017D0006D426091450470914604CE0145960E9489
:1017E000BB5864E876E0CE0101960E94B142BE018A
:1017F0006B5E7F4FCE0101960E94D941BC01CE01A4
:1018000083960E94A942CE0183960E947258CE010F
:1018100083960E946D42CE0101960E946D42CE01D8
:1018200045960E946D4240911702509118026091B6
:10183000190270911A0222E0CE0145960E9472426E
:1018400061EA76E0CE0101960E94B142BE016B5E74
:101850007F4FCE0101960E94D94166EE78E00E944A
:10186000C241BC01CE0183960E94A942CE0183965B
:101870000E947258CE0183960E946D42CE0101965D
:101880000E946D42CE0145960E946D424091130226
:1018900050911402609115027091160222E0CE015F
:1018A00045960E94724261EB76E0CE0101960E945D
:1018B000B142BE016B5E7F4FCE0101960E94D941BD
:1018C00066EE78E00E94C241BC01CE0183960E9480
:1018D000A942CE0183960E947258CE0183960E943F
:1018E0006D42CE0101960E946D42CE0145960E9446
:1018F0006D421092120280914611909147118330EF
:10190000910508F092C08130910541F460E070E0EB
:1019100082E491E10E942341F82E62C0029709F00F
:101920005FC062EB77E0CE0101960E94B142BE013A
:101930006F5F7F4F82E491E10E946054182FCE01C7
:1019400001960E946D42112309F44AC061E070E0E3
:1019500082E491E10E9423411A8219821C821B8237
:101960001E821D828D8B1E8ABE016B5E7F4FCE0153
:1019700001960E944342BE016F5F7F4F86E391E173
:101980000E943441CE0101960E946D4260E070E0F9
:1019900082E491E10E942341F82E8091800C8823FB
:1019A000F9F061EC76E0CE0101960E94B14262E46A
:1019B00071E1CE0101960E94D94160E27BE00E9474
:1019C000C241BC0183EA9FE00E940F43CE01019611
:1019D0000E946D4266E371E183EA9FE00E947A6AA9
:1019E0008F2D0F2C000C990B0E947C9C892BB1F041
:1019F0000E94D0740E942F6F60E27BE0CE010196BE
:101A00000E94B1424AE050E060E070E0CE010196F1
:101A10000E94CC5ACE0101960E946D428F2D0E94E9
:101A20005C480E941E850C94841D21E030E040E05B
:101A300050E062E471E1CE0101960E94C542BE0110
:101A40006F5F7F4F84E291E10E943441CE010196A5
:101A50000E946D4264EF76E0CE0145960E94B1424D
:101A6000BE016B5E7F4F82E491E10E946054811160
:101A700016C068E27BE0CE0101960E94B142BE0131
:101A80006F5F7F4F82E491E10E94605411E0811109
:101A900001C010E0CE0101960E946D4201C011E02C
:101AA000CE0145960E946D42112309F4B4C042E074
:101AB00050E062E471E1CE0101960E94D96FBE014F
:101AC0006F5F7F4F84E291E10E943441CE01019625
:101AD0000E946D4264E271E1CE0101960E94A9422A
:101AE000CE0101960E94FB59CE0101960E946D42E3
:101AF0000E94C88220E030E048EC52E40E94B99590
:101B00000E944398AB01BC0140936F045093700452
:101B10006093710470937204CE0101960E94346B3D
:101B2000CE0101960E94FB59CE0101960E946D42A2
:101B300060916F04709170048091710490917204AF
:101B40008B019C0100591F452140310901341C497A
:101B50002105310588F067EC76E0CE0101960E9400
:101B6000B14264E271E1CE0101960E94D9416AED71
:101B700076E00E94C241B7C11A821982FE013396F3
:101B800026E0DF011D922A95E9F70E945A9520E090
:101B900030E048EC52E40E94AA978E010F5F1F4F7D
:101BA00022E047E00E94C490BC018AE291E10E94D9
:101BB00043426AEE76E0CE0145960E94B1426AE267
:101BC00071E1CE0145960E94D94167EF76E00E940F
:101BD000C241BC018AE291E10E945842CE01459681
:101BE0000E946D421092400C10923F0C80916F0445
:101BF00090917004A0917104B09172048093AC0C28
:101C00009093AD0CA093AE0CB093AF0C80E090E03D
:101C10000E94E76E71C16CEF76E0CE0145960E949E
:101C2000B142BE016B5E7F4F82E491E10E9460543D
:101C3000811116C062E077E0CE0101960E94B142A8
:101C4000BE016F5F7F4F82E491E10E94605411E01A
:101C5000811101C010E0CE0101960E946D4201C0C9
:101C600011E0CE0145960E946D42112309F465C032
:101C700026E030E045E050E062E471E1CE010196FB
:101C80000E94C542BE016F5F7F4F84E291E10E94D6
:101C90003441CE0101960E946D4284E291E10E949E
:101CA000B8406B017C016FE276E0CE0101960E94A4
:101CB000B142CE0101960E94D482AC014F5F5F4FCA
:101CC00062E471E1CE0145960E94D96FBE016B5E60
:101CD0007F4F84E291E10E943441CE0145960E94FB
:101CE0006D42CE0101960E946D4284E291E10E9414
:101CF000B8409B01E3E3F4E041E050E0A0913304FD
:101D0000B0913404A417B5075CF0A281B3812A17FF
:101D10003B0711F4138212824F5F5F4F3296EECF72
:101D20009601220F331FF901ED5CFB4F7183608335
:101D300082E090E00E9427762AC568E077E0CE0135
:101D400045960E94B142BE016B5E7F4F82E491E1F5
:101D50000E946054811116C06EE077E0CE010196BA
:101D60000E94B142BE016F5F7F4F82E491E10E9409
:101D7000605411E0811101C010E0CE0101960E9473
:101D80006D4201C011E0CE0145960E946D421123C3
:101D900039F1E3E3F4E081E090E020913304309105
:101DA00034042817390774F0863091051CF49383A6
:101DB000828305C09C012E5F3F4F338322830196AF
:101DC0003296EBCF82E090E00E9427761092400C92
:101DD00010923F0C80E090E00E94E76E0C94701D22
:101DE00064E177E0CE0145960E94B142BE016B5E90
:101DF0007F4F82E491E10E946054811116C06BE133
:101E000077E0CE0101960E94B142BE016F5F7F4F25
:101E100082E491E10E94605411E0811101C010E060
:101E2000CE0101960E946D4201C011E0CE0145969F
:101E30000E946D421123F9F08091AA0C9091AB0C95
:101E4000892BA1F481E090E09093AB0C8093AA0CD5
:101E50008EED93E09093400C80933F0C0E940F6FA7
:101E600068EC70E080E090E00E94E684E0E0F0E062
:101E700019950C94721D62E277E0CE0145960E949E
:101E8000B142BE016B5E7F4F82E491E10E946054DB
:101E9000811116C06AE277E0CE0101960E94B1423C
:101EA000BE016F5F7F4F82E491E10E94605411E0B8
:101EB000811101C010E0CE0101960E946D4201C067
:101EC00011E0CE0145960E946D421123A1F162E31B
:101ED00077E0CE0101960E94B14269E172E1CE0144
:101EE00001960E94D941BC018AE291E10E945842C8
:101EF000CE0101960E946D426BE67AE0CE0101961A
:101F00000E94B1426AE271E1CE0101960E94D9417C
:101F1000BC01CE0145960E94A942CE0145960E9481
:101F20007258CE0145960E946D42CE0101960E94E4
:101F30006D420C94701D6CE377E0CE0145960E94D3
:101F4000B142BE016B5E7F4F82E491E10E9460541A
:101F5000811116C063E477E0CE0101960E94B14280
:101F6000BE016F5F7F4F82E491E10E94605411E0F7
:101F7000811101C010E0CE0101960E946D4201C0A6
:101F800011E0CE0145960E946D42112349F069E8A7
:101F900075E0CE0101960E94B1426FE172E19FCFE0
:101FA0006AE477E0CE0145960E94B142BE016B5EC5
:101FB0007F4F82E491E10E946054811116C06FE46A
:101FC00077E0CE0101960E94B142BE016F5F7F4F64
:101FD00082E491E10E94605411E0811101C010E09F
:101FE000CE0101960E946D4201C011E0CE014596DE
:101FF0000E946D421123C1F16FE276E0CE0101969D
:102000000E94B142CE0101960E94D482AC014F5F82
:102010005F4F62E471E1CE0145960E94D96FBE0127
:102020006B5E7F4F84E291E10E943441CE01459680
:102030000E946D42CE0101960E946D4284E291E1C0
:102040000E94B8406115710521F481E080938504F8
:1020500007C06130710511F00C94701D1092850459
:102060000E94DF740C94701D64E577E0CE01459604
:102070000E94B142BE016B5E7F4F82E491E10E94FB
:102080006054811116C068E577E0CE0101960E9488
:10209000B142BE016F5F7F4F82E491E10E946054C4
:1020A00011E0811101C010E0CE0101960E946D4245
:1020B00001C011E0CE0145960E946D42112309F442
:1020C00024C143E050E062E471E1CE0101960E9438
:1020D000D96FBE016F5F7F4F84E291E10E9434416E
:1020E000CE0101960E946D4264E271E1CE0101963B
:1020F0000E94A942CE0101960E94FB59CE01019691
:102100000E946D421092400C10923F0C64E271E10B
:1021100085E292E10E94584264E271E18FE192E12E
:102120000E94584288EC9CE0009739F048E050E06B
:10213000BC0185E292E10E947B5486E29DE000971B
:1021400039F04CE050E0BC018FE192E10E947B54F9
:1021500080913F0C9091400C0E94E76E6CE577E017
:10216000CE0101960E94B1426FE172E1CE0101966B
:102170000E94D941BC01CE0183960E94A942CE01A2
:1021800001960E946D428091220D9091230D892B22
:1021900039F4BE016D5D7F4F8CEC9DE00E940F43D2
:1021A0008091220D9091230D029709F09BC06FE161
:1021B00072E1CE0189960E94A94264E677E0CE01E1
:1021C00001960E94B142CE0101960E94FB8DCE0184
:1021D00001960E946D4264EF71E080E090E00E9401
:1021E000E68467E677E0CE0101960E94B142CE0117
:1021F00001960E94FB8DCE0101960E946D4264EF14
:1022000071E080E090E00E94E68460E777E0CE0134
:1022100001960E94B142CE0101960E94FB8DCE0133
:1022200001960E946D4264EF71E080E090E00E94B0
:10223000E68469E777E0CE0101960E94B142CE01C3
:1022400001960E94FB8DCE0101960E946D4264EFC3
:1022500071E080E090E00E94E68467E877E0CE01DC
:1022600001960E94B142CE0101960E94FB8DCE01E3
:1022700001960E946D4264EF71E080E090E00E9460
:10228000E6846CE577E0CE0101960E94B142BE0182
:10229000675D7F4FCE0101960E94D941BC01CE01FE
:1022A00045960E94A942CE0101960E946D42CE0140
:1022B00045960E94C340BE016B5E7F4FCE010196E2
:1022C0000E94A942CE0101960E94FB8DCE0101968B
:1022D0000E946D42CE0145960E946D42CE018996C4
:1022E0000E946D4268EC7CE0CE0101960E94B142F2
:1022F000CE0101960E94FB59CE0101960E946D42CB
:1023000010921202CE01839696C065E977E0CE0165
:1023100045960E94B142BE016B5E7F4F82E491E11F
:102320000E946054811116C06AE977E0CE010196DF
:102330000E94B142BE016F5F7F4F82E491E10E9433
:10234000605411E0811101C010E0CE0101960E949D
:102350006D4201C011E0CE0145960E946D421123ED
:1023600009F46DC044E050E062E471E1CE010196F1
:102370000E94D96FBE016F5F7F4F84E291E10E949E
:102380003441CE0101960E946D426FE977E0CE01A3
:1023900045960E94B14264E271E1CE0145960E94E9
:1023A000D941BC01CE0101960E94A942CE014596B9
:1023B0000E946D428091220D9091230D892B39F45A
:1023C000BE016F5F7F4F8CEC9DE00E940F4368EB76
:1023D0007BE080E090E00E94E6848091220D909165
:1023E000230D029779F4BE016F5F7F4FCE014596B2
:1023F0000E94A942CE0145960E94FB8DCE014596D2
:102400000E946D4268EB7BE080E090E00E94E684F1
:10241000BE016F5F7F4FCE0145960E94A942CE015B
:1024200045960E94FB59CE0145960E946D4210923E
:102430001202CE0101960E946D420C94721D66EA52
:1024400077E0CE0145960E94B142BE016B5E7F4FA0
:1024500082E491E10E946054811116C06AEA77E03B
:10246000CE0101960E94B142BE016F5F7F4F82E4B0
:1024700091E10E94605411E0811101C010E0CE0191
:1024800001960E946D4201C011E0CE0145960E9466
:102490006D42112309F456C062E471E184E291E1D6
:1024A0000E94584281E08093120262E471E1CE0101
:1024B00001960E94A942CE0101960E94FB59CE01CD
:1024C00001960E946D428091220D9091230D0297FA
:1024D000A1F064E271E18CEC9DE00E940F4368EB97
:1024E0007BE080E090E00E94E6840E94A14960EDDC
:1024F00077E080E090E00E94E6848091220D909148
:10250000230D029771F464E271E1CE0101960E94FD
:10251000A942CE0101960E94FB8DCE0101960E9438
:102520006D428091461190914711892B11F40C94C2
:10253000701D6BE67AE0CE0101960E94B14262E422
:1025400071E1E2CC6EEA77E0CE0145960E94B1429D
:10255000BE016B5E7F4F82E491E10E946054811165
:1025600016C064EB77E0CE0101960E94B142BE0135
:102570006F5F7F4F82E491E10E94605411E081110E
:1025800001C010E0CE0101960E946D4201C011E031
:10259000CE0145960E946D42112309F461C08091DD
:1025A000220D9091230D019711F00C94701DCE0116
:1025B00001960E9422628D819E81009711F40C94F5
:1025C0006C1DE981FA812081222311F40C946C1D89
:1025D000079710F40C946C1D6AE374E0CE014596E5
:1025E0000E94A14248EC50E06FEF7FEFCE0145968C
:1025F0000E94CC5ACE0145960E946D42BE016F5F8B
:102600007F4FCE0145960E94A94240ED57E06FEF03
:102610007FEFCE0145960E945E6FCE0145960E94E7
:102620006D426AEB77E0CE0145960E94B14262E4CA
:1026300071E1CE0145960E94D941BC01CE0183963D
:102640000E94A942CE0183960E947258CE018396C1
:102650000E946D42CE0145960E946D420C946C1D05
:1026600068EC77E0CE0145960E94B142BE016B5EF8
:102670007F4F82E491E10E946054811116C06DEC9D
:1026800077E0CE0101960E94B142BE016F5F7F4F9D
:1026900082E491E10E94605411E0811101C010E0D8
:1026A000CE0101960E946D4201C011E0CE01459617
:1026B0000E946D421123F1F025E030E044E050E04B
:1026C00062E471E1CE0101960E94C542BE016F5FD6
:1026D0007F4F84E291E10E943441CE0101960E9435
:1026E0006D4284E291E10E94B8407093230D6093A3
:1026F000220D4DC062ED77E0CE0145960E94B142B9
:10270000BE016B5E7F4F82E491E10E9460548111B3
:1027100016C067ED77E0CE0101960E94B142BE017E
:102720006F5F7F4F82E491E10E94605411E081115C
:1027300001C010E0CE0101960E946D4201C011E07F
:10274000CE0145960E946D42112381F126E030E0D2
:1027500044E050E062E471E1CE0101960E94C5427E
:10276000BE016F5F7F4F84E291E10E943441CE0150
:1027700001960E946D4284E291E10E94B8407093FC
:10278000250D6093240D709346046093450462E424
:1027900071E1CE0101960E94A942CE0101960E94EC
:1027A000FB59CE0101960E946D4210CB6CED77E093
:1027B000CE0145960E94B142BE016B5E7F4F82E41E
:1027C00091E10E946054811116C063EE77E0CE0162
:1027D00001960E94B142BE016F5F7F4F82E491E19A
:1027E0000E94605411E0811101C010E0CE010196F9
:1027F0000E946D4201C011E0CE0145960E946D42DB
:10280000112369F127E030E046E050E062E471E135
:10281000CE0101960E94C542BE016F5F7F4F84E2E8
:1028200091E10E943441CE0101960E946D4284E202
:1028300091E10E94B840672B19F41092800C03C0FC
:1028400081E08093800C62E471E1CE0101960E94E8
:10285000A942CE0101960E94FB590C946C1D6AEEB0
:1028600077E0CE0183960E94B142BE016D5D7F4F3D
:1028700082E491E10E94605481112BC06DEE77E0FB
:10288000CE0145960E94B142BE016B5E7F4F82E44D
:1028900091E10E946054811116C060EF77E0CE0193
:1028A00001960E94B142BE016F5F7F4F82E491E1C9
:1028B0000E94605411E0811101C010E0CE01019628
:1028C0000E946D4201C011E0CE0145960E946D420A
:1028D00001C011E0CE0183960E946D42112309F4DC
:1028E0002BC1BAE0AB2EB12CC12CD12C760188249F
:1028F0008A9403E0902E6EE170E080E090E00E9408
:10290000E684809110020E949C84B4010E94259A62
:10291000072E000C880B990B0E945A9520E030E09E
:1029200040EA50E40E94B9959B01AC01C701B60191
:102930000E94E4966B017C01F1E0AF1AB108D9F670
:1029400020E030E040E251E40E94AA976B017C0154
:1029500063EF77E0CE0145960E94B142BE016B5E07
:102960007F4F82E491E10E946054811116C067EFAD
:1029700077E0CE0101960E94B142BE016F5F7F4FAA
:1029800082E491E10E94605401E0811101C000E005
:10299000CE0101960E946D4201C0012FCE014596E5
:1029A0000E946D42002309F43FC020E030E040E681
:1029B00050E4C701B6010E94B9959B01AC0160E0EB
:1029C00070E080E890E40E94E396AB01BC01409384
:1029D0000C0250930D0260930E0270930F0222E0DE
:1029E000CE0101960E947242BE016F5F7F4F8AE264
:1029F00091E10E943441CE0101960E946D426BEF3D
:102A000077E0CE0101960E94B1426AE271E1CE0107
:102A100001960E94D941BC018AE291E10E9458428C
:102A2000CE0101960E946D426AE078E0CE014596A3
:102A30000E94B142BE016B5E7F4F82E491E10E9431
:102A40006054811115C06FE078E0CE0101960E94BC
:102A5000B142BE016F5F7F4F82E491E10E946054FA
:102A600011E0811101C010E0CE0101960E946D427B
:102A7000CE0145960E946D42112309F43FC020E02B
:102A800030E040E650E4C701B6010E94B9959B01D1
:102A9000AC0160E070E080E291E40E94E396AB015B
:102AA000BC01409308025093090260930A0270939C
:102AB0000B0222E0CE0101960E947242BE016F5FBE
:102AC0007F4F8AE291E10E943441CE0101960E943B
:102AD0006D4264E178E0CE0101960E94B1426AE263
:102AE00071E1CE0101960E94D941BC018AE291E1D7
:102AF0000E945842CE0101960E946D426BE67AE038
:102B0000CE0101960E94B1426AE271E1CE010196C6
:102B10000E94D941BC01CE0145960E94A942CE0136
:102B200045960E947258CE0145960E946D42CE0194
:102B300001960E946D42D6C764E278E0CE0101960C
:102B40000E94B142BE016F5F7F4F82E491E10E941B
:102B50006054182FCE0101960E946D42112309F492
:102B60006CC08091461190914711079708F4BAC73D
:102B700046E050E062E471E1CE0101960E94D96F17
:102B8000BE016F5F7F4F84E291E10E943441CE012C
:102B900001960E946D420E94C882AB01BC01409325
:102BA0001702509318026093190270931A0221E0E1
:102BB000CE0145960E94724261EA76E0CE0101960E
:102BC0000E94B142BE016B5E7F4FCE0101960E9412
:102BD000D94166EE78E00E94C241BC018AE291E1EF
:102BE0000E945842CE0101960E946D42CE01459648
:102BF0000E946D426AE271E1CE0101960E94A942F3
:102C0000CE0101960E947258CE0101960E946D423B
:102C10000E941E8528EE33E040E050E00E94B2960C
:102C2000CA01B9010E9458956093E40B7093E50BBB
:102C30008093E60B9093E70B55C76BE278E0CE01EB
:102C400001960E94B142BE016F5F7F4F82E491E125
:102C50000E946054182FCE0101960E946D421123EC
:102C600009F448C08091461190914711079708F4E4
:102C700039C746E050E062E471E1CE0101960E945E
:102C8000D96FBE016F5F7F4F84E291E10E943441B2
:102C9000CE0101960E946D420E94C882AB01BC0128
:102CA000409313025093140260931502709316021E
:102CB00021E0CE0145960E94724261EB76E0CE01A2
:102CC00001960E94B142BE016B5E7F4FCE0101961C
:102CD0000E94D94166EE78E00E94C241BC018AE2BE
:102CE00091E10E945842CE0101960E946D42CE01B0
:102CF0004596E6C68E010B5E1F4F62E378E0C80181
:102D00000E94B142B80182E491E10E9460548111B5
:102D100017C066E378E0CE0101960E94B142BE0181
:102D20006F5F7F4F82E491E10E946054FF24F3942F
:102D3000811101C0F12CCE0101960E946D4202C0AA
:102D4000FF24F394C8010E946D42FF2009F455C08E
:102D500080910602909107020E94FC7760935B04C9
:102D600070935C0480935D0490935E046093C00C48
:102D70007093C10C8093C20C9093C30C80E090E0E0
:102D8000A0E8BFE38093630490936404A093650478
:102D9000B09366048093B80C9093B90CA093BA0CCE
:102DA000B093BB0C8091800C882381F06EE174E0BD
:102DB00083EA9FE00E941D4360915B0470915C0474
:102DC00080915D0490915E040E94FC4F1092400C33
:102DD00010923F0C80E090E00E94E76E40915B040F
:102DE00050915C0460915D0470915E0422E0C80122
:102DF0000E9472426AE378E050C663E478E0C8015A
:102E00000E94B142B80182E491E10E9460548111B4
:102E100017C069E478E0CE0101960E94B142BE017C
:102E20006F5F7F4F82E491E10E946054FF24F3942E
:102E3000811101C0F12CCE0101960E946D4202C0A9
:102E4000FF24F394C8010E946D42FF2009F4B8C02A
:102E500080914611909147110797E8F046E050E0C5
:102E600062E471E1CE0101960E94D96FBE016F5FED
:102E70007F4F84E291E10E943441CE0101960E948D
:102E80006D420E94C88260934B0470934C048093FF
:102E90004D0490934E04809104029091050299276D
:102EA0000E943B77BC01990F880B990B0E945A95A1
:102EB0002DE038E643E55BE30E94B9956B017C01A8
:102EC00020919E0430919F044091A0045091A10450
:102ED0000E94549518164CF06091860470918704F6
:102EE00080918804909189041BC02091B204309194
:102EF000B3044091B4045091B504C701B6010E94D7
:102F0000999887FF05C0C701B6010E94A56D08C04A
:102F100060919A0470919B0480919C0490919D040F
:102F200020E030E048EC52E40E94B9956B017C014E
:102F300020E030E0A9010E945495181634F0C12C0D
:102F4000D12CA8EAEA2EA1E4FA2EC0924B04D0922A
:102F50004C04E0924D04F0924E04C092E00CD092EA
:102F6000E10CE092E20CF092E30C8091800C88235B
:102F700081F06CE074E083EA9FE00E941D43609161
:102F80004B0470914C0480914D0490914E040E942A
:102F9000FC4F1092400C10923F0C80E090E00E9499
:102FA000E76E40914B0450914C0460914D04709138
:102FB0004E0422E0C8010E9472426FE478E06DC5C1
:102FC00069E578E0C8010E94B142B80182E491E16C
:102FD0000E946054811117C06EE578E0CE01019621
:102FE0000E94B142BE016F5F7F4F82E491E10E9477
:102FF0006054FF24F394811101C0F12CCE0101969D
:103000000E946D4202C0FF24F394C8010E946D42E9
:10301000FF2009F494C080914611909147110697C2
:10302000F8F045E050E062E471E1CE0101960E94C3
:10303000D96FBE016F5F7F4F84E291E10E943441FE
:10304000CE0101960E946D420E94C8820E94DA98C9
:1030500060935304709354048093550490935604E2
:103060008091BE049091BF040E945B9020E030E00C
:1030700048E051E40E94AA976093BA047093BB049D
:103080008093BC049093BD046093D00C7093D10CDA
:103090008093D20C9093D30C80915304909154045C
:1030A000A0915504B09156048093D80C9093D90CFC
:1030B000A093DA0CB093DB0C8091800C882341F153
:1030C0006BEF73E083EA9FE00E941D43209153045D
:1030D00030915404409155045091560460E070E0E2
:1030E00080E291E40E94589941E050E00E947F6C98
:1030F00063E678E083EA9FE00E94E8436091BA04C7
:103100007091BB048091BC049091BD040E94FC4F5F
:103110001092400C10923F0C80E090E00E94E76E0D
:103120004091BA045091BB046091BC047091BD04FD
:1031300023E0C8010E9472426AE678E0BEC065E7FB
:1031400078E0C8010E94B142B80182E491E10E9496
:103150006054811117C06AE778E0CE0101960E94A1
:10316000B142BE016F5F7F4F82E491E10E946054E3
:10317000FF24F394811101C0F12CCE0101960E942D
:103180006D4202C0FF24F394C8010E946D42FF20EB
:1031900009F49FC080914611909147110697F8F06D
:1031A00045E050E062E471E1CE0101960E94D96FE2
:1031B000BE016F5F7F4F84E291E10E943441CE01F6
:1031C00001960E946D420E94C8820E94DA98609324
:1031D0004F04709350048093510490935204809153
:1031E000BE049091BF040E945B9020E030E048E074
:1031F00051E40E94AA976093B6047093B704809339
:10320000B8049093B9046093D40C7093D50C809358
:10321000D60C9093D70C80914F0490915004A091BC
:103220005104B09152048093DC0C9093DD0CA09378
:10323000DE0CB093DF0C8091800C882341F16BEEA3
:1032400073E083EA9FE00E941D4320914F04309178
:103250005004409151045091520460E070E080E2CB
:1032600091E40E94589941E050E00E947F6C63E62F
:1032700078E083EA9FE00E94E8436091B604709191
:10328000B7048091B8049091B9040E94FC4F109249
:10329000400C10923F0C80E090E00E94E76E40915D
:1032A000B6045091B7046091B8047091B90423E05A
:1032B000C8010E9472426FE778E0CE0101960E9439
:1032C000B142B801CE0101960E94D94163E778E08E
:1032D00097C068E878E0C8010E94B142B80182E472
:1032E00091E10E946054811117C06CE878E0CE0132
:1032F00001960E94B142BE016F5F7F4F82E491E16F
:103300000E946054FF24F394811101C0F12CCE017E
:1033100001960E946D4202C0FF24F394C8010E94EE
:103320006D42FF2009F46FC09090020260E0892D89
:103330000E946084F9E1AF2EB12CC12CD12C760112
:10334000892D0E949C84BC01990F880B990B0E94C7
:103350005A959B01AC01C701B6010E94E4966B012E
:103360007C016AE070E080E090E00E94E68441E049
:10337000A41AB10829F720E030E040EA50E4C70180
:10338000B6010E94B99520E030E040E85AE30E947F
:10339000B99520E030E048EC51E40E94AA97609390
:1033A0004704709348048093490490934A046093BF
:1033B000F60C7093F70C8093F80C9093F90C109224
:1033C000400C10923F0C80E090E00E94E76E40912C
:1033D0004704509148046091490470914A0422E0E6
:1033E000C8010E94724268E376E0CE0101960E9415
:1033F000B142B801CE0101960E94D94165E076E064
:103400000E94C24153C360E978E0C8010E94B14202
:10341000B80182E491E10E946054811117C064E90F
:1034200078E0CE0101960E94B142BE016F5F7F4FEE
:1034300082E491E10E946054FF24F394811101C061
:10344000F12CCE0101960E946D4202C0FF24F3943C
:10345000C8010E946D42FF2009F43CC126E030E023
:1034600044E050E062E471E1CE0101960E94C54261
:10347000BE016F5F7F4F84E291E10E943441CE0133
:1034800001960E946D4284E291E10E94B8404B0196
:103490005C016B016FE276E0CE0101960E94B142C1
:1034A000CE0101960E94D482AC014F5F5F4F62E46F
:1034B00071E1C8010E94D96FB80184E291E10E94D4
:1034C0003441C8010E946D42CE0101960E946D42B6
:1034D000F09000020E94C8822B013C01140161E0BF
:1034E000261A31088091800C8823B9F063E773E0D5
:1034F00083EA9FE00E941D434AE050E0B40183EA62
:103500009FE00E949E4360E27BE083EA9FE00E948E
:10351000E843C301B2010E94FC4F6F2DC8010E9415
:10352000FE7B18870F831D821E82198289E08A83A1
:1035300081E08B838C831C8A1B8ACE0101960E94BA
:103540005052CE0101960E94E051CE0101960E9498
:103550000551EE80F12C7BE0E716F1041CF0EAE067
:10356000EE2EF12C8BE58816910408F44CC077E11F
:10357000A72E7CE0B72E4501412C512C3201C12CE5
:10358000D12CCE14DF04BCF46C2DCE0101960E9428
:1035900095509B01AC01D4016D937D938D939D93C8
:1035A0004D01C301B2010E94E4962B013C01BFEF23
:1035B000CB1ADB0AE6CFB7010F2C000C880B990B56
:1035C0000E945A959B01AC01C301B2010E94AA97C7
:1035D0002B013C01C12CD12CCE14DF040CF058C0BF
:1035E000F5012081318142815381C301B2010E94E2
:1035F000E396D5016D937D938D939D935D01BFEF10
:10360000CB1ADB0AE9CF1C141D0414F5EC14FD04DD
:1036100024F41701E1E02E1A3108622DCE01019643
:103620000E9495509B01AC01C101880F991F880F22
:10363000991FBC01695E734F1B01C301B2010E9457
:10364000E396D1016D937D938D939C93139720C046
:10365000CD28F1F487E1A82E8CE0B82EC12CD12C16
:10366000CE14DF04ACF46C2DCE0101960E9495506F
:103670009B01AC01C301B2010E94E396F501619385
:103680007193819391935F01FFEFCF1ADF0AE8CF27
:10369000E7E1FCE0AAEFBCE04191519161917191A9
:1036A0004D935D936D937D934CE0EF33F407A1F759
:1036B0001092400C10923F0C80E090E00E94E76E68
:1036C00044E050E062E471E1C8010E94D96F68E90A
:1036D00078E0E3C169EB78E0C8010E94B142B8012B
:1036E00082E491E10E946054811117C06DEB78E093
:1036F000CE0101960E94B142BE016F5F7F4F82E40E
:1037000091E10E946054FF24F394811101C0F12CD7
:10371000CE0101960E946D4202C0FF24F394C801BD
:103720000E946D42FF2009F455C0809106029091DD
:1037300007020E94FC7760935704709358048093AB
:10374000590490935A046093C40C7093C50C8093F1
:10375000C60C9093C70C80E090E5A3ECB7E480938F
:103760005F0490936004A0936104B093620480931B
:10377000BC0C9093BD0CA093BE0CB093BF0C809179
:10378000800C882381F06DEC73E083EA9FE00E9457
:103790001D43609157047091580480915904909191
:1037A0005A040E94FC4F1092400C10923F0C80E093
:1037B00090E00E94E76E4091570450915804609148
:1037C000590470915A0422E0C8010E94724261ECCF
:1037D00078E063C16CEC78E0C8010E94B142B801A6
:1037E00082E491E10E946054811117C060ED78E09D
:1037F000CE0101960E94B142BE016F5F7F4F82E40D
:1038000091E10E946054FF24F394811101C0F12CD6
:10381000CE0101960E946D4202C0FF24F394C801BC
:103820000E946D42FF2009F484C08091461190915E
:1038300047110497E8F044E050E062E471E1CE0102
:1038400001960E94D96FBE016F5F7F4F84E291E1C4
:103850000E943441CE0101960E946D420E94C882AE
:10386000609363047093640480936504909366048A
:103870008091630490916404A0916504B091660402
:103880008093B80C9093B90CA093BA0CB093BB0C76
:103890008091800C882391F064EB73E083EA9FE0D1
:1038A0000E941D43609163047091640480916504DB
:1038B0009091660442E050E00E947F6C8091060285
:1038C000909107020E94FC7760935B0470935C0404
:1038D00080935D0490935E046093C00C7093C10C60
:1038E0008093C20C9093C30C8091800C882381F04C
:1038F0006AEA73E083EA9FE00E941D4360915B04E3
:1039000070915C0480915D0490915E040E94FC4F74
:103910001092400C10923F0C80E090E00E94E76E05
:1039200040915B0450915C0460915D0470915E0471
:10393000AEC06CED78E0C8010E94B142B80182E4EB
:1039400091E10E946054811117C060EE78E0CE01D1
:1039500001960E94B142BE016F5F7F4F82E491E108
:103960000E946054FF24F394811101C0F12CCE0118
:1039700001960E946D4202C0FF24F394C8010E9488
:103980006D42FF2009F4AEC080914611909147111D
:103990000497E8F044E050E062E471E1CE01019662
:1039A0000E94D96FBE016F5F7F4F84E291E10E9458
:1039B0003441CE0101960E946D420E94C8826093FC
:1039C0005F0470936004809361049093620480911B
:1039D0005F0490916004A0916104B09162048093AF
:1039E000BC0C9093BD0CA093BE0CB093BF0C809107
:1039F000800C882391F061E973E083EA9FE00E94E4
:103A00001D4360915F047091600480916104909106
:103A1000620442E050E00E947F6C80910602909127
:103A200007020E94FC7760935704709358048093B8
:103A3000590490935A046093C40C7093C50C8093FE
:103A4000C60C9093C70C8091800C882381F067E8A6
:103A500073E083EA9FE00E941D43609157047091D8
:103A600058048091590490915A040E94FC4F10927E
:103A7000400C10923F0C80E090E00E94E76E409175
:103A80005704509158046091590470915A0422E0EF
:103A9000C8010E94724264ED78E0CE0101960E9456
:103AA000B142B801CE0101960E94D941BC018AE21F
:103AB00091E10E945842CE0101960E946D42C801D8
:103AC0000E946D426AE271E1CE0101960E94A94214
:103AD000CE0101960E947258CE0101960E946D425D
:103AE0001092120280911202882371F062E471E157
:103AF000CE0101960E94A942CE0101960E94FB5977
:103B0000CE0101960E946D420E941E856093E80BD3
:103B10007093E90B8093EA0B9093EB0BEA960FB648
:103B2000F894DEBF0FBECDBFDF91CF911F910F91F3
:103B3000FF90EF90DF90CF90BF90AF909F908F90CD
:103B40007F906F905F904F903F902F9008952F92AD
:103B50003F924F925F926F927F928F929F92AF921D
:103B6000BF92CF92DF92EF92FF920F931F93CF936A
:103B7000DF93CDB7DEB7CD54D1090FB6F894DEBFD1
:103B80000FBECDBF26969FAF8EAF2697E0900F0C4D
:103B9000F090100C8091800C882361F06EE176E04B
:103BA00083EA9FE00E941D4326968EAD9FAD269727
:103BB0000E94B95926960EAD1FAD26970B5F1F4F79
:103BC0000530110540F180910F0C9091100C269654
:103BD0002EAD3FAD26972817390739F10E942F6F78
:103BE0000E94D07426964EAD5FAD26975093100C70
:103BF00040930F0CBA01CE0101960E94BB58BE0142
:103C00006F5F7F4F86E391E10E943441CE010196C0
:103C10000E946D420AC026968EAD9FAD26970296F1
:103C200021F40E94DF740C94B23164E77BE08AE2F5
:103C300091E10E9443420530110590F060E27BE083
:103C4000CE0101960E94B1424AE050E06FEF7FEF53
:103C5000CE0101960E94CC5ACE0101960E946D427F
:103C60002696EEADFFAD26977996E533F10510F077
:103C70000C94C0308827EE58FF4F8F4F0C94389A21
:103C80008091850C882309F426C189E69EE00E9474
:103C9000FD5461E080912E040E94608460E0809178
:103CA0002C040E9460840E9413580E94EB5B0E94C7
:103CB000085CAB01BC0123E0CE0180960E947242F9
:103CC000BE01605E7F4FCE0101960E94A94267E26D
:103CD00079E0CE0101960E94C241BC0184E291E1EB
:103CE0000E945842CE0101960E946D42CE018096FC
:103CF0000E946D4261E279E0CE0101960E94B142DC
:103D000064E271E1CE0101960E94D941BC018AE2D0
:103D100091E10E945842CE0101960E946D420E949C
:103D2000085C6B017C010E94C1844B015C016EE167
:103D300070E080E090E00E94E6840E94085C2B0125
:103D40003C010E94C1849B01AC01281939094A0930
:103D50005B0949015A0131ED831637E09306A1044E
:103D6000B1040CF441C0A7019601C301B2010E9445
:103D7000E3966B017C0120E030E0A9010E94999854
:103D800018165CF426EA3BE944EC5BE3C701B60194
:103D90000E94549587FF0BC027C026EA3BE944ECFC
:103DA0005BEBC701B6010E9499981816ECF0C501AB
:103DB000B40128EE33E040E050E00E948696CA014C
:103DC000B9010E945A954B015C0120E030E04AE7BE
:103DD00054E4C701B6010E94B995A50194010E945F
:103DE000AA97AB01BC0103C040E050E0BA0122E059
:103DF000CE0180960E947242BE01605E7F4FCE016E
:103E000001960E94A94264EE78E0CE0101960E94DC
:103E1000C241BC018EE191E10E945842CE0101965F
:103E20000E946D42CE0180960E946D4268EE78E05D
:103E3000CE0101960E94B1426EE171E1CE01019680
:103E40000E94D941BC018AE291E10E94F841CE0171
:103E500001960E946D4260E27BE0CE0101960E94D5
:103E6000B1426EE171E1CE0101960E94D941BC01DF
:103E700084E291E10E94F841CE0101960E946D42D8
:103E800063E474E0CE0101960E94A1424AE050E052
:103E900060E070E0CE0101960E94275ACE010196A3
:103EA0000E946D4264E271E1CE0101960E94A94236
:103EB00045E050E06FEF7FEFCE0101960E945E6F0C
:103EC000CE0101960E946D426CEE78E08AE291E1AB
:103ED0000E94EA41E3C1C0901302D0901402E09026
:103EE0001502F09016020E941E856CAF7DAF8EAF5A
:103EF0009FAF89E69EE00E94FD5461E080912E0410
:103F00000E94608460E080912C040E9460840E9482
:103F100013580E94EB5B0E94085C24966CAF7DAF47
:103F20008EAF9FAF24970E94C1844B015C016AE071
:103F300070E080E090E00E94E6846FEF78E08AE233
:103F400091E10E94434220E030E04AE754E4C70197
:103F5000B6010E94B9952A966CAF7DAF8EAF9FAF28
:103F60002A97412C512C3201C12CD12C7601C7014A
:103F7000B6010E945A952A962CAD3DAD4EAD5FAD6F
:103F80002A970E94549587FF89C10E941E852CADF7
:103F90003DAD4EAD5FAD621B730B840B950B0E9464
:103FA000589520E030E04AE754E40E94AA97AB011C
:103FB000BC0123E0CE0101960E947242BE016F5FF8
:103FC0007F4F84E291E10E943441CE0101960E942C
:103FD0006D420E94085C6B017C010E94C1849B01C0
:103FE000AC01281939094A095B0949015A0131ED27
:103FF000831637E09306A104B1040CF443C020E01B
:1040000030E0A901C701B6010E94999818165CF426
:1040100026EA3BE944EC5BE3C701B6010E945495F4
:1040200087FF0BC02FC026EA3BE944EC5BEBC701DE
:10403000B6010E94999818162CF1C501B40128EE1A
:1040400033E040E050E00E948696CA01B9010E9428
:104050005A954B015C0124962CAD3DAD4EAD5FAD44
:104060002497C701B6010E94E39620E030E04AE7BA
:1040700054E40E94B995A50194010E94AA974B01AE
:104080005C0103C0812C912C540164E271E1CE01EA
:1040900001960E94A94266EE78E0CE0101960E9448
:1040A000C241BC0184E291E10E945842CE010196D6
:1040B0000E946D4223E0B701A601CE0180960E94C6
:1040C0007242BE01605E7F4FCE0101960E94A942FE
:1040D0006DE179E0CE0101960E94C241BC018EE102
:1040E00091E10E945842CE0101960E946D42CE019C
:1040F00080960E946D4222E0B501A401CE01019696
:104100000E9472426CE27BE0CE0180960E94B14236
:1041100064E271E1CE0180960E94D94160E279E0CB
:104120000E94C2416EE171E10E94D94169EE78E0DE
:104130000E94C241BE016F5F7F4F0E94D94164EE71
:1041400078E00E94C241BC018AE291E10E94F841FC
:10415000CE0180960E946D42CE0101960E946D4272
:1041600020E030E0A901C501B4010E94999887FDC3
:1041700006C060E27BE08EE191E10E94EA4122E02C
:10418000B501A401CE0180960E947242BE01605E1C
:104190007F4FCE0101960E94A94264EE78E0CE01E5
:1041A00001960E94C241BC018EE191E10E94F8415A
:1041B000CE0101960E946D42CE0180960E946D4212
:1041C0006AE271E1CE0101960E94A942CE010196F8
:1041D0000E947258CE0101960E946D42C301B20145
:1041E00025E030E040E050E00E948696672B682B87
:1041F000692B21F56AE474E0CE0101960E94A14288
:1042000045E050E060E070E0CE0101960E94275A40
:10421000CE0101960E946D426EE171E1CE010196E0
:104220000E94A94245E050E06FEF7FEFCE0101967A
:104230000E945E6FCE0101960E946D4264E77BE0B2
:104240008AE291E10E94434265E070E080E090E004
:104250000E94E6840E941E856B017C012CAD3DAD61
:104260004EAD5FADC21AD30AE40AF50A0E94085C9B
:1042700024966CAF7DAF8EAF9FAF24970E94C18410
:104280004B015C016AE070E080E090E00E94E6840F
:104290003FEF431A530A630A730A69CE60E08091C4
:1042A0002E040E9460840C94EE3080910002909164
:1042B00001020E9423780C94EE304091020227966E
:1042C0004FAF279760E0842F0E9460848091850C17
:1042D00081110BC08FE090E0A0E0B0E02E968CAF93
:1042E0009DAFAEAFBFAF2E970AC022E030E040E0F6
:1042F00050E02E962CAF3DAF4EAF5FAF2E9769E5E5
:1043000074E08AE291E10E94FE416AE271E1CE012D
:1043100001960E94A9424AE050E06FEF7FEFCE0184
:1043200001960E94275ACE0101960E946D421CAE52
:1043300021961FAE2197212C312CC12CD12C760136
:1043400002E310E0812C912C540127968FAD279722
:104350000E949C84092E000CAA0BBB0B880E991E90
:10436000AA1EBB1E65E070E080E090E00E94E6843B
:104370000150110951F74090470450904804609053
:10438000490470904A04C501B4010E945A9520E086
:1043900030E040EA50E40E94B99520E030E040E887
:1043A0005AE30E94B99520E030E048E452E40E94CC
:1043B000AA97A30192010E94E39620E030E040E733
:1043C00051E40E94B9954B015C01A30192016AE995
:1043D00079E989E390E40E94E3969B01AC01C50171
:1043E000B4010E94AA9720E030E0A9010E94E4965F
:1043F00020E030E040E251E40E94B9955B018C017D
:104400002CAD21963FAD2197A1010E9499981816D5
:104410002CF4ACAE2196BFAE2197180120E030E01D
:10442000A901B501C8010E94549587FF04C0A12CC1
:10443000B12C00E010E022E0A501B801CE01809689
:104440000E947242BE01605E7F4FCE0101960E94C3
:10445000A94264E279E0CE0101960E94C241BC010A
:1044600084E291E10E945842CE0101960E946D4281
:10447000CE0180960E946D4264E271E1CE01019608
:104480000E94A9424AE050E060E070E0CE0101964F
:104490000E945E6FCE0101960E946D420E941E85B1
:1044A0008090EC0B9090ED0BA090EE0BB090EF0B8A
:1044B000950184010C591F4F2F4F3F4F06171707C7
:1044C0002807390710F40C9413310E941E850E94AE
:1044D00058952B013C01C501B4010E945A9520E07A
:1044E00030E048EC51E40E94E4969B01AC01C3012A
:1044F000B2010E94549587FF02C00C9413316CE303
:1045000070E080E090E00E94E6843FEFC31AD30A97
:10451000E30AF30A2E968CAD9DADAEADBFAD2E97DE
:104520008C159D05AE05BF050CF00ACF64E670E062
:1045300080E090E00E94E6840E942F6F64E670E0C5
:1045400080E090E00E94E68461E574E084E291E11D
:104550000E94FE4164E271E1CE0101960E94A942EF
:1045600044E150E060E070E0CE0101960E94275ADD
:10457000CE0101960E946D4222E04CAD21965FADC6
:104580002197B101CE0180960E947242BE01605E09
:104590007F4FCE0101960E94A94264E279E0CE01EC
:1045A00001960E94C241BC0184E291E10E945842FE
:1045B000CE0101960E946D42CE0180960E946D420E
:1045C00064E271E1CE0101960E94A94242E350E00B
:1045D0006FEF7FEFCE0101960E945E6FCE010196D4
:1045E0000E946D4264E170E080E090E00E94E68409
:1045F0000E94506F6EE170E080E090E00E94E684DF
:104600006EE170E080E090E00E94E68469E279E08B
:10461000CE0101960E94B14264E271E1CE010196A1
:104620000E94D9416DE279E00E94C2416AE271E1E3
:104630000E94D941BC018AE291E10E9458420C9447
:104640009630809104029091050299270E943B7751
:10465000BC01990F880B990B0E945A952DE038E602
:1046600043E55BE30E94B9956B017C0120919E04B8
:1046700030919F044091A0045091A1040E94549550
:1046800018164CF06091860470918704809188041C
:10469000909189041BC02091B2043091B3044091E1
:1046A000B4045091B504C701B6010E94999887FFE0
:1046B00005C0C701B6010E94A56D08C060919A04AB
:1046C00070919B0480919C0490919D0420E030E0C7
:1046D00048EC52E40E94B99520E030E048EA51E409
:1046E0000E94B99520914B0430914C0440914D04A7
:1046F00050914E040E94AA976B017C0166E674E01B
:1047000084E291E10E94FE4164E271E1CE010196F2
:104710000E94A94242E350E060E070E0CE010196C1
:104720000E94275ACE0101960E946D4222E0B701F5
:10473000A601CE0101960E94724267E379E0CE01A4
:1047400080960E94B142BE016F5F7F4FCE0180967E
:104750000E94D94161E379E00E94C241BC018AE232
:1047600091E10E945842CE0180960E946D42CE0196
:1047700001960E946D426AE271E1CE0101960E94AB
:10478000A94242E350E06FEF7FEFCE0101960E9415
:104790005E6FCE0101960E946D428091850C882348
:1047A00011F40C94EE3060E273E080E090E0CBC254
:1047B0000E942F6F6AE974E08AE291E10E94FE4153
:1047C0006AE271E1CE0101960E94A9424AE050E0FE
:1047D00060E070E0CE0101960E94275ACE0101965A
:1047E0000E946D4261E974E084E291E10E94FE4121
:1047F00064E271E1CE0101960E94A94244E150E0D9
:104800006FEF7FEFCE0101960E945E6FCE010196A1
:104810000E946D428091F40B9091F50B82309105CE
:1048200049F40E940A8281111AC01092F50B10926D
:10483000F40B15C0892BC9F40E940A82882339F031
:1048400082E090E09093F50B8093F40B08C00E94F7
:104850000A828111F5CF0E940A828111F1CF8091E5
:10486000F40B9091F50B029741F165E874E08AE250
:1048700091E10E94FE416AE271E1CE0101960E943F
:10488000A9424AE050E060E070E0CE0101960E944B
:10489000275ACE0101960E946D426AE271E1CE0173
:1048A00001960E94A94260E27BE0CE0101960E943F
:1048B000C24164E271E10C94FD2D8AE090E00E9417
:1048C0000A756B017C0120E030E0A9010E9454953B
:1048D000181634F08AE090E00E940A756B017C01A2
:1048E0000BE010E020E030E042ED53E4C701B601F8
:1048F0000E945495181684F00150110969F068EC73
:1049000070E080E090E00E94E68483E090E00E9406
:104910000A756B017C01E6CF20E030E0A901C701F8
:10492000B6010E94549518163CF067E774E08AE2DD
:1049300091E10E94FE4131C020E030E048EC52E4B9
:10494000C701B6010E94549587FF02C021E001C053
:1049500020E0B701A601CE0101960E94724266E3F3
:1049600079E0CE0180960E94B142BE016F5F7F4F19
:10497000CE0180960E94D9416BE379E00E94C2414A
:10498000BC018AE291E10E945842CE0180960E94C9
:104990006D42CE0101960E946D426AE271E1CE0144
:1049A00001960E94A94242E350E06FEF7FEFCE01F3
:1049B00001960E945E6FCE0101960E946D426EE6E6
:1049C00074E084E291E10E94FE4164E271E1CE0173
:1049D00001960E94A94242E350E060E070E0CE01FF
:1049E00001960E94275AD5CE0E941E852B013C01BC
:1049F00089E69EE00E94FD5464E670E080E090E06D
:104A00000E94E68440E855E260E070E089E69EE0BE
:104A10000E94846E64E670E080E090E00E94E6848C
:104A200063ED74E084E291E10E94FE4164E271E191
:104A3000CE0101960E94A94242E350E06FEF7FEF62
:104A4000CE0101960E94275ACE0101960E946D4226
:104A500068EC74E084E291E10E94FE4164E271E15D
:104A6000CE0101960E94A94242E350E06FEF7FEF32
:104A7000CE0101960E945E6FCE0101960E946D42AA
:104A80008091150C9091160C8D7F1CAEC12CD12CF1
:104A9000E12CF12C00E010E0019709F479C0ACEDB5
:104AA0008A2EA5E09A2EA12CB12CDE019096B9AFEA
:104AB000A8AFFE017E96FBAFEAAF0E941E85DC0127
:104AC000CB0184199509A609B709883B9B40A1052C
:104AD000B10508F05DC089E69EE00E94733E892B17
:104AE00009F44FC080926D0E90926E0EA0926F0EE0
:104AF000B092700E0E94506E97FD06C082349105F0
:104B0000C9F780E090E002C08FEF9FEF892BC9F5D5
:104B10009E012F5F3F4F22963FAF2EAF2297190184
:104B20000E94506E97FF06C089818D3451F520E0B8
:104B300030E009C0D1018D931D01E8ADF9ADEA1750
:104B4000FB0771F7F1CF2296AEADBFAD22978D91E5
:104B50002296BFAFAEAF2297280F311DEAADFBAD55
:104B6000AE17BF0781F72E5B3F4F8E8D90E0982FD9
:104B700088274F8D840F911D2817390711F40C9445
:104B8000173162E370E080E090E00E94E68495CF08
:104B90000E941E85DC01CB0184199509A609B7097D
:104BA000883B9B40A105B10518F42CAD2111BDC077
:104BB0000E942F6F64E271E1CE0180960E94A942AB
:104BC00042E350E066E070E0CE0180960E94275AF2
:104BD000CE0180960E946D424CAD442311F40C949A
:104BE000303182E090E09093160C8093150CB60162
:104BF000CE0180960E94BB58B701CE0186960E94D6
:104C0000BB58B801CE01C2960E94BB58BE016E5C73
:104C10007F4FCE018C960E94A94262E278E0CE01DD
:104C20008C960E94C241BE016A5D7F4F0E94D941AD
:104C300062E278E00E94C241BE01605E7F4F0E9446
:104C4000D941BC018AE291E10E945842CE018C9682
:104C50000E946D42CE01C2960E946D42CE018696A0
:104C60000E946D42CE0180960E946D426AE271E11F
:104C7000CE0180960E94A9424AE050E06FEF7FEF9C
:104C8000CE0180960E945E6FCE0180960E946D429A
:104C900062EC74E08BE292E10E941D43B601CE010A
:104CA00080960E94BB58B701CE0186960E94BB58E1
:104CB000B801CE018C960E94BB586FE379E0CE011B
:104CC000C2960E94B142BE01645D7F4FCE01C29682
:104CD0000E94D94160E27BE00E94C241BE016A5D50
:104CE0007F4F0E94D94160E27BE00E94C241BE0139
:104CF000605E7F4F0E94D9416FE479E00E94C2411B
:104D0000BC018AE291E10E945842CE01C2960E9403
:104D10006D42CE018C960E946D42CE0186960E9415
:104D20006D42CE0180960E946D4262E370E080E0A9
:104D300090E00E94E68489E69EE00E94FD5462E3D2
:104D400070E080E090E00E94E6840C94EE300091E8
:104D500006021091070265E579E084E291E10E9484
:104D600043420E942F6F64E271E1CE0101960E94DE
:104D7000A9424AE050E06FEF7FEFCE0101960E941A
:104D8000275ACE0101960E946D42C8010E94FC770D
:104D900024966CAF7DAF8EAF9FAF249780905B045D
:104DA00090905C04A0905D04B0905E04A501940115
:104DB00060915704709158048091590490915A045D
:104DC0000E94E3962B013C0120E030E0A9010E9403
:104DD0005495882309F453C0C0906304D0906404B0
:104DE000E0906504F090660420E030E0A901C7017E
:104DF000B6010E94549518160CF041C080915F04D2
:104E000090916004A0916104B09162048CAF9DAF59
:104E1000AEAFBFAF9C01AD01C701B6010E94549572
:104E2000882369F1A70196016CAD7DAD8EAD9FAD74
:104E30000E94AA970E94E5986CAF7DAF8EAF9FAF9E
:104E4000A501940124966CAD7DAD8EAD9FAD2497E8
:104E50000E94E396A30192010E94AA972CAD3DAD5A
:104E60004EAD5FAD0E94B9950E9417989B01AC01B1
:104E7000C701B6010E94B9956B017C0103C0C12C2A
:104E8000D12C760164E271E1CE0101960E94A94223
:104E90004AE050E060E070E0CE0101960E94275A9F
:104EA000CE0101960E946D4220E030E64AEE56E4C3
:104EB000C701B6010E94999818163CF46FED74E092
:104EC0008AE291E10E94FE4125C021E0B701A601DE
:104ED000CE0180960E9472426FE579E0CE01019684
:104EE0000E94B142BE01605E7F4FCE0101960E94DA
:104EF000D94163E679E00E94C241BC018AE291E1B6
:104F00000E945842CE0101960E946D42CE018096C9
:104F10000E946D426AE271E1CE0101960E94A942AF
:104F20004AE050E06FEF7FEFCE0101960E945E6F86
:104F3000CE0101960E946D4264E670E080E090E050
:104F40000E94E6842ACC0091DE041091DF040E94C6
:104F50002F6FC8010E943B778C0162E370E080E014
:104F600090E00E94E684B801110F880B990B0E9413
:104F70005A9520E030E040EA50E40E94B99520E0E4
:104F800030EC4FE754E40E94AA97AB01BC0123E048
:104F9000CE0101960E9472426AE279E0CE018096CB
:104FA0000E94B142BE016F5F7F4FCE0180960E948A
:104FB000D94165E076E00E94C241BC018AE291E1FC
:104FC0000E945842CE0180960E946D42CE01019609
:104FD0000E946D4267E679E084E291E10E944342DB
:104FE00064E271E1CE0101960E94A9424AE050E0DC
:104FF00068E070E0CE0101960E94275ACE0101962A
:105000000E946D426AE271E1CE0101960E94A942BE
:105010004AE050E06FEF7FEFCE0101960E945E6F95
:10502000CE0101960E946D4264E271E18AE291E153
:105030000E94F841B2CB90910E0C81E089278093B9
:105040000E0C8091850C882331F06AE271E18CECC2
:105050009DE00E947A6A68EC70E080E090E073CE98
:105060001092850C0C94EE3081E08093850C66E301
:1050700071E18CE391E10E94584280910F0C909174
:10508000100C9093840C8093830C0C94EE308091E0
:105090008712882321F0109287120C94EE300E9420
:1050A000AE7E0C94EE3086E09FE00E94FD5440E01E
:1050B00052EC61E070E086E09FE00E94846E8CED2F
:1050C00095E0A0E0B0E080930A0F90930B0FA093BF
:1050D0000C0FB0930D0F64E670E080E090E00E944A
:1050E000E6848091F40B9091F50B019759F483E0DD
:1050F00090E00E945F77811140C01092F50B1092F2
:10510000F40B1AC081E090E00E945F77882339F0A9
:1051100081E090E09093F50B8093F40B0DC083E059
:1051200090E00E945F778111F3CF83E090E00E94CE
:105130005F778111EDCF06C08091F40B9091F50B54
:105140000197D9F06EE175E084E291E10E94FE41A1
:1051500064E271E1CE0101960E94A94244E150E06F
:105160006FEF7FEFCE0101960E945E6FCE01019638
:105170000E946D4262E175E0CFC066E075E08AE2B0
:1051800091E10E94FE416AE271E1CE0101960E9426
:10519000A942CE0101960E94FB59CE0101960E94C0
:1051A0006D4262E370E080E090E00E94E6846AE293
:1051B00071E1CE0101960E94A94242E350E06FEFF7
:1051C0007FEFCE0101960E94275ACE0101960E94E0
:1051D0006D426AEF74E084E291E10E94FE4164E274
:1051E00071E1CE0101960E94A94244E150E06FEFC7
:1051F0007FEFCE0101960E945E6FCE0101960E9464
:105200006D428BEB88A38AEA89A381E08AA3C12C33
:10521000D12CE12CF12C412C512C3201EAE02E2E24
:10522000312CC701B1010E94259A892B49F443E032
:1052300050E0BE01605E7F4F86E09FE00E94183E16
:1052400065E070E080E090E00E94E684BFEFEB1A3A
:10525000FB0A00E010E0812C912C540186E09FE0D5
:105260000E94733E892B81F4E4E08E169104A10420
:10527000B10454F094E0C916D10464F4A0E9EA162C
:10528000A1E0FA0671F606C00630110514F40C947C
:105290005C31F0CFC301B2010E945A9520E030E0AA
:1052A00040E251E40E94AA9720E030E040E85EE34B
:1052B0000E94B9956B017C0120E030E040EA51E4A6
:1052C0000E949998181634F521E0B701A601CE0185
:1052D00001960E94724267EE77E0CE0180960E94AE
:1052E000B142BE016F5F7F4FCE0180960E94D941CF
:1052F0006FE679E00E94C241BC018AE291E10E941E
:105300005842CE0180960E946D42CE0101960E94C5
:105310006D4206C06EEE74E08AE291E10E94FE41A9
:105320006AE271E1CE0101960E94A9424AE050E092
:1053300060E070E0CE0101960E94275ACE010196EE
:105340000E946D426AE271E1CE0101960E94A9427B
:1053500060E27BE0CE0101960E94C24164E271E10D
:105360000E94D941BC018AE291E10E945842CE01DB
:1053700001960E946D4286E09FE00E94FD540DCA96
:1053800069EB75E0CE0101960E94A1424AE050E02F
:105390006FEF7FEFCE0101960E945E6FCE01019606
:1053A0000E946D426091DC047091DD04809145049F
:1053B000909146040E94264664E1862E912CA12CF1
:1053C000B12CE12CF12C5FEFE51AF50AC501B4010F
:1053D0000E94E6846091DC047091DD0480914504B4
:1053E000909146040E9426468C0183E0E816F10461
:1053F00034F03EE1E316F10444F4012B51F044E1B2
:10540000840E911CA11CB11CDECF0115110509F001
:105410000CC180914504909146048B309105C9F4EC
:105420008091881190918911A0918A11B0918B116E
:105430008093520C9093530CA093540CB093550C42
:105440008091841190918511A0918611B09187115E
:105450001DC08631910521F30C9701F58091450C13
:105460009091460CA091470CB091480C8093520C3F
:105470009093530CA093540CB093550C8091410C15
:105480009091420CA091430CB091440C80934E0C2F
:1054900090934F0CA093500CB093510C4091520C30
:1054A0005091530C6091540C7091550C21E0CE0139
:1054B00001960E9472426EEB7BE0CE0180960E94C4
:1054C000B142BE016F5F7F4FCE0180960E94D941ED
:1054D000BC018AE291E10E945842CE0180960E946E
:1054E0006D42CE0101960E946D4240914E0C50914A
:1054F0004F0C6091500C7091510C21E0CE0101963F
:105500000E94724262E779E0CE0180960E94B14229
:10551000BE016F5F7F4FCE0180960E94D941BC01D2
:105520008AE291E10E94F841CE0180960E946D428C
:10553000CE0101960E946D4264E379E08AE291E136
:105540000E94EA4164E77BE0CE0101960E94B142ED
:1055500044E150E060E070E0CE0101960E94275ADD
:10556000CE0101960E946D42C090520CD090530C17
:10557000E090540CF090550C20E030E0A901C701F8
:10558000B6010E94999820E030E040E05FE387FD9B
:1055900005C0C701B6010E94E49604C0C701B60168
:1055A0000E94E3960E944398AB01BC01CE01019694
:1055B0000E94346BBE016F5F7F4F84E291E10E94D5
:1055C0003441CE0101960E946D4260E087E00E9466
:1055D000096B64E271E18BE292E10E940F436FED8F
:1055E0008BE292E10E94084368E779E08BE292E166
:1055F0000E94E84360914E0C70914F0C8091500CCA
:105600009091510C0E9443984AE050E08BE292E165
:105610000E949E4364E379E08BE292E10E94E843BA
:1056200064E670E080E090E08ECB0F3F9FEF1907BB
:10563000ACF06BEA75E0CE0101960E94A1424AE00F
:1056400050E060E070E0CE0101960E94275ACE0142
:1056500001960E946D4268E875E062C00E3FAFEFB0
:105660001A0709F449C06AE775E0CE0101960E9465
:10567000A1424AE050E060E070E0CE0101960E9455
:10568000275ACE0101960E946D426BE675E08AE2D0
:1056900091E10E94FE41B801CE0101960E94BB58E3
:1056A000BE016F5F7F4F8AE291E10E94F841CE0117
:1056B00001960E946D4200912E1110912F110B5EE8
:1056C0001F4FB8018AE291E10E946E41882309F4DC
:1056D00085C520912A1130912B1180912E11909126
:1056E0002F1165E575E0820F931F0E940C911093B6
:1056F0002F1100932E1172C56AE475E0CE01019658
:105700000E94A1424AE050E060E070E0CE010196C4
:105710000E94275ACE0101960E946D426AE275E00E
:105720008AE291E10E94FE4159C5809130048823AC
:1057300009F454C564E77BE0CE0101960E94B142B2
:105740004AE050E061E070E0CE0101960E94275AE5
:10575000CE0101960E946D420E94F64C3FC5809199
:10576000850C811109C02EE130E040E050E02CAF03
:105770003DAF4EAF5FAF08C082E090E0A0E0B0E088
:105780008CAF9DAFAEAFBFAF67EC75E08AE291E141
:105790000E94FE416AE271E1CE0101960E94A94297
:1057A0004AE050E06FEF7FEFCE0101960E945E6FFE
:1057B000CE0101960E946D42812C912C5401412C06
:1057C000512C320183E20E94EE6A87E090E00E9451
:1057D000E96A0E94E76A66E970E080E090E00E9472
:1057E000E68483E20E94EE6A80E290E00E94E96A29
:1057F0000E94E76A66E970E080E090E00E94E6843B
:1058000062E070E083E290E00E94DB55C12CD12C75
:10581000760180915A0C90E020915B0C821B9109DB
:10582000181619066CF480E490E10E94FB7AFE2CB5
:10583000ED2CDC2CCC24C80ED11CE11CF11CE9CFD2
:10584000C701B6010E945A952AE939E949E95FE39F
:105850000E94AA970E944398AB01BC01841695064A
:10586000A606B70614F44A015B01CE0180960E9499
:10587000346BBE01605E7F4FCE0101960E94A9424B
:105880006BE779E0CE0101960E94C241BC0184E23F
:1058900091E10E945842CE0101960E946D42CE01D4
:1058A00080960E946D4264E271E1CE0101960E94F1
:1058B000A9424EE150E060E070E0CE0101960E9406
:1058C000CC5ACE0101960E946D429FEF491A590AA7
:1058D000690A790A2CAD3DAD4EAD5FAD2415350595
:1058E000460557050CF06ECFB501A401CE01809698
:1058F0000E94346BBE01605E7F4FCE0101960E9414
:10590000A9426BE779E0CE0101960E94C241BC0139
:1059100084E291E10E945842CE0101960E946D42BC
:10592000CE0180960E946D4264E271E1CE01019643
:105930000E94A9424AE050E060E070E0CE0101968A
:105940000E94275ACE0101960E946D42B501A40122
:10595000CE0101960E94346B6FE779E0CE0180960C
:105960000E94B142BE016F5F7F4FCE0180960E94C0
:10597000D94162E879E00E94C2416AE271E10E9485
:10598000D941BC018AE291E10E945842CE01809641
:105990000E946D42CE0101960E946D42D0C90091D5
:1059A000DA041091DB0481E08093E00464E670E0A7
:1059B00080E090E00E94E6840E942F6FC8010E9460
:1059C0003B7760E074E0681B790BCE0101960E9482
:1059D000BB5867E879E0CE0180960E94B142BE01D3
:1059E0006F5F7F4FCE0180960E94D941BC018AE251
:1059F00091E10E945842CE0180960E946D42CE01F4
:105A000001960E946D4260E087E00E94096B67ED9D
:105A100075E0CE0101960E94A14242E350E068E0A9
:105A200070E0CE0101960E94275ACE0101960E9495
:105A30006D426AE271E1CE0101960E94A94242E301
:105A400050E06FEF7FEFCE0101960E945E6FCE01B6
:105A500001960E946D426EE879E0C7C08091D8043B
:105A60009091D9040E943B778C019093F70B80931F
:105A7000F60B62E370E080E090E00E94E684B801FB
:105A8000CE0101960E94BB58BE016F5F7F4F8AE234
:105A900091E10E943441CE0101960E946D428091B5
:105AA000821190918311892B09F45EC06EE771E138
:105AB000CE0180960E94A942BE01605E7F4FCE015A
:105AC00001960E94A94244E150E060E070E0CE01FE
:105AD00001960E94275ACE0101960E946D4268E904
:105AE00079E0CE0101960E94B1426AE271E1CE01F5
:105AF00001960E94D941BC0184E291E10E94584282
:105B0000CE0101960E946D4264E271E1CE010196E0
:105B10000E94A94244E150E06FEF7FEFCE01019671
:105B20000E945E6FCE0101960E946D42BE01605ED2
:105B30007F4FCE0101960E94A94260E27BE0CE0138
:105B400001960E94C24164E271E10E94D941BC0108
:105B50008AE291E10E945842CE0101960E946D4274
:105B6000CE0180960C94CB2363EA79E084E291E144
:105B70000E94434264E271E1CE0101960E94A94273
:105B800044E150E060E070E0CE0101960E94275AA7
:105B9000CE0101960E946D4267E879E0CE01019640
:105BA0000E94B1426AE271E1CE0101960E94D941A0
:105BB000BC0184E291E10E945842CE0101960E940C
:105BC0006D4264E271E1CE0101960E94A94244E176
:105BD00050E06FEF7FEFCE0101960E945E6FCE0125
:105BE00001960E946D4268E979E0CE0101960E941B
:105BF000B1426AE271E1CE0101960E94D941BC0135
:105C00008AE291E10E945842CE0101960E946D42C3
:105C10000C94CD2380913004882309F4DFC2809155
:105C2000850C882329F082E090E00E94E56FD6C2BF
:105C3000C0901302D0901402E0901502F09016026A
:105C400020E030E040E450E4C701B6010E9499989A
:105C500018166CF420E030E04AEF54E4C701B601B6
:105C60000E94B9950E9443986B017C0106C040E3F5
:105C7000C42E45E7D42EE12CF12C0E942F6F60E05A
:105C800080E00E94096B68EE75E08BE292E10E9471
:105C90001D4361E080E00E94096B60EE75E08BE2DD
:105CA00092E10E941D4364E670E080E090E00E9473
:105CB000E6840E941E856093F00B7093F10B809335
:105CC000F20B9093F30B0E941E850091F00B109144
:105CD000F10B2091F20B3091F30BDC01CB01801B17
:105CE000910BA20BB30B8C159D05AE05BF050CF0F7
:105CF00075C283E090E00E94E56F0E941E8564E11A
:105D000070E080E090E00E94E684DDCF0E94FE62B9
:105D10008CEC9DE00E94113F61C268E076E084E275
:105D200091E10E94FE4164E271E1CE0101960E9480
:105D3000A9424AE050E060E070E0CE0101960E9486
:105D4000275ACE0101960E946D4230901002809138
:105D5000060C811105C00E941E8581E08093060C0F
:105D60008091FE0B811105C00E941E8581E0809309
:105D7000FE0B1092FD0B1092FC0B0091FC0B10918E
:105D8000FD0B083211050CF07BC0832D0E949C8412
:105D9000F801EE0FFF1FEE5CF24F918380830E94AB
:105DA000806C20E030E040EA50E40E94B99520E0A9
:105DB00030E040E85AE30E94B9952B013C01809005
:105DC0000C0290900D02A0900E02B0900F02A5015F
:105DD0009401609108027091090280910A029091E9
:105DE0000B020E94E3969B01AC0160E070E080EC46
:105DF00090E40E94E3966B017C0120E030E0A90171
:105E00000E94549520E030E040E650E4811105C046
:105E1000C301B2010E94B9951EC0C301B2010E9424
:105E2000B995A50194010E94E49620E030E040E895
:105E300050E40E94E396A70196010E94AA9720E0F1
:105E400030E040EC50E40E94B99520E030E040E8BA
:105E500050E40E94E4966093F80B7093F90B8093E2
:105E6000FA0B9093FB0B64E170E080E090E00E94FD
:105E7000E6840F5F1F4F1093FD0B0093FC0B7DCF4B
:105E8000C090F80BD090F90BE090FA0BF090FB0B60
:105E900020E030E0A901C701B6010E94999887FD72
:105EA0001EC022E0B701A601CE0101960E947242F7
:105EB00067EA79E0CE0180960E94B142BE016F5F31
:105EC0007F4FCE0180960E94D941BC018AE291E1C8
:105ED0000E945842CE0180960E946D4269C169EFCE
:105EE00075E08AE291E10E94FE4166C18091300432
:105EF000882309F473C18091850C811127C0C0905B
:105F00001302D0901402E0901502F090160220E0E7
:105F100030E04AE754E4C701B6010E94B9950E94F7
:105F200043984B015C0120E030E040EA50E4C701B7
:105F3000B6010E94B99520E030E040EA50E40E94AA
:105F4000E4960E944398A501940108C021E030E046
:105F500040E050E06AE070E080E090E00E9453662C
:105F60003DC18091220D9091230D0097F1F581E0C4
:105F700090E09093230D8093220D6BEA79E0CE019F
:105F800001960E94B142CE0101960E94FB59CE01BA
:105F900001960E946D4264EB79E0CE0101960E9469
:105FA000B1426FE172E1CE0101960E94D941BC017C
:105FB000CE0180960E94A94248EC50E06FEF7FEF3F
:105FC000CE0180960E94275ACE0180960E946D4293
:105FD000CE0101960E946D428CEC9DE00E94FD5422
:105FE00040E052EC61E070E078C0029799F51092C1
:105FF000230D1092220D6AEB79E0CE0101960E94EA
:10600000B142CE0101960E94FB59CE0101960E9439
:106010006D4268EC79E0CE0101960E94B1426FE1D9
:1060200072E1CE0101960E94D941BC01CE01809659
:106030000E94A94248EC50E06FEF7FEFCE018096BE
:106040000E94275ACE0180960E946D42CE01019691
:106050000E946D428091220D9091230D0197A9F528
:1060600082E090E09093230D8093220D6CEC79E018
:10607000CE0101960E94B142CE0101960E94FB59C9
:10608000CE0101960E946D426DED79E0CE01019640
:106090000E94B1426FE172E1CE0101960E94D941A6
:1060A000BC01CE0180960E94A94248EC50E06FEFFF
:1060B0007FEFCE0180960E94275ACE0180960E94E3
:1060C0006D42CE0101960E946D428CEC9DE00E94D3
:1060D000FD5440E855E260E070E08CEC9DE00E94E9
:1060E000846E1092400C10923F0C80E090E00E9471
:1060F000E76E62EE79E0CE0101960E94B14269E15D
:1061000072E1CE0101960E94D941BC01CE01809678
:106110000E94A94240ED57E06FEF7FEFCE018096DD
:106120000E945E6FCE0180960E946D42CE01019664
:106130000E946D4253C08091AA0C9091AB0C892BA8
:10614000A1F481E090E09093AB0C8093AA0C8EEDCB
:1061500093E09093400C80933F0C0E940F6F68EC8B
:1061600070E080E090E00E94E684E0E0F0E01995C5
:1061700035C00E94A7810E942F6F0E94D0742EC04C
:10618000F092100CE0920F0C61E176E08AE291E16E
:106190000E94FE4164E77BE0CE0101960E94B1427D
:1061A0004AE050E060E070E0CE0101960E94275A7C
:1061B000CE0101960E946D426AE271E1CE01019624
:1061C0000E94A9424AE050E06FEF7FEFCE010196B6
:1061D0000E945E6FCE0101960E946D4280912E1149
:1061E00090912F110097C1F0419740F426962EAD63
:1061F0003FAD2697223031050CF0A1C06AE271E173
:10620000CE0101960E94A942CE0101960E947258C9
:10621000CE0101960E946D4264E670E080E090E05D
:106220000E94E6849FC00E94506F0C947F220C81D4
:1062300010E0102F00278D81080F111DEE80F12C2A
:10624000FE2CEE248F81E80EF11CC884D12CDC2CAE
:10625000CC248985C80ED11C31E03CAF0C94C125FB
:1062600067EB74E08AE291E10E94FE416AE271E12B
:10627000CE0180960E94A9424AE050E060E070E0C2
:10628000CE0180960E945E6FCE0180960E946D4284
:1062900064EA74E08AE291E10E94FE418091150C6B
:1062A0009091160C029711F00C9495261092160CF2
:1062B0001092150C0C94952686E09FE00E94733E88
:1062C000892B69F086E09FE00E94513EE1E0F0E01A
:1062D000EC0FFD1FE00FF11F80830F5F1F4F65E084
:1062E00070E080E090E00E94E6840630110501F540
:1062F000998188A198131CC09A8189A1981318C00C
:106300009B818AA1981314C08D8190E0A0E0B0E039
:10631000BA2FA92F982F88272C81820F911DA11D9C
:10632000B11D480E591E6A1E7B1EFFEFCF1ADF0AF1
:106330002FEF821A920AA20AB20A0C942E296AE25C
:1063400071E1CE0101960E94A9424AE050E06FEF50
:106350007FEFCE0101960E945E6FCE0101960E94F2
:106360006D424CCFC35BDF4F0FB6F894DEBF0FBE5C
:10637000CDBFDF91CF911F910F91FF90EF90DF90F4
:10638000CF90BF90AF909F908F907F906F905F90D5
:106390004F903F902F9008952F923F924F925F928F
:1063A0006F927F928F929F92AF92BF92CF92DF9225
:1063B000EF92FF920F931F93CF93DF93CDB7DEB78A
:1063C00028970FB6F894DEBF0FBECDBFFC0182E563
:1063D00090E19387828780914F1090E09587848722
:1063E00080911C1190E09787868780914C108530B2
:1063F00009F063C680915410909155108858910906
:106400008D35910588F480914F10843041F480914E
:106410005610909157108097479708F47DC080914F
:106420004F10843408F05EC080914F108A3108F418
:10643000D5C08091521090915310843F914050F4F8
:10644000118610868FEF9FEFDC0184839583A683EE
:10645000B7833CC0809154109091551085974B970D
:1064600008F0BCC008E5E02E00E1F02E82E090E0EC
:1064700040E050E0BA018C010F5F1F4F20914F1098
:1064800030E0021713076CF4970122503109D9014B
:106490002D913C91275031092730310508F47FC0F8
:1064A000C801019795958795918780870C971CF473
:1064B0001186108693C0448355836683778384E076
:1064C00090E00DC044835583668377838BE090E032
:1064D00006C044835583668377838CE090E0918384
:1064E00080831EC580915610909157108254910957
:1064F0008E9708F099CF20E030E0C12CD12C7601A6
:10650000A901485A5F4EDA014D915C9149505109F9
:106510004930510598F088CF8091581090915910CA
:106520000997099708F07BCF118610868FEF9FEFB0
:10653000DC0184839583A683B783C2C5B901665AFB
:106540007F4EDB014D915C9147515109423151051C
:10655000C0F4D701C601880F991FAA1FBB1F6C0189
:106560007D016894C0F82C5F3F4F2038310541F61B
:1065700020E230E031872087C482D582E682F7822C
:106580009FC5DB014D915C91465051094730510543
:1065900008F04ACFCC0CDD1CEE1CFF1CE4CFD70169
:1065A0002D913C91235131092F30310550F4440F86
:1065B000551F661F771F41600296B4E0EB0EF11C79
:1065C0005ACFD7012D913C912A50310929303105FC
:1065D00028F4440F551F661F771FEECF80914F1090
:1065E0008A3108F460C0809152109091531080322B
:1065F000934008F425CF8091541090915510C69780
:10660000869708F050C08091561090915710C69709
:10661000869708F048C0BAE5EB2EB0E1FB2E83E088
:1066200090E040E050E0BA018C010F5F1F4F2091D5
:106630004F1030E00217130764F49701225031091C
:10664000D9012D913C912C5031092B30310560F04E
:10665000C801019795958795918780870C970CF0D5
:1066600031CF118610861FC0D7012D913C91255244
:1066700031092B31310550F4440F551F661F771F28
:1066800041600296B4E0EB0EF11CCECFD7012D9104
:106690003C912C5031092A30310528F4440F551F04
:1066A000661F771FEECF80914F10823208F452C0E0
:1066B00080915410909155100697079708F04AC0A2
:1066C00048E5C42E40E1D42E82E090E040E050E066
:1066D000BA018C010F5F1F4F20914F1030E002175D
:1066E0001307F4F4D6011297ED90FC9011979D01D9
:1066F000BEE1EB1AF108A7E1EA16F104E0F4440F59
:10670000551F661F771F4160D6012D913C91B4E063
:10671000CB0ED11C2350310925303105C8F0C801FA
:106720000197959587959187808740970CF0D1CEFA
:10673000118610860FC0D9012D913C912C50310942
:106740002B30310538F4440F551F661F771FDCCFFF
:106750000296BFCF7F011C821B8281E090E09A836A
:10676000898380914F108D3070F41C821B8281E0F0
:1067700090E09A838983F701848595851816190618
:106780000CF474C0D1C029E733E0AE014D5F5F4F18
:10679000BE016F5F7F4FC7010E942683892B29F7B7
:1067A00029E733E0AE014D5F5F4FBE016F5F7F4F62
:1067B000C7010E9426830197C1F629E733E0AE01A5
:1067C0004D5F5F4FBE016F5F7F4FC7010E94268301
:1067D000892B59F6812C912C540100E010E0809116
:1067E0004F1090E029813A812817390794F529E75D
:1067F00033E0AE014D5F5F4FBE016F5F7F4FC7015A
:106800000E9426836C0129E733E0AE014D5F5F4FA4
:10681000BE016F5F7F4FC7010E942683F1E0CF1654
:10682000D10451F4892B09F0A0CF880C991CAA1C23
:10683000BB1C689480F80AC0CD2809F096CF019758
:1068400009F093CF880C991CAA1CBB1C0F5F1F4F2B
:10685000C6CFD70119961C930E931897F70184821F
:106860009582A682B78281E090E039CE0284F385DA
:10687000E02D82E090E09A838983828193818997D9
:106880004E9708F051C083E090E09A838983848119
:1068900095810B970A9708F047C02CEB31E0AE01C9
:1068A0004D5F5F4FBE016F5F7F4FC7010E94268320
:1068B000892BD1F52CEB31E0AE014D5F5F4FBE016E
:1068C0006F5F7F4FC7010E942683019769F5412CB6
:1068D000512C320100E010E0F701248535858981D3
:1068E0009A81821793070CF02FC12CEB31E0AE0197
:1068F0004D5F5F4FBE016F5F7F4FC7010E942683D0
:106900005C010330110509F0E5C02CEB31E0AE016C
:106910004D5F5F4FBE016F5F7F4FC7010E942683AF
:10692000A816B90609F4D6C0D7011A96ED91FC91C4
:106930001B9782819381C6978697E0F48481958125
:106940004B974597B8F4DF0116966F0126ECC20EFF
:10695000D11C20E030E040E050E060E070E080E0FA
:1069600090E00D911C911197095011090830110503
:1069700008F4F4C080914F10893370F182819381C3
:10698000895791098335910508F41BC125C0D901A8
:1069900012966D917C911397665171096131710561
:1069A00008F037C1D501C401880F991FAA1FBB1F6A
:1069B0004C015D01689480F84E5F5F4F2C5F3F4F44
:1069C0004B33510509F40CC1D9016D917C916A508A
:1069D000710969307105D8F280914F10823231F41B
:1069E000828193810A97099708F423C18281938158
:1069F0008957910983359105D0F480914F108132E8
:106A0000B0F084819581CA97899788F49F012A5FA5
:106A10003F4F812C912C540143E050E0D9016D91FE
:106A20007C916A5071096930710508F41EC1828138
:106A300093818C549109C59778F480914F108430DC
:106A400031F4848195818097479708F46CC18091D7
:106A50004F10843408F04EC180914F10863460F19D
:106A6000828193810C970B9708F4A9C125C0D901A5
:106A700012966D917C9113976E5171096731710572
:106A800008F0D1C1D501C401880F991FAA1FBB1FEF
:106A90004C015D01689480F84E5F5F4F2C5F3F4F63
:106AA0004534510509F4A6C1D9016D917C916C5012
:106AB00071096B307105D8F280914F10883508F458
:106AC000E4C182819381855891098B35910508F441
:106AD000BAC1DBC12CEB31E0AE014D5F5F4FBE01AF
:106AE0006F5F7F4FC7010E9426836C010330110541
:106AF00079F42CEB31E0AE014D5F5F4FBE016F5F6B
:106B00007F4FC7010E942683C816D90609F00CCF13
:106B1000A114B10459F4CA94CD2809F005CF440C4E
:106B2000551C661C771C689440F80BC0AA94AB28CF
:106B300009F0FACECD2809F0F7CE440C551C661C9E
:106B4000771C0F5F1F4FC8CE11870087F701448263
:106B500055826682778282E090E0C1CC12960D91D8
:106B60001C911397015111090D301105E0F401E05A
:106B70000E94409A21601496AC15BD0509F0F1CE33
:106B8000F701248335834683578300E20E945B9A92
:106B90002283338385E090E09183808380E390E0DB
:106BA00091878087BDC112960D911C911397045057
:106BB00011090530110508F0DDCE01E00E94409A70
:106BC000DACF84819581CA97899708F005CF9F0114
:106BD0002A5F3F4F812C912C540143E050E0F4CECA
:106BE0009F012A583F4FD9012D913C912A503109DC
:106BF0002930310508F0F0CE2CE130E0F701318783
:106C00002087D70184829582A682B7828AE090E0AD
:106C100085C1D90112966D917C91139766507109C7
:106C20006730710508F0D8CE880C991CAA1CBB1CD3
:106C3000C3CE20914F10CF01820F911D820F911D65
:106C4000DC0112978D919C910A97099708F0CECE9E
:106C5000F701118610868FEF9FEFDC018483958307
:106C6000A683B78386E090E03ACCD90112966D9165
:106C70007C911397665171096131710558F5D50101
:106C8000C401880F991FAA1FBB1F4C015D016894A6
:106C900080F84E5F5F4F2C5F3F4F4332510509F044
:106CA000BDCE9F012A5B3F4FD9012D913C912A50C7
:106CB00031092930310508F0BACE20E130E0F70182
:106CC00031872087D70184829582A682B78286E0A9
:106CD00090E024C1D90112966D917C911397665072
:106CE00071096730710508F0A2CE880C991CAA1CA6
:106CF000BB1CCFCF8481958189549109C39708F03B
:106D0000ABCE9F012A5F3F4FAF014A575F4F812CA7
:106D1000912C5401D9016D917C91695071096930B0
:106D20007105B8F099CE868197810997099708F087
:106D30008ECED70119961C921E9218978FEF9FEF57
:106D4000DC01F70184839583A683B78387E090E015
:106D5000C6CBD90112966D917C911397665171093A
:106D600061317105E0F4D501C401880F991FAA1F94
:106D7000BB1F4C015D01689480F82C5F3F4F2417C6
:106D8000350741F620E230E0F70131872087D7014F
:106D900084829582A682B78287E090E0BFC0D90145
:106DA00012966D917C911397665071096730710549
:106DB00008F052CE880C991CAA1CBB1CDECF848123
:106DC00095810997099708F077CE868197818C97EE
:106DD0004F9708F071CE8085918589974D9708F07F
:106DE0006BCE9F01265F3F4F812C912C540145E0D3
:106DF00050E05ACE9F0126573F4FD9012D913C912B
:106E00002C5031092B30310508F056CE20E230E00D
:106E1000F70131872087D70184829582A682B782C5
:106E200088E090E07BC0D90112966D917C91139718
:106E3000695071096930710508F03ECE880C991CC3
:106E4000AA1CBB1C29CE84819581825491098E97FE
:106E5000E0F48F01045C1F4F8DE190E040E050E0D2
:106E600020914F1030E024503109821793070CF025
:106E700063C0980122503109D9012D913C912950CC
:106E800031092830310508F46EC080914F108032EE
:106E900009F07EC0828193810697069708F078C03A
:106EA000848195810997099708F072C09F012A5F34
:106EB0003F4FAF01425C5F4F812C912C5401D901AF
:106EC0006D917C91665071096630710508F060C063
:106ED000D90112966D917C911397695171096331B3
:106EE000710508F0D5C0D501C401880F991FAA1FEC
:106EF000BB1F4C015D01689480F82C5F3F4F241745
:106F00003507E9F62EE030E0F70131872087D70119
:106F100084829582A682B7828FE090E08D939C93C5
:106F200081E090E0D0C0D8012D913C9128513109E9
:106F30002231310550F1CB01019795958795D70105
:106F400019969C938E9318978A970CF49ECF052ED2
:106F5000000C660B770BF7014483558366837783B8
:106F600089E090E0BCCABC016F5F7F4FD8012D91D2
:106F70003C912750310927303105A8F6440F551FA1
:106F8000416002960C5F1F4F6BCF440F551FF9CF26
:106F9000D7011C962D903C901D97B6E02B1631041E
:106FA0000CF486C08F010E5F1F4F75EC872E7DE9B4
:106FB000972E7CE1A72E71E8B72EE3E0CE2ED12CE0
:106FC000F801648175816080718080E090E00E94AA
:106FD00058956D837E838F839887B30180E090E01E
:106FE0000E9458952B013C012DEC3CEC4CE45FE3F6
:106FF0000E94B9959B01AC016D817E818F8198853E
:107000000E94549587FD19C02DEC3CEC4CE45FE3E5
:107010006D817E818F8198850E94B9959B01AC011D
:10702000C301B2010E945495E82F880FFF0BEE2791
:10703000FF0FEE1FFF27319602C0E0E0F0E0A50150
:10704000940163E971E080E091E00E94029A4F01AF
:10705000FF0FAA08BB0886269726A826B926FFEFA9
:10706000CF1ADF0A0E5F1F4F2C143D0409F0A8CF82
:10707000D70114968D929D92AD92BC92179780E2A3
:1070800090E019969C938E9318978FEF9FEF46CFC1
:10709000D90112966D917C911397695071096930ED
:1070A000710508F075CF880C991CAA1CBB1C25CF54
:1070B00082E080934C1010924F1080E090E003C06B
:1070C00083E090E00CCA28960FB6F894DEBF0FBE9E
:1070D000CDBFDF91CF911F910F91FF90EF90DF9087
:1070E000CF90BF90AF909F908F907F906F905F9068
:1070F0004F903F902F9008954F925F926F927F92A2
:107100009F92AF92BF92CF92DF92EF92FF920F9336
:107110001F93CF93DF93CDB7DEB7A9970FB6F8943F
:10712000DEBF0FBECDBF982E882351F08091800C1A
:10713000882331F064E77BE083EA9FE00E94616B83
:107140000E94895860E08DE20E94E65960E18DE27C
:107150000E94E65968E08DE20E94E6594090941141
:10716000509095116090961170909711498E5A8E9B
:107170006B8E7C8EC0909811D0909911E0909A11EE
:10718000F0909B11CD8EDE8EEF8EF8A280919C1137
:1071900090919D11A0919E11B0919F118EA39FA3DC
:1071A000A8A7B9A789A39AA3ABA3BCA39920D1F19F
:1071B0008091800C8823B1F162E07AE0CE010196E3
:1071C0000E94A142CE0101960E94FB59CE01019678
:1071D0000E946D428E01075E1F4F5E0195E2A90E6F
:1071E000B11CD8016D917D918D919D918D0146E0ED
:1071F00050E00E947F6C60E27BE083EA9FE00E94A7
:10720000E843A016B10669F764E77BE0CE0101967A
:107210000E94B142CE0101960E94FB59CE01019617
:107220000E946D4223E938E144E85FE3C301B20103
:107230000E94B9952B013C016D877E878F87988BC3
:1072400022E430E645E85FE3C701B6010E94B99544
:107250006B017C01698B7A8B8B8B9C8B25E83BEED9
:1072600041E95FE36EA17FA188A599A50E94B99528
:107270006D8B7E8B8F8B988F4092941150929511CD
:107280006092961170929711C0929811D0929911B4
:10729000E0929A11F0929B1160939C1170939D1152
:1072A00080939E1190939F11992009F4A2C0809120
:1072B000800C882309F49DC065EF79E0CE0101962A
:1072C0000E94A142CE0101960E94FB59CE01019677
:1072D0000E946D428E01035F1F4F6E01B9E1CB0E1C
:1072E000D11C7801F80161917191819191918F0187
:1072F00042E050E00E947F6C60E27BE083EA9FE026
:107300000E94E8430C151D0569F764E77BE0CE0198
:1073100001960E94B142CE0101960E94FB59CE0116
:1073200001960E946D4240EA51E166E070E082E31E
:107330000E947F59A090A011B090A111C090A211FD
:10734000D090A3110091A4111091A51168EE79E0DD
:1073500083EA9FE00E941D434AE050E0B50183EAC2
:107360009FE00E949E4360E27BE083EA9FE00E94F0
:10737000E8434AE050E0B60183EA9FE00E949E4362
:1073800060E27BE083EA9FE00E94E8434AE050E04D
:10739000B80183EA9FE00E949E4364E77BE083EAB2
:1073A0009FE00E94616BCE0101960E940B506FED31
:1073B00079E083EA9FE00E941D438E010F5F1F4F1B
:1073C000D8016D917D918D919D918D014AE050E0A4
:1073D0000E947F6C60E27BE083EA9FE00E94E843CA
:1073E0000E151F0569F764E77BE083EA9FE00E94C2
:1073F000616B61E08DE10E94E6599920B1F08091C6
:10740000800C882391F06BEC79E083EA9FE00E9486
:107410001D43AE014B5D5F4F61E070E08DE10E9466
:107420007F598DA190E00E94B95962E08EE10E94DF
:10743000E65963E08FE10E94E65964E080E20E9431
:10744000E659992009F450C08091800C882309F4F2
:107450004BC06FEA79E083EA9FE00E941D43AE01D2
:107460004B5D5F4F61E070E08EE10E947F59CDA0DF
:10747000D12CAE014B5D5F4F61E070E08FE10E9467
:107480007F59EDA0F12CAE014B5D5F4F61E070E0E4
:1074900080E20E947F590DA110E04AE050E0B60161
:1074A00083EA9FE00E949E4360E27BE083EA9FE0E4
:1074B0000E94E8434AE050E0B70183EA9FE00E945F
:1074C0009E4360E27BE083EA9FE00E94E8434AE05B
:1074D00050E0B80183EA9FE00E949E4364E77BE0AE
:1074E00083EA9FE00E94616B65E081E20E94E659B9
:1074F0009920B1F08091800C882391F06CE979E0BB
:1075000083EA9FE00E941D43AE014B5D5F4F61E047
:1075100070E081E20E947F598DA190E00E94B959EC
:1075200066E082E20E94E6599920B1F08091800CD9
:10753000882391F064E879E083EA9FE00E941D438C
:10754000AE014B5D5F4F61E070E082E20E947F59C7
:107550008DA190E00E94B95967E083E20E94E6594C
:107560009920B1F08091800C882391F06EE679E04B
:1075700083EA9FE00E941D43AE014B5D5F4F61E0D7
:1075800070E083E20E947F598DA190E00E94B9597A
:1075900068E084E20E94E6599920B1F08091800C65
:1075A000882391F066E579E083EA9FE00E941D431D
:1075B000AE014B5D5F4F61E070E084E20E947F5955
:1075C0008DA190E00E94B95969E085E20E94E659D8
:1075D0009920B1F08091800C882391F06CE379E0E0
:1075E00083EA9FE00E941D43AE014B5D5F4F61E067
:1075F00070E085E20E947F598DA190E00E94B95908
:107600006AE086E20E94E6599920B1F08091800CF0
:10761000882391F066E279E083EA9FE00E941D43AF
:10762000AE014B5D5F4F61E070E086E20E947F59E2
:107630008DA190E00E94B9596BE088E20E94E65962
:107640009920A9F08091800C882389F06DE079E081
:1076500083EA9FE0F2D7AE014B5D5F4F61E070E0DF
:1076600088E20E947F598DA190E00E94B9596CE098
:1076700089E20E94E659992009F471C08091800C3A
:10768000882309F46CC065EF78E083EA9FE0D5D7E2
:10769000AE014B5D5F4F61E070E089E20E947F596F
:1076A0008DA190E00E94B9596EED78E083EA9FE0E9
:1076B000C4D766E070E087E20E94CC5990E00E9457
:1076C000B95967EC78E083EA9FE0B7D765E070E0EE
:1076D00087E20E94CC5990E00E94B95960EB78E0B3
:1076E00083EA9FE0AAD764E070E087E20E94CC5969
:1076F00090E00E94B95967E978E083EA9FE09DD75E
:1077000062E070E087E20E94CC5990E00E94B95993
:107710006EE778E083EA9FE090D761E070E087E26F
:107720000E94CC5990E00E94B95965E678E083EA5E
:107730009FE083D760E070E087E20E94CC5990E040
:107740000E94B95964E578E083EA9FE076D763E068
:1077500070E087E20E94CC5990E00E94B95941E064
:1077600067E070E087E20E94AE4F41E063E070E0C6
:1077700087E20E94AE4F41E063E070E08AE20E943F
:10778000AE4F992089F08091800C882369F06BE3DB
:1077900078E083EA9FE051D763E070E08AE20E94DC
:1077A000CC5990E00E94B95940E063E070E08AE271
:1077B0000E94AE4F992089F08091800C882369F057
:1077C00061E278E083EA9FE038D763E070E08AE224
:1077D0000E94CC5990E00E94B95941E062E070E00B
:1077E0008AE20E94AE4F992089F08091800C882314
:1077F00069F065E078E083EA9FE01FD762E070E01F
:107800008AE20E94CC5990E00E94B95940E062E0BF
:1078100070E08AE20E94AE4F992089F08091800C3E
:10782000882369F068EE77E083EA9FE006D762E09C
:1078300070E08AE20E94CC5990E00E94B95941E080
:1078400061E070E08AE20E94AE4F992089F0809159
:10785000800C882369F06CEC77E083EA9FE0EDD63A
:1078600061E070E08AE20E94CC5990E00E94B95930
:1078700040E061E070E08AE20E94AE4F992089F01A
:107880008091800C882369F06FEA77E083EA9FE0BB
:10789000D4D661E070E08AE20E94CC5990E00E9468
:1078A000B95941E060E070E08AE20E94AE4F992051
:1078B00089F08091800C882369F063E977E083EA9E
:1078C0009FE0BBD660E070E08AE20E94CC5990E075
:1078D0000E94B95940E060E070E08AE20E94AE4F39
:1078E000992089F08091800C882369F066E777E021
:1078F00083EA9FE0A2D660E070E08AE20E94CC5961
:1079000090E00E94B95941E066E070E087E20E9491
:10791000AE4F41E065E070E087E20E94AE4F41E08B
:1079200064E070E087E20E94AE4F40E062E070E009
:1079300087E20E94AE4F40E061E070E087E20E9483
:10794000AE4F40E060E070E087E20E94AE4F9920C9
:1079500009F46DC08091800C882309F468C06EE53D
:1079600077E083EA9FE069D666E070E08BE20E94F0
:10797000CC5990E00E94B95960E477E083EA9FE037
:107980005CD665E070E08BE20E94CC5990E00E94EA
:10799000B95962E277E083EA9FE04FD664E070E095
:1079A0008BE20E94CC5990E00E94B95969E077E0DF
:1079B00083EA9FE042D662E070E08BE20E94CC59FD
:1079C00090E00E94B95960EF76E083EA9FE035D6F7
:1079D00061E070E08BE20E94CC5990E00E94B959BE
:1079E00067ED76E083EA9FE028D660E070E08BE206
:1079F0000E94CC5990E00E94B95964EC76E083EA89
:107A00009FE01BD663E070E08BE20E94CC5990E0CF
:107A10000E94B9596FEA76E083EA9FE00ED664E0EF
:107A200070E08CE20E94CC5990E00E94B95940E08D
:107A300064E070E08CE20E94AE4FAE014B5D5F4FA0
:107A400061E070E08CE20E947F596DA1607F66600A
:107A50008CE20E94E659992009F45BC08091800C69
:107A6000882309F456C06BE976E083EA9FE0E5D508
:107A7000AE014B5D5F4F61E070E08CE20E947F5988
:107A80006DA16F7070E066507109072E000C880BB5
:107A9000990B0E945A959B01AC0160E070E080E078
:107AA00090E40E94589920E030E048EC50E40E94B5
:107AB000B9950E94FC4F64E876E083EA9FE0BDD56B
:107AC000AE014B5D5F4F61E070E080E30E947F5943
:107AD0006DA14AE050E083EA9FE00E94E04F6CE62F
:107AE00076E083EA9FE0A9D561E070E080E30E9440
:107AF000CC5990E00E94B95963E576E083EA9FE0B3
:107B00009CD561E070E08FE20E94CC5990E00E9429
:107B1000B95941E061E070E08FE20E94AE4F9920D8
:107B200089F08091800C882369F06BE376E083EA2A
:107B30009FE083D561E070E08EE20E94CC5990E036
:107B40000E94B95941E061E070E08EE20E94AE4FC0
:107B500040E067E070E081E30E94AE4F992009F4B5
:107B600050C08091800C882309F44BC068E276E015
:107B700083EA9FE062D567E070E081E30E94CC5920
:107B800090E00E94B95967EE79E083EA9FE020D641
:107B9000AE014B5D5F4F61E070E080E00E947F5975
:107BA0008DA10E94567D64E77BE083EA9FE00E94FE
:107BB000616B0DE110E063E17AE083EA9FE008D6B3
:107BC00040E150E0B80183EA9FE0B8D567E678E08D
:107BD00083EA9FE0FDD5AE014B5D5F4F61E070E051
:107BE000802F0E947F598DA10E94567D64E77BE023
:107BF00083EA9FE00E94616B0F5F1F4F0A331105FC
:107C0000D1F6A9960FB6F894DEBF0FBECDBFDF91B7
:107C1000CF911F910F91FF90EF90DF90CF90BF9089
:107C2000AF909F907F906F905F904F9008950895D0
:107C3000CF92DF92EF92FF920F931F93CF93DF9338
:107C40006C017A018B01C0E0D0E0CE15DF0581F038
:107C5000D8016D918D01D601ED91FC910190F081DB
:107C6000E02DC6011995892B11F02196EECF7E01EA
:107C7000C701DF91CF911F910F91FF90EF90DF909F
:107C8000CF900895FC01538D448D252F30E0842F33
:107C900090E0821B930B541710F0CF960895019734
:107CA0000895FC01918D828D981761F0828DDF011E
:107CB000A80FB11D5D968C91928D9F5F9F73928FDF
:107CC00090E008958FEF9FEF0895FC01918D828DD4
:107CD000981731F0828DE80FF11D858D90E00895A1
:107CE0008FEF9FEF0895FC01918D228D892F90E0F9
:107CF000805C9F4F821B91098F73992708958CECAC
:107D00009DE0F1DF21E0892B09F420E0822F089526
:107D100089E69EE0E8DF21E0892B09F420E0822F4C
:107D2000089586E09FE0DFDF21E0892B09F420E061
:107D3000822F089583EA9FE0D6DF21E0892B09F4A2
:107D400020E0822F0895FC01848DDF01A80FB11D72
:107D5000A35ABF4F2C91848D90E001968F73992781
:107D6000848FA689B7892C93A089B1898C9183705F
:107D700080648C93938D848D981306C00288F38958
:107D8000E02D80818F7D80830895EF92FF920F9385
:107D90001F93CF93DF93EC0181E0888F9B8D8C8DB7
:107DA000981305C0E889F989808185FD25C0F62EE4
:107DB0000B8D10E00F5F1F4F0F731127E02E8C8D7E
:107DC000E8120BC00FB607FCFACFE889F989808169
:107DD00085FFF5CFCE01B7DFF2CF8B8DFE01E80F27
:107DE000F11DE35AFF4FF0829FB7F8940B8FEA8999
:107DF000FB89808180620AC09FB7F894EE89FF8971
:107E00006083E889F98980818370806480839FBF63
:107E100081E090E0DF91CF911F910F91FF90EF9063
:107E20000895CF93DF93EC01888D8823C1F0EA8910
:107E3000FB89808185FD05C0A889B9898C9186FD63
:107E40000EC00FB607FCF5CF808185FFF2CFA88961
:107E5000B9898C9185FFEDCFCE0175DFE8CFDF9139
:107E6000CF91089580E090E0892B19F063DF8111B4
:107E700016C080E090E0892B19F053DF811112C009
:107E800080E090E0892B19F043DF81110EC080E083
:107E900090E0892B79F033DF81110AC008950E94A8
:107EA0000000E7CF0E940000EBCF0E940000EFCF60
:107EB0000C94000008950E94789CCF93DF93EC010E
:107EC00088819981009711F00E940F9B1982188276
:107ED0001D821C821B821A82DF91CF9108950F931D
:107EE0001F93CF93DF938C01EB0188E2FB0111928A
:107EF0008A95E9F74BE050E06CE97AE0CE010E9408
:107F0000B49C1B8681E090E0A0E0B0E08C879D8768
:107F1000AE87BF87F80185899689A789B08D888B40
:107F2000998BAA8BBB8B82E090E0A0E0B0E08C8BB9
:107F30009D8BAE8BBF8B1CA21DA21EA21FA280E038
:107F400090E0A8E4B4E4888F998FAA8FBB8F80E07B
:107F500090E0A8E4B4EC8C8F9D8FAE8FBF8F8DEC3A
:107F60009CECACE4BEE388A399A3AAA3BBA3DF91D6
:107F7000CF911F910F9108954F925F926F927F92D0
:107F80008F929F92AF92BF92CF92DF92EF92FF9229
:107F90000F931F93CF93DF938C01EB0184E2FB01DE
:107FA00011928A95E9F78EE10E94EE6A83E090E0F3
:107FB0000E94E96A0E94E76A66E08EE10E94E75843
:107FC00080915A0C90E020915B0C821B91098630C5
:107FD0009105ECF380E490E10E94FB7A882E80E426
:107FE00090E10E94FB7A982E80E490E10E94FB7A57
:107FF000682E80E490E10E94FB7A782E80E490E184
:108000000E94FB7A482E80E490E10E94FB7A582E71
:10801000B82CA12CB5016929072E000C880B990BEF
:108020000E945A954B015C01F80165837683878332
:108030009087D42CC12CB6016529072E000C880B23
:10804000990B0E945A95F8016187728783879487FC
:10805000F62CE12CB7016729072E000C880B990B31
:108060000E945A95F801658776878787908B118AD9
:10807000128A138A148A84E290E0A0E0B0E0888338
:108080009983AA83BB8385899689A789B08D8C83C0
:108090009D83AE83BF8382E090E0A0E0B0E088875C
:1080A0009987AA87BB87188A198A1A8A1B8AC0905F
:1080B0008004D0908104E0908204F0908304A701B2
:1080C0009601C501B4010E94AA9720E030E048EC77
:1080D00052E40E94B9956C8B7D8B8E8B9F8BA70190
:1080E0009601F80161857285838594850E94AA971F
:1080F00020E030E048EC52E40E94B995688F798F17
:108100008A8F9B8F20917C0430917D0440917E0466
:1081100050917F04F80165857685878590890E9456
:10812000AA9720E030E048EC52E40E94B9956C8FA9
:108130007D8F8E8F9F8F81E0DF91CF911F910F9167
:10814000FF90EF90DF90CF90BF90AF909F908F9077
:108150007F906F905F904F900895862F0C940A84C3
:10816000862F642F0C943284862F642F0C946084A5
:10817000FC0180819181009711F00C94E69060E001
:1081800070E0CB010895AF92BF92CF92DF92EF9251
:10819000FF920F931F93CF93DF93DC01CD90DC9080
:1081A0001197C114D10409F443C01496CD91DC9108
:1081B00015972097E9F18C0176015701BFEFAB1AB3
:1081C000BB0AF7018081082E000C990B0E942495B0
:1081D000892B11F07501F1CF2197CC0DDD1D888120
:1081E000082E000C990B0E942495892B29F0CE159E
:1081F000DF0510F02197F3CFAE014F5F5F4F4E19AF
:108200005F09D80115965C934E931497CE14DF0442
:1082100020F4B701C6010E948D9CD801ED91FC911C
:10822000119714968D919C911597E80FF91F108264
:10823000DF91CF911F910F91FF90EF90DF90CF9042
:10824000BF90AF900895FC012481358162177307B8
:1082500048F480819181009729F0FC01E60FF71F17
:108260008081089580E008950F931F93CF93DF934B
:108270008C01EB01FC0180819181009739F06881CC
:10828000798161157105A1F40E940F9B8881998104
:10829000F801918380838A819B81938382838C817F
:1082A0009D8195838483198218821B821A820FC054
:1082B000F801428153812C813D814217530720F3FD
:1082C0000E949F9C8C819D81F801958384831D82EF
:1082D0001C82DF91CF911F910F9108950F931F93EF
:1082E000CF93DF93EC0188819981009729F02A814F
:1082F0003B812617370788F48B016F5F7F4F0E9401
:10830000989B009761F0998388831B830A832C8153
:108310003D81232B11F4FC01108281E001C080E03B
:10832000DF91CF911F910F910895EF92FF920F93DC
:108330001F93CF93DF936115710511F480E01BC08B
:1083400041155105B9F07B01EC018C819D818A01B9
:10835000080F191FB801CE01C1DF882379F32881E6
:1083600039818C819D81B701820F931F0E949F9C50
:108370001D830C8381E0DF91CF911F910F91FF90BE
:10838000EF900895CF93DF93EC016115710559F0DB
:10839000FB0101900020E9F73197AF01461B570B15
:1083A000C4DF811102C0CE0188DDCE01DF91CF9103
:1083B0000895CF93DF93EC01FB01448155816081E7
:1083C0007181B3DF811102C0CE0177DDCE01DF9173
:1083D000CF9108956115710549F0FB0101900020CE
:1083E000E9F73197AF01461B570B9FCF80E0089507
:1083F000FB01448155816081718197CFEF92FF929B
:108400000F931F93CF93DF93EC018B0161157105DF
:1084100049F0CB010E9413917C01BC01CE015EDFCB
:10842000811103C0CE0149DD07C0FD82EC82B80195
:10843000888199810E940C91CE01DF91CF911F918B
:108440000F91FF90EF900895EF92FF920F931F937B
:10845000CF93DF93EC017B018A01BA013FDF8111E9
:1084600003C0CE012ADD07C01D830C83B7018881BC
:1084700099810E949F9CCE01DF91CF911F910F9116
:10848000FF90EF900895CF93DF93EC016115710594
:1084900051F0FB0101900020E9F73197AF01461B35
:1084A000570BD2DF01C009DDCE01DF91CF910895D6
:1084B000CF93DF93EC01FB018617970751F06081A2
:1084C00071816115710521F044815581BDDF01C0C5
:1084D000F4DCCE01DF91CF910895FC018081918180
:1084E0000C940F9BEF92FF920F931F93CF93DF9308
:1084F000CDB7DEB7A1970FB6F894DEBF0FBECDBFE4
:108500007C01CB01BA01F701118210821382128221
:108510001582148242E0420F8E010F5F1F4F0E94AE
:10852000C490BC01C701AFDFA1960FB6F894DEBFBF
:108530000FBECDBFDF91CF911F910F91FF90EF90B4
:108540000895FC0111821082138212821582148216
:1085500055CFFC011182108213821282158214827F
:10856000A7CFFC011182108213821282158214821D
:108570006115710549F0FB0101900020E9F7319781
:10858000AF01461B570B60CF0895BF92CF92DF9289
:10859000EF92FF920F931F93CF93DF937C016B01B8
:1085A0008A01E9012417350720F4812F8901C42F9E
:1085B000D82F64E77BE0C701D4DFD60114968D91F4
:1085C0009C91159708171907C0F48C179D0708F49C
:1085D000EC01D601ED91FC911197EC0FFD1FB080DD
:1085E00010826D917C91600F711FC7014CDFD60125
:1085F000ED91FC91EC0FFD1FB082C701DF91CF918F
:108600001F910F91FF90EF90DF90CF90BF90089552
:10861000DC01ED91FC910190F081E02D1994DB01DA
:1086200014964D915C9115976D917C91DC01ED91C3
:10863000FC910280F381E02D1994EF92FF920F9349
:108640001F93CF93DF938C017B01C0E0D0E0F70153
:10865000EC0FFD1F6491662361F0D801ED91FC9150
:108660000190F081E02DC8011995892B11F0219618
:10867000EECFCE01DF91CF911F910F91FF90EF9040
:1086800008956115710579F0FB0101900020E9F76B
:108690003197AF01461B570BDC01ED91FC91028035
:1086A000F381E02D199480E090E008958F929F92DD
:1086B000AF92BF92EF92FF920F931F93CF93DF93EE
:1086C000CDB7DEB7A1970FB6F894DEBF0FBECDBF12
:1086D0007C01FA01CB0119A2223008F42AE08E01B4
:1086E0000F5D1F4F822E912CA12CB12CBF01A50133
:1086F00094010E94B296F901CA01015011096A3031
:1087000014F4605D01C0695CD8016C93232B242BA9
:10871000252B61F7B801C701B4DFA1960FB6F89415
:10872000DEBF0FBECDBFDF91CF911F910F91FF90A4
:10873000EF90BF90AF909F908F900895CF92DF926F
:10874000EF92FF920F931F93CF93DF934115510543
:1087500079F4DC01ED91FC910190F081E02DDF9145
:10876000CF911F910F91FF90EF90DF90CF901994D0
:108770006B01770FEE08FF084A305105E9F4F7FE68
:1087800019C0EC016DE244DF8C0144275527BA0182
:108790004C195D096E097F092AE0CE0187DF800F41
:1087A000911FDF91CF911F910F91FF90EF90DF907C
:1087B000CF9008952AE001C0242FB701A601DF91D0
:1087C000CF911F910F91FF90EF90DF90CF906ECFE0
:1087D00058CF1F920F920FB60F9211240BB60F9223
:1087E0002F933F934F935F936F937F938F939F93B9
:1087F000AF93BF93EF93FF938CEC9DE0A4DAFF91CE
:10880000EF91BF91AF919F918F917F916F915F9108
:108810004F913F912F910F900BBE0F900FBE0F9075
:108820001F9018951F920F920FB60F9211240BB63E
:108830000F922F933F934F935F936F937F938F93F9
:108840009F93AF93BF93EF93FF938CEC9DE00E94B7
:10885000F183FF91EF91BF91AF919F918F917F91A4
:108860006F915F914F913F912F910F900BBE0F90A1
:108870000FBE0F901F9018951F920F920FB60F9278
:1088800011240BB60F922F933F934F935F936F93E7
:108890007F938F939F93AF93BF93EF93FF9389E65B
:1088A0009EE051DAFF91EF91BF91AF919F918F912F
:1088B0007F916F915F914F913F912F910F900BBEE0
:1088C0000F900FBE0F901F9018951F920F920FB62A
:1088D0000F9211240BB60F922F933F934F935F93F8
:1088E0006F937F938F939F93AF93BF93EF93FF9378
:1088F00089E69EE00E94F183FF91EF91BF91AF91D5
:108900009F918F917F916F915F914F913F912F91A7
:108910000F900BBE0F900FBE0F901F9018951F92D7
:108920000F920FB60F9211240BB60F922F933F9315
:108930004F935F936F937F938F939F93AF93BF9367
:10894000EF93FF9386E09FE0FED9FF91EF91BF91F7
:10895000AF919F918F917F916F915F914F913F91D7
:108960002F910F900BBE0F900FBE0F901F90189578
:108970001F920F920FB60F9211240BB60F922F93E6
:108980003F934F935F936F937F938F939F93AF9397
:10899000BF93EF93FF9386E09FE00E94F183FF91E6
:1089A000EF91BF91AF919F918F917F916F915F9167
:1089B0004F913F912F910F900BBE0F900FBE0F90D4
:1089C0001F9018951F920F920FB60F9211240BB69D
:1089D0000F922F933F934F935F936F937F938F9358
:1089E0009F93AF93BF93EF93FF9383EA9FE0ABD93D
:1089F000FF91EF91BF91AF919F918F917F916F9177
:108A00005F914F913F912F910F900BBE0F900FBE32
:108A10000F901F9018951F920F920FB60F9211246E
:108A20000BB60F922F933F934F935F936F937F9368
:108A30008F939F93AF93BF93EF93FF9383EA9FE04E
:108A40000E94F183FF91EF91BF91AF919F918F9120
:108A50007F916F915F914F913F912F910F900BBE3E
:108A60000F900FBE0F901F901895DC0180E06150B1
:108A700098F02D91982F9227E92FEF70F0E0E253B4
:108A8000F54F249192959F70E92FF0E0E252F54F57
:108A9000E491822F8E27EBCF0895DF92EF92FF9221
:108AA0000F931F93CF93DF93EC01D62EE42E08E0B3
:108AB00010E0FF24F39461E08D2D8F2109F460E034
:108AC000CE010E94987BFF0C01501109A1F7E11023
:108AD00010C0F894E981FA81918188818095892379
:108AE0008183E981FA8192818881809589238283BB
:108AF0007894DF91CF911F910F91FF90EF90DF90CD
:108B00000895EF92FF920F931F93CF93DF938C0101
:108B10007B0140E065E5C1DFE70188E0E80EF11C7C
:108B2000699140E0C801B9DFCE15DF05C9F7DF91D3
:108B3000CF911F910F91FF90EF9008956F927F92C8
:108B40008F929F92AF92BF92CF92DF92EF92FF925D
:108B50000F931F93CF93DF93EC017B018A018E81EA
:108B60009F810E94C77B882399F1B7018E819F81E5
:108B7000C8DF40E06EEB8E819F818FDF7801680156
:108B800089E0C80ED11CAE80BF8088E0882E912C71
:108B9000712C66246394C5010E94747B8111762830
:108BA000660CE1E08E1A9108B1F7F70171927F012E
:108BB000EC15FD0541F78E819F810E94C77B8130B6
:108BC00039F468E0C80151DF91E0F80120852813ED
:108BD00090E0892FDF91CF911F910F91FF90EF903F
:108BE000DF90CF90BF90AF909F908F907F906F90CD
:108BF0000895CF93DF93CDB7DEB729970FB6F894DA
:108C0000DEBF0FBECDBFAE014F5F5F4F97DF882342
:108C100089F08D818F3361F020F48F3159F489E030
:108C20000CC08F3519F08F3739F004C08BE005C0C8
:108C30008AE003C080E001C08CE029960FB6F8946A
:108C4000DEBF0FBECDBFDF91CF9108958F929F926F
:108C5000AF92BF92CF92DF92EF92FF920F931F934A
:108C6000CF93DF938C01862F0B30110509F06FC075
:108C700090919111992309F0F89462E10E94F058C3
:108C800020919111222309F07894009709F072C085
:108C9000E0908C11F0908D116F2D70E080E090E0ED
:108CA0000E945A952DEC3CEC4CEC5DE30E94B9958A
:108CB0004B015C016E2D70E080E090E00E945A95BF
:108CC0009B01AC01C501B4010E94E496609384113C
:108CD000709385118093861190938711C0918E11A6
:108CE000D0918F116C2F6F7770E080E090E00E9440
:108CF0005A954B015C016D2F70E080E090E00E947E
:108D00005A952DEC3CEC4CEC5DE30E94B9959B012F
:108D1000AC01C501B4010E94E496C7FD09C060938F
:108D200088117093891180938A1190938B110BC0D5
:108D3000DC01CB01B0588093881190938911A093E6
:108D40008A11B0938B11FE0CCF0DCD0F71C006317F
:108D5000110509F0B4C090919111992309F0F8948C
:108D600061E00E94F05820919111222309F078943B
:108D70000097A9F040E050EC69E774EC409384114F
:108D800050938511609386117093871140938811D9
:108D90005093891160938A1170938B1195C0F09054
:108DA0008D11D0918C1160918C1170918D1176275D
:108DB0006727762780E090E00E9458952DEC3CECE8
:108DC0004CEC5DE30E94B99560938411709385111A
:108DD0008093861190938711E0908F11C0918E112E
:108DE0008C2F8F776E2D70E0782B80E090E00E94C2
:108DF00058952DEC3CEC4CEC5DE30E94B995C7FD19
:108E000009C0609388117093891180938A1190939F
:108E10008B110BC0DC01CB01B0588093881190936B
:108E20008911A0938A11B0938B11DF0DED0ECE0D39
:108E300080919011C81346C0C0908411D0908511C4
:108E4000E0908611F090871120E030E048EC52E489
:108E5000C701B6010E94999818161CF0C0E0D0E036
:108E600002C0CBEFDFEF20E030E0A901C701B6017F
:108E70000E94549587FF02C0CAEFDFEFC0908811AF
:108E8000D0908911E0908A11F0908B1120E030E0B1
:108E900048EC52ECC701B6010E94549587FF02C00E
:108EA000C9EFDFEF20E030E040EF52E4C701B60148
:108EB0000E9499981816ACF4C8EFDFEF12C0CFEFFC
:108EC000DFEF0FC08FEF9FEF8F3FFFEF9F0709F49A
:108ED000D6C0009709F4B0CF029609F4DCC0CCEFFD
:108EE000DFEF0C30110509F0D9C08CE50E94EE6A65
:108EF00080E090E00E94E96A0E94E76A65E08CE504
:108F00000E94E758C82FD0E02097A1F0C530D105C6
:108F1000A4F001E41CE080E490E10E94FB7AF801F7
:108F200080870F5F1F4FC80181549C408C179D079D
:108F300094F306C0CEEFDFEFB1C0CDEFDFEFAEC0F0
:108F4000C091490C00914A0C602F70E080E090E0E5
:108F50000E945A952DEC3CEC4CEC5DE30E94B995D7
:108F60006B017C016C2F70E080E090E00E945A95CC
:108F70009B01AC01C701B6010E94E4966093410CCD
:108F80007093420C8093430C9093440CD0914B0C03
:108F900010914C0C6D2F6F7770E080E090E00E9494
:108FA0005A956B017C01612F70E080E090E00E9497
:108FB0005A952DEC3CEC4CEC5DE30E94B9959B017D
:108FC000AC01C701B6010E94E496D7FF5BC0DC018B
:108FD000CB01B0588093450C9093460CA093470C5E
:108FE000B093480C8C2F800FC82FCD0FC10F8091EC
:108FF0004D0CC81344C0C090410CD090420CE0907E
:10900000430CF090440C20E030E048EC52E4C701FF
:10901000B6010E94999818161CF0C0E0D0E002C07A
:10902000CBEFDFEF20E030E040EA50E4C701B601CB
:109030000E94549587FF02C0CAEFDFEFC090450C35
:10904000D090460CE090470CF090480C20E030E0C7
:1090500040EF51ECC701B6010E94549587FF02C052
:10906000C9EFDFEF20E030E040EF52E4C701B60186
:109070000E949998181694F4C8EFDFEF0FC0CFEF55
:10908000DFEF0CC06093450C7093460C8093470C47
:109090009093480CA7CFCEEFDFEF23CFCE01DF9127
:1090A000CF911F910F91FF90EF90DF90CF90BF90E5
:1090B000AF909F908F900895CF92DF92EF92FF92A2
:1090C0000F931F93CF93DF93CDB7DEB728970FB6DB
:1090D000F894DEBF0FBECDBF823409F43EC0C4F4A5
:1090E000803309F457C074F4833209F44BC08A32D8
:1090F00009F06CC067EB7AE082E491E1C4D98FEFAC
:109100009FEF61C0813309F452C08134E1F05EC049
:109110008136C9F02CF4833451F1843439F056C0CF
:10912000833629F1D4F0843609F050C080913A1189
:1091300090913B11892B09F4EFC086E391E118D897
:1091400097FF75C0E9C06BEA7AE082E491E19BD9B0
:1091500080910F0C9091100C36C06EEA7AE082E498
:1091600091E191D91092850C8CEF9FEF2CC061EBAF
:109170007AE082E491E187D981E08093850C8DEFDC
:109180009FEF21C064EB7AE082E491E17CD98EEF1D
:109190009FEF19C06EE07BE086E391E174D96EE049
:1091A0007BE082E491E16FD980E090E00CC068EB55
:1091B0007AE086E391E167D968EB7AE082E491E1B5
:1091C00062D981E090E00E94A71DACC01A8219828A
:1091D0001C821B821E821D828F831886BE01695FDE
:1091E0007F4FCE0101964FD9BE016F5F7F4F86E35F
:1091F00091E13AD8CE01019670D960E070E086E343
:1092000091E121D8082E000C990B0E947C9C892B9F
:1092100039F086E391E10E94B840CB010E94A71D7E
:1092200064E670E080E090E00E94E6847BC080917C
:10923000800C882359F064EA7AE083EA9FE0C8DA78
:1092400066E371E183EA9FE00E947A6A86E391E136
:109250000E94B8400AEF1FEF2FEF3FEF680179013E
:10926000C61AD70AE80AF90AB701A601CE01019683
:109270000E94346BBE016F5F7F4F86E391E10E94D5
:109280003441CE01019629D986E391E141C08FEFA7
:10929000E81AF80A85E6E816F10459F06EE170E084
:1092A00080E090E00E94E6840E940153182F112371
:1092B00071F38091800C882369F064EA7AE083EA94
:1092C0009FE086DA612F83EA9FE0A2D983EA9FE0DC
:1092D0000E94766A10330CF414516AE270E0611B4C
:1092E000710917FD7395CE0101960E94BB58BE010E
:1092F0006F5F7F4F82E491E10E943441CE0101967D
:10930000ECD862E471E186E391E1D2D882E491E1A4
:109310000E94B840CB0157CF0E940153182FE12C77
:10932000F12CC5CF28960FB6F894DEBF0FBECDBF87
:10933000DF91CF911F910F91FF90EF90DF90CF9031
:109340000895FF920F931F93CF93DF93CDB7DEB7AE
:109350002C970FB6F894DEBF0FBECDBF1092820CD3
:1093600064E77BE0CE010796FCD864E77BE082E40B
:1093700091E189D800E010E0FF24F3948CEC9DE0AB
:109380000E94733E181619062CF58091820C8111EB
:1093900021C08CEC9DE00E94513E8A3071F08D30EE
:1093A00061F09091820C911108C0682FCE01079650
:1093B0000E944C540F5F1F4F06C08B859C85892BE4
:1093C00011F0F092820C6FE070E080E090E00E947B
:1093D000E684D4CF62E370E080E090E00E94E6840F
:1093E000012B51F08CEC9DE00E94113F64E670E08F
:1093F00080E090E00E94E6848091820C811104C09C
:109400008B859C85892BB9F08091800C882369F02D
:10941000BE01695F7F4FCE0101969BD8CE010196B8
:109420000E947258CE01019658D8BE01695F7F4FE5
:1094300082E491E13DD8CE0107964FD82C960FB625
:10944000F894DEBF0FBECDBFDF91CF911F910F917A
:10945000FF9008958F929F92AF92BF92CF92DF922A
:10946000EF92FF92CF93DF93CDB7DEB72C970FB675
:10947000F894DEBF0FBECDBF63EA7BE0CE0101965C
:1094800060D84CE251E06FEF7FEFCE0101960E9471
:109490005E6FCE01019621D86091DC047091DD04ED
:1094A0008091450490914604D1DB84E1882E912C73
:1094B000A12CB12CE12CF12C2FEFE21AF20AC501FC
:1094C000B4010E94E6846091DC047091DD04809117
:1094D000450490914604BADB23E0E216F10434F02F
:1094E0002AE0E216F10444F4892B49F084E1880E65
:1094F000911CA11CB11CE0CF892B09F088C180917F
:109500004504909146048B309105C9F480918811EF
:1095100090918911A0918A11B0918B118093520C76
:109520009093530CA093540CB093550C80918411DC
:1095300090918511A0918611B09187111DC086313F
:10954000910521F30C9701F58091450C9091460C03
:10955000A091470CB091480C8093520C9093530CFF
:10956000A093540CB093550C8091410C9091420CF7
:10957000A091430CB091440C80934E0C90934F0CEF
:10958000A093500CB093510C4091520C5091530C3D
:109590006091540C7091550C21E0CE0107960E9409
:1095A00072426EEB7BE0CE0101960E94B142BE0199
:1095B000695F7F4FCE0101960E94D941BC018AE2CA
:1095C00091E10E945842CE0101960E946D42CE0167
:1095D00007960E946D4240914E0C50914F0C609145
:1095E000500C7091510C21E0CE0107960E947242FE
:1095F00062E779E0CE0101960E94B142BE01695F47
:109600007F4FCE0101960E94D941BC018AE291E1CF
:109610000E94F841CE0101960E946D42CE0107964C
:109620000E946D4264E379E08AE291E10E94EA419E
:1096300064E77BE0CE0101960E94B14244E150E034
:1096400060E070E0CE0101960E94275ACE0101969B
:109650000E946D42C090520CD090530CE090540C7C
:10966000F090550C20E030E0A901C701B6010E943E
:10967000999820E030E040E05FE387FD05C0C70136
:10968000B6010E94E49604C0C701B6010E94E396A9
:109690000E944398AB01BC01CE0101960E94346B3D
:1096A000BE016F5F7F4F84E291E10E943441CE01A1
:1096B00001960E946D4260E087E00E94096B64E2BF
:1096C00071E18BE292E10E940F436FED8BE292E138
:1096D0000E94084368E779E08BE292E179D86091D3
:1096E0004E0C70914F0C8091500C9091510C0E9437
:1096F00043984AE050E08BE292E120D864E379E0BD
:109700008BE292E165D864E670E080E090E00E9430
:10971000E684C090520CD090530CE090540CF09022
:10972000550C20E030E040EF51E4C701B6010E9443
:10973000999887FD03C064E97BE054C020E030E0E5
:1097400040ED51E4C701B6010E94999887FD1FC002
:1097500064E87BE0CE0101960E94A1424AE050E01D
:109760006FEF7FEFCE0101960E945E6FCE010196F2
:109770000E946D4280917304882331F06CED75E096
:1097800080E090E00E94E68464E77BE02BC020E06C
:1097900030E040EB51E4C701B6010E94999887FD83
:1097A00003C066E67BE01EC067E57BE0CE01019664
:1097B0000E94A1424AE050E06FEF7FEFCE01019698
:1097C0000E945E6FCE0101960E946D4280917304EB
:1097D000882331F06CED75E080E090E00E94E68433
:1097E00069E47BE0CE0101960E94A1424AE050E08C
:1097F0006FEF7FEFCE0101960E945E6FCE01019662
:109800000E946D4262E370E080E090E0DCC00E9464
:109810002F6F6EE170E080E090E00E94E6840E948D
:1098200013586B017C0164E670E080E090E00E94D8
:10983000E6846EEB7BE08AE291E10E94434221E004
:10984000B701A601CE0101960E947242BE016F5F70
:109850007F4F8AE291E10E94F841CE0101960E9479
:109860006D426AE271E1CE0101960E94A9424AE08E
:1098700050E060E070E0CE0101960E94275ACE01D0
:1098800001960E946D4280918504882379F0809131
:109890008404882359F06FED8BE292E10E94084323
:1098A0006BEB7AE08BE292E10E94E8436AEB7AE0AC
:1098B0008AE291E10E94EA41C092520CD092530C8C
:1098C000E092540CF092550C20E030E040EF51E46F
:1098D000C701B6010E94999887FD03C069E37BE048
:1098E00054C020E030E040ED51E4C701B6010E94D1
:1098F000999887FD1FC069E27BE0CE0101960E9426
:10990000A1424AE050E06FEF7FEFCE0101960E9446
:109910005E6FCE0101960E946D4280917304882390
:1099200031F06CED75E080E090E00E94E68469E142
:109930007BE02BC020E030E040EB51E4C701B601F2
:109940000E94999887FD03C06BE07BE01EC06CEF1E
:109950007AE0CE0101960E94A1424AE050E06FEF0A
:109960007FEFCE0101960E945E6FCE0101960E94AC
:109970006D4280917304882331F06CED75E080E0D6
:1099800090E00E94E6846EEE7AE0CE0101960E949D
:10999000A1424AE050E06FEF7FEFCE0101960E94B6
:1099A0005E6FCE0101960E946D426CE271E080E034
:1099B00090E00E94E68480917304882331F068EE81
:1099C00073E080E090E00E94E6842C960FB6F89455
:1099D000DEBF0FBECDBFDF91CF91FF90EF90DF9044
:1099E000CF90BF90AF909F908F9008954F925F92CD
:1099F0006F927F928F929F92AF92BF92CF92DF929F
:109A0000EF92FF92CF93DF93CDB7DEB72C970FB6CF
:109A1000F894DEBF0FBECDBF0E942F6F0E9441564B
:109A20002B013C010E9413584B015C0160916F04B3
:109A30007091700480917104909172040E945A9503
:109A40006B017C010E9441560E945A95A701960124
:109A50000E94AA9721E03EED42E45EE30E945899FD
:109A60009B01AC0160E070E080E89FE30E94E39618
:109A700020E03AE24DE257E40E94B9956B017C0187
:109A8000C301B2010E945A9520E030E048EC52E454
:109A90000E94AA97AB01BC0122E0CE0101960E9470
:109AA0007242BE016F5F7F4F8EE191E10E943441AF
:109AB000CE0101960E946D4268EF76E08EE191E161
:109AC0000E94EA416EE171E184E291E10E94584214
:109AD00064EF76E0CE0101960E94B1426EE171E141
:109AE000CE0101960E94D941BC018EE191E10E9414
:109AF0005842CE0101960E946D426EEB7BE08AE2F5
:109B000091E10E94434221E0B501A401CE010196FA
:109B10000E947242BE016F5F7F4F8AE291E10E9414
:109B2000F841CE0101960E946D426DEB7AE08AE227
:109B300091E10E94EA4121E0B701A601CE01019620
:109B40000E947242BE016F5F7F4FCE0107960E9456
:109B5000A94267E279E0CE0107960E94C241BC01AA
:109B60008AE291E10E94F841CE0107960E946D427F
:109B7000CE0101960E946D426EE171E1CE01019627
:109B80000E94A94260E27BE0CE0101960E94C241A0
:109B90006AE271E10E94D941BC018AE291E10E942E
:109BA0005842CE0101960E946D4264E271E1CE01FD
:109BB00001960E94A9424AE050E060E070E0CE01C8
:109BC00001960E94275ACE0101960E946D4221E023
:109BD000B501A401CE0101960E947242BE016F5FE1
:109BE0007F4F80E391E10E943441CE0101960E94B3
:109BF0006D4260E371E1CE0101960E94A9424AE004
:109C000050E06FEF7FEFCE0101960E945E6FCE01B4
:109C100001960E946D4265E070E080E090E00E9455
:109C2000E68468E779E0CE0101960E94B142CE0158
:109C30000196C5D6CE0101960E946D4221E0B70182
:109C4000A601CE0101960E947242BE016F5F7F4F56
:109C5000CE0107960E94A94267E279E0CE010796FD
:109C60000E94C241BC0180E391E10E945842CE01B2
:109C700007960E946D42CE0101960E946D4260E3FC
:109C800071E1CE0101960E94A9424AE050E068EFDE
:109C90007FEFCE0101960E945E6FCE0101960E9479
:109CA0006D4265E070E080E090E00E94E684809183
:109CB000850C882331F068E572E080E090E00E9436
:109CC000E6842C960FB6F894DEBF0FBECDBFDF91B1
:109CD000CF91FF90EF90DF90CF90BF90AF909F908B
:109CE0008F907F906F905F904F90089596E0899F3E
:109CF000D0011124AA55BE4E90967C936E935F9727
:109D000091E091969C93919790911212E091131289
:109D1000F0911412992339F0309751F0811108C055
:109D20008091C21104C0309719F05C968C911994FF
:109D30000895BF92CF92DF92EF92FF920F931F93FD
:109D4000CF93DF93EC016B018D85811105C0CE01AE
:109D50000E94C77B811105C01B861D861C8680E082
:109D600060C040E060EFCE010E944D4501E0E12C73
:109D7000B12C11E0CE010E94747BF82ECE010E941E
:109D8000747B91E0F91203C08130B1F434C02E2D00
:109D900030E0F8121BC08B85181738F4FE01E20F73
:109DA000F31F8381802341F402C0811729F0F12C35
:109DB000193058F41C8709C0FE01EE0DF11D838196
:109DC000802B8383FF24F39409C0B12EFE01E20FA0
:109DD000F31F9381802F8095892383836F2DCE017C
:109DE0000E94987B1F5F000F11F4E39401E087E06D
:109DF0008E1508F0BFCF113408F4AECFBB86B1107A
:109E000002C081E08D878B81882309F4A5CFDE0114
:109E10001396F6012B968D918193CA17DB07D9F71C
:109E200081E0DF91CF911F910F91FF90EF90DF9034
:109E3000CF90BF900895DF92EF92FF920F931F9300
:109E4000CF93DF937C018B01D42EDC011696ED912C
:109E5000FC911797138615861486DF011B9633969F
:109E60001E92EA17FB07E1F7C0E0B801F70186810F
:109E700097815FDFD82F882371F0DC1209C067E07B
:109E8000C8010E943545D80117969C91891721F089
:109E9000CF5FDC1650F7D0E08D2FDF91CF911F916F
:109EA0000F91FF90EF90DF9008950F931F93CF9342
:109EB000DF93C82FD62F86E0C89FF0011124EA5502
:109EC000FE4E11A2878D90A181309105D1F040F016
:109ED00082309105A1F10397E1F560E070E033C0B5
:109EE0006623B9F161E070E08C2F00DF0E941E85CF
:109EF0006093FE117093FF118093001290930112F2
:109F000028C00E941E850091FE111091FF11209122
:109F1000001230910112AB01BC01401B510B620BCE
:109F2000730B8091101290911112A0E0B0E0841791
:109F30009507A607B70718F462E070E004C0D111D6
:109F400008C063E070E08C2FDF91CF911F910F91DB
:109F5000CDCEDF91CF911F910F910895FF920F9376
:109F60001F93CF93DF931F92CDB7DEB7182F062F25
:109F7000F42EAE014F5F5F4F61E070E00E947F59A9
:109F80004981FF2049F021E030E001C0220F0A950D
:109F9000EAF7242B298309C081E090E001C0880FF3
:109FA0000A95EAF78095842389836981812F0E942D
:109FB000E6590F90DF91CF911F910F91FF90089577
:109FC0000F931F93CF93DF93EC019A01452B19F464
:109FD0000E94C53E06C0462F50E060E070E00E943F
:109FE00056438C01CE010E94766A800F911FDF914B
:109FF000CF911F910F910895CF93DF9342E00E947C
:10A00000A56BEC0183EA9FE00E94766A8C0F9D1F8E
:10A01000DF91CF9108958F929F92AF92BF92CF928E
:10A02000DF92EF92FF920F931F93CF93DF9300D0B5
:10A0300000D0CDB7DEB75C0140EA51E166E070E0E8
:10A0400082E30E947F598091A0119091A1119A837F
:10A0500089838091A2119091A3119C838B8380911D
:10A06000A4119091A5119E838D83CE0101966C0160
:10A0700084E9E82E81E1F82E8501F6016191719164
:10A080006F01F70181909190A190B1907F01072E0F
:10A09000000C880B990B0E945A95A50194010E940F
:10A0A000B995F80161937193819391938F01F0EACF
:10A0B000EF16F1E1FF0609F726960FB6F894DEBF1A
:10A0C0000FBECDBFDF91CF911F910F91FF90EF9009
:10A0D000DF90CF90BF90AF909F908F900895CF93D7
:10A0E000DF93C82F809118120E94EE6A6C2F80E4D3
:10A0F00090E10E94437B80E00E948B6A63E0809144
:10A1000018120E94E75880E490E10E94FB7AEC016B
:10A1100080E490E10E94FB7A20E030E0382FC90112
:10A120008C2B9D2BDF91CF9108950F931F93CF938D
:10A13000DF93CDB7DEB761970FB6F894DEBF0FBEE1
:10A14000CDBF8C01462FBE01665F7F4F74DE81114B
:10A1500005C060E070E08EEF92EC4CC0AE014F5F46
:10A160005F4FBE01665F7F4FC8010E949E458823F6
:10A1700061F12A8130E0C901982F8827990F990F42
:10A18000990F698128E0629FB00111249C01262B60
:10A19000372B8A858031E1F4688570E08F81AB01CF
:10A1A000481B5109CA019695982F8827979587953E
:10A1B0000E94259A60517109207F53E0220F331FBE
:10A1C0005A95E1F7620F731F04C060E874EE01C096
:10A1D000B901613854EE75070CF4BBCF072E000CA3
:10A1E000880B990B0E945A9520E030E040E05CE338
:10A1F0000E94B99561960FB6F894DEBF0FBECDBF31
:10A20000DF91CF911F910F9108959F92AF92BF92CE
:10A21000CF92DF92EF92FF920F931F93CF93DF9332
:10A22000CDB7DEB761970FB6F894DEBF0FBECDBFD6
:10A230008C018CE0F8018183C12CD12C2FE5E22E1A
:10A240003FE7B32E4FE1A42E5FE3952EF801848102
:10A2500090E0C816D9060CF0A1C04C2DBE01665F77
:10A260007F4FC801E8DDF8018181893038F0F82E90
:10A27000FCE0F81728F49CE0F92E02C089E0F82EE3
:10A280008A85803139F0BE01665F7F4FC8010E9428
:10A29000F94501C08CE0F81609F47CC0AE014F5FAF
:10A2A0005F4FBE01665F7F4FC8010E949E458823B5
:10A2B00009F470C08A85803109F46CC08BE0F8160F
:10A2C00051F0ECE0FE1629F0FAE0FF1206C09D8284
:10A2D00005C0BD8203C0ED8201C0AD82F801868158
:10A2E00097810E94C77BBE01665F7F4FF801868120
:10A2F00097810E94814540E06EE4F8018681978154
:10A300000E944D4540E06B81F801868197810E9453
:10A310004D4540E06C81F801868197810E944D4552
:10A320008A85803139F040E06D81F801868197811E
:10A330000E944D45F801868197810E94C77BBE012E
:10A34000665F7F4FF801868197810E948145F80101
:10A35000408168E4868197810E944D4564E170E008
:10A3600080E090E00E94E684F8018081882331F04B
:10A370006AE070E080E090E00E94E684F801868167
:10A3800097810E94C77BF80181818F1508F48F2D7A
:10A39000F8018183FFEFCF1ADF0A58CF61960FB61D
:10A3A000F894DEBF0FBECDBFDF91CF911F910F910B
:10A3B000FF90EF90DF90CF90BF90AF909F90089567
:10A3C0008F929F92AF92BF92CF92DF92EF92FF92C5
:10A3D0000F931F93CF93DF93EC018E819F810E9497
:10A3E000C77B40E06CEC8E819F810E944D45488187
:10A3F00064E48E819F810E944D458A81882309F4FF
:10A4000042C0E981E950E33040F4F0E0EE0FFF1F75
:10A41000E951FB4F0081118102C00EEE12E08B81E9
:10A420008823F9F0888181111CC00E941E854B0190
:10A430005C016801110FEE08FF088E819F810E9468
:10A44000747B813001F10E941E85DC01CB018C19E7
:10A450009D09AE09BF0988159905AA05BB0568F3D2
:10A4600012C0B801110F880B990BDF91CF911F918A
:10A470000F91FF90EF90DF90CF90BF90AF909F90A3
:10A480008F900C94E684DF91CF911F910F91FF90F4
:10A49000EF90DF90CF90BF90AF909F908F900895F6
:10A4A000EF92FF920F931F93CF93DF93CDB7DEB759
:10A4B00028970FB6F894DEBF0FBECDBF8C01DC012C
:10A4C0001696ED91FC911797138615861486DF0179
:10A4D0001B9633961E92EA17FB07E1F7F8011482E8
:10A4E0001582EE24E394BE016F5F7F4FD80116966C
:10A4F0008D919C9117971DDC882309F475C067E046
:10A50000CE0101960E94354598858913ECCFF8015C
:10A510008081811124C0868197810E94C77BBE0102
:10A520006F5F7F4FD80116968D919C9117970E946F
:10A53000814540E064EBF801868197810E944D459A
:10A54000D80116968D919C9117970E94747BF82ED6
:10A55000F801868197810E94C77BFF20B1F1D80165
:10A560001196FC9089818031D9F1BE016F5F7F4FD8
:10A57000C8010E94F9458F1518F4F80181810BC0BC
:10A580008981803111F48CE006C0BE016F5F7F4F7E
:10A59000C8010E94F945D80111968C931197149621
:10A5A0008C9114978F5F14968C938981883281F0F7
:10A5B00030F4803169F0823209F095CF09C08B33D5
:10A5C00039F0823409F08FCF03C0F801E082C7CFA1
:10A5D000D80115968C9115978F5F15968C9383CF24
:10A5E000BCE0BF1550F2CFCF28960FB6F894DEBF6F
:10A5F0000FBECDBFDF91CF911F910F91FF90EF90D4
:10A6000008956F927F928F929F92AF92BF92CF9256
:10A61000DF92EF92FF920F931F93CF93DF9381E02E
:10A62000809312120E941E85009102121091031253
:10A630002091041230910512AB01BC01401B510B5B
:10A64000620B730B80910E1290910F12A0E0B0E09C
:10A6500084179507A607B70708F0E6C0C0E0809109
:10A660000C12C81730F0712C812C912C540183945A
:10A6700040C0E0910812F0910912EC0FF11D62E068
:10A6800080810E946084CF5FEACFC62DD0E0E09148
:10A690000812F0910912EC0FFD1F80810E940A84BC
:10A6A0002496CC0FDD1FCA55DE4E892B09F04BC016
:10A6B000888199818C299D299983888363948091CD
:10A6C0000C12681610F3E0910A12F0910B12E00FD1
:10A6D000F11F61E080810E94328480910A12909182
:10A6E0000B12FC01E00FF11F60E080810E9460848A
:10A6F000739480910D12781658F5072D10E0E091B3
:10A700000A12F0910B12E00FF11F61E080810E94AC
:10A710006084E0910A12F0910B12E00FF11F60E0EB
:10A7200080810E943284D501C401072C04C0880FA7
:10A73000991FAA1FBB1F0A94D2F76C017C01E094F9
:10A74000F094612CBCCF888199818E219F21B4CF58
:10A7500026EAE22E21E1F22EF7018FEF9FEF278DFF
:10A7600030A1232B21F4148E968F858F11A236965B
:10A7700021E1E23EF20799F7C0E096E0D92E809100
:10A780000C12C81758F5D0E00C2F10E0000F111F65
:10A7900002551E4E20910D12D217F0F4F80140819F
:10A7A00051810D2E02C0569547950A94E2F7642F09
:10A7B0006170C29F900111242D0F311DE6EAF1E175
:10A7C00080E0A58DB68D2A173B0709F44DC08F5F39
:10A7D00036968A30B1F72CC0CF5FD1CFC0E0F701F9
:10A7E00081A18111C1E0F6E0EF0EF11C22EEE2162C
:10A7F00021E1F206A1F70E941E8560930212709378
:10A8000003128093041290930512CC2369F0809177
:10A81000C711882349F08091C5119091C611019705
:10A8200019F48091C21129C01092121280E025C043
:10A8300040FF1BC0E6EAF1E180E090E0448D411169
:10A8400016C0E0910612F0910712E20FF31F40814B
:10A85000D89EF001D99EF00D1124EA55FE4E448F8A
:10A86000368F258F10A2178E20DBDF5F93CF0196E6
:10A8700036968A30910511F7F8CFDF91CF911F916D
:10A880000F91FF90EF90DF90CF90BF90AF909F908F
:10A890008F907F906F900895CF93DF931F921F92B8
:10A8A000CDB7DEB769831A8241E050E0BE016F5F29
:10A8B0007F4F0E9495410F900F90DF91CF910895A7
:10A8C000FB0144815581FC01248135812417350722
:10A8D00078F080819181009759F0FB01608171814E
:10A8E0006115710529F00E94A69C21E0892B09F0D1
:10A8F00020E0822F08950F931F93CF93DF93FC01E5
:10A90000C481D581209719F4FB01108211C04150F8
:10A9100051094C175D0708F4EA018B01FC016081C5
:10A920007181AE01C8010E94B49CC00FD11F188272
:10A93000DF91CF911F910F9108959091A80D9111E2
:10A94000FCCF91E09093A80D9093A70D2FEF20934B
:10A95000A60D1092A50D260F2093A40D9093830DA4
:10A960009091830D880F892B8093830D8091820DA8
:10A97000813061F41092820D8091830D8093BB0031
:10A980008091BC0083FDF8CF85EC01C085EE8093FB
:10A99000BC008091A80D8130E1F38091A50D861750
:10A9A00010F46091A50DA4E8BDE0ECE5FCE080E0CA
:10A9B000861721F09D9191938F5FFACF0895CF93E1
:10A9C000DF93209185042223A9F02091840422237F
:10A9D00089F0EC016FED8BE292E10E9408438C81DB
:10A9E0009D81892B39F0BE018BE292E1DF91CF91FD
:10A9F0000C940F43DF91CF910895CF93DF93EC0137
:10AA00000E94113FEA89FB8980818F7E8083EA89D9
:10AA1000FB898081877F8083EA89FB8980818F77AA
:10AA20008083EA89FB8980818F7D80838A8D898FED
:10AA3000DF91CF9108953F924F925F926F927F92F4
:10AA40008F929F92AF92BF92CF92DF92EF92FF923E
:10AA50000F931F93CF93DF9300D01F921F92CDB718
:10AA6000DEB7982E0E941E852B013C0120ED420E80
:10AA700027E0521E611C711C60E0809115120E943B
:10AA8000328445E0842ECE0101966C01AA24A39461
:10AA9000B12CF601282D11922A95E9F7860135E0AF
:10AAA000332E27E0E22EF12C809116120E940A84A8
:10AAB000019739F40E941E85641575058605970572
:10AAC00098F3809116120E940A84892B39F40E940F
:10AAD0001E85641575058605970598F380911712F4
:10AAE0000E940A84892B51F0F8012081C5010E2CA7
:10AAF00001C0880F0A94EAF7822B8083F1E0EF1AF5
:10AB0000F10890F63A940F5F1F4F3110CACF0E94A0
:10AB10001E85641575058605970550F061E08091E6
:10AB200015120E94328460E070E080EC9FE72CC038
:10AB300089818911AECF9A818B81890F890D9C8182
:10AB40008913A7CF8D818D3009F0A3CF61E080916B
:10AB500015120E9432846A818B8170E0762F6627FD
:10AB6000680F711D072E000C880B990B0E945A95D7
:10AB700020E030E040E85DE30E94B99523E333E94B
:10AB800048E853E40E94E3960F900F900F900F90C7
:10AB90000F90DF91CF911F910F91FF90EF90DF9079
:10ABA000CF90BF90AF909F908F907F906F905F906D
:10ABB0004F903F900895613208F060E2BEDE10923F
:10ABC0005B0C80935A0C0895CF93C82F87E70E949F
:10ABD000EE6A6C2F80E490E10E94437B0E94E76A5A
:10ABE00087E70E94EE6A61E070E087E790E0E3DFCC
:10ABF00080E490E10E94FB7AC82F0E94E76A8C2FC4
:10AC0000CF910895CF93DF93C82F87E70E94EE6A14
:10AC10006C2F80E490E10E94437B0E94E76A87E703
:10AC20000E94EE6A62E070E087E790E0C4DF80E4B3
:10AC300090E10E94FB7AD82F80E0C82F80E490E159
:10AC40000E94FB7AC82BD92B0E94E76ACE01DF91C4
:10AC5000CF91089587E70E94EE6A64EF80E490E167
:10AC60000E94437B6EE280E490E10E94437B0E945D
:10AC7000E76A65E070E080E090E00E94E68486EF9D
:10AC8000C1CF4F925F926F927F928F929F92AF92BD
:10AC9000BF92CF92DF92EF92FF920F931F93CF93C9
:10ACA000DF9300D01F921F92CDB7DEB7D3DF4C01E8
:10ACB000A12CB12C209148112295220F220F207C2B
:10ACC0002C5C298387E70E94EE6A64EF80E490E1C0
:10ACD0000E94437B698180E490E10E94437B0E9453
:10ACE000E76A80914811811105C065E070E080E05D
:10ACF00090E012C0813029F468E070E080E090E0DC
:10AD00000BC0823029F46EE070E080E090E004C077
:10AD10006AE170E080E090E00E94E68486EF72DFF6
:10AD20006C01E12CF12CFE2CED2CDC2CCC2488EFDA
:10AD30004BDFC82A309148113D8380915D1190917D
:10AD40005E11A5019401281B390B41095109A091FD
:10AD50005B11B0915C110E94A2962B013C01AFE007
:10AD60007594679457944794AA95D1F760915511BB
:10AD700070915611CB01770FAA0BBB0BBC01CD0113
:10AD8000BBE0660F771F881F991FBA95D1F72091F6
:10AD90005711309158118901330F220B330BA90140
:10ADA0009801240D351D461D571D0E948696420EA2
:10ADB000531E641E751E40EA441A4FE0540A61088F
:10ADC0007108A3019201C301B2010E94029A9B0182
:10ADD000AC011CE055954795379527951A95D1F705
:10ADE00029833A834B835C83E0914911F0914A11A6
:10ADF000A0914D11B0914E11A30192010E94AC9609
:10AE00004B015C010DE0B594A794979487940A9543
:10AE1000D1F7A0914F11B091501129813A814B8106
:10AE20005C810E94AC96BB2797FDB095AB2F880D37
:10AE3000991DAA1DBB1D0296A11DB11D32E0B5953D
:10AE4000A795979587953A95D1F79C01AD01305814
:10AE50004F4F5F4FA0915911B0915A110E94A29685
:10AE60004B015C014FE0B694A794979487944A9560
:10AE7000D1F788E090E03D81831B910904C0F694EE
:10AE8000E794D794C7948A95D2F7A0915111B091C5
:10AE9000521129813A814B815C810E94AC969B01C1
:10AEA000AC016BE055954795379527956A95D1F795
:10AEB00029833A834B835C83A0914B11B0914C1151
:10AEC000A30192010E94AC96DC01CB017BE0B59519
:10AED000A795979587957A95D1F749815A816B8186
:10AEE0007C81480F591F6A1F7B1FCF01FF0FAA0BE0
:10AEF000BB0BE2E0880F991FAA1FBB1FEA95D1F791
:10AF0000840F951FA61FB71F0D8004C0880F991FBF
:10AF1000AA1FBB1F0A94D2F7BC01CD016E5F7F4F01
:10AF20008F4F9F4F24E030E040E050E00E94869633
:10AF3000D701C601821B930BA40BB50B9C01AD017D
:10AF400080E593ECA0E0B0E0BC01CD010D8004C031
:10AF500096958795779567950A94D2F70E94029AFD
:10AF600097FD0BC0660F771F881F991FA5019401DD
:10AF70000E94B29649015A010AC0A50194010E949B
:10AF8000B29649015A01880C991CAA1CBB1C99272E
:10AF9000B7FC9A958B2D7A2D692D9B01AC010E94EF
:10AFA000029A9B01AC01AEEDBBE00E94A2966B0140
:10AFB0007C01A3E4B3EEA50194010E94AE96BB27E9
:10AFC00097FDB095AB2F6701FF24D7FCF094EF2CD1
:10AFD0008C0D9D1DAE1DBF1D8153914FAF4FBF4FB7
:10AFE00044E0B595A795979587954A95D1F7BC010B
:10AFF000CD01680D791D8A1D9B1D0F900F900F903C
:10B000000F900F90DF91CF911F910F91FF90EF90D4
:10B01000DF90CF90BF90AF909F908F907F906F9078
:10B020005F904F900895CF92DF92EF92FF920F932F
:10B030001F9310DEAC0160E070E0E8E4F1E1858987
:10B0400096899A01AB01281B390B41095109A38943
:10B05000B4890E94A2966B017C018FE0F594E7947D
:10B06000D794C7948A95D1F765857685CB01770FFC
:10B07000AA0BBB0BBC01CD012BE0660F771F881F0D
:10B08000991F2A95D1F7278530898901330F220B23
:10B09000330BA90198012C0D3D1D4E1D5F1D0E9413
:10B0A0008696DA01C9018C0D9D1DAE1DBF1D089647
:10B0B000A11DB11DBC01CD0134E095958795779513
:10B0C00067953A95D1F70E945A9520E030E040E22A
:10B0D00051E40E94AA971F910F91FF90EF90DF908B
:10B0E000CF900895CF93DF93FC0124813581232BEA
:10B0F00069F0EC01BC0183EA9FE00E947A6ABE011C
:10B100008CEC9DE0DF91CF910C947A6ADF91CF9126
:10B11000089510925B0C10925A0C1092AA0D109286
:10B12000CB0D1092A80D81E08093A70D1092820D97
:10B1300061E084E10E94328461E085E10E94328412
:10B14000E9EBF0E080818E7F808380818D7F80833A
:10B1500088E48093B80085E48093BC0089EE9AE788
:10B160009093590C8093580C8AEE9AE79093570C61
:10B170008093560C08950F931F93CF93DF93CDB711
:10B18000DEB762970FB6F894DEBF0FBECDBF8C015D
:10B19000CB01F8011182108213821282158214826F
:10B1A0004AE0BE016F5F7F4F0E941C91BE016F5F3E
:10B1B0007F4FC8010E94434262960FB6F894DEBFEB
:10B1C0000FBECDBFDF91CF911F910F9108956132D6
:10B1D00008F060E2B2DB10925B0C80935A0C089589
:10B1E000AF92BF92CF92DF92EF92FF920F931F9395
:10B1F000CF93DF93C82FD62F10928C1110928D1100
:10B2000010928E1110928F111092901161E00E9495
:10B21000608460E08C2F0E9432846D2F70E080E0AB
:10B2200090E00E94E68460E08C2F0E9460848BE9AD
:10B2300090E00197F1F700E911E08C2F0E940A8459
:10B24000892B31F401501109C1F78EEF9FEF4CC0EB
:10B2500000E911E08C2F0E940A84019709F43FC095
:10B2600018E2D0E800E090E9E92EFF24F3948C2F57
:10B270000E940A84892B29F481E0E81AF108B9F7C1
:10B28000E4CF0E94C1846B017C0180E9A82EBB241D
:10B29000B3948C2F0E940A84019729F481E0A81AA4
:10B2A000B108B9F7D2CF0E94C184DC01CB018C195F
:10B2B0009D09AE09BF098997A105B10538F0E02FB6
:10B2C000F0E0EC57FE4E80858D2B8087D69511F4EB
:10B2D0000F5FD0E8115039F680E090E005C00150D2
:10B2E000110909F0B7CFB1CFDF91CF911F910F9125
:10B2F000FF90EF90DF90CF90BF90AF900895EF92C6
:10B30000FF920F931F93CF93DF93C82F8B017A0186
:10B3100083E50E94EE6A6C2F80E490E10E94437BFB
:10B320000E94E76A83E50E94EE6AB80183E590E037
:10B3300042DCE701CE018E199F0930915A0C209111
:10B340005B0C321731F080E490E10E94FB7A899324
:10B35000F1CF0817190729F01092921181E080931C
:10B360009311DF91CF911F910F91FF90EF900C946B
:10B37000E76ACF93DF934AE050E0BC0183EA9FE0A5
:10B380000E949E43EC0183EA9FE00E94766A8C0F44
:10B390009D1FDF91CF9108951F93CF93DF931F924D
:10B3A000CDB7DEB7162FAE014F5F5F4F61E070E0A3
:10B3B000A6DF898190E002C0959587951A95E2F7FE
:10B3C00081700F90DF91CF911F910895CF93DF93FC
:10B3D000D82FC62F83E50E94EE6A6D2F80E490E19E
:10B3E0000E94437B6C2F80E490E10E94437BDF91BD
:10B3F000CF910C94E76A0F931F93CF93DF9300D004
:10B4000000D0CDB7DEB72091800C2223A9F08C01AB
:10B410006BE67AE0CE0101960E94B142B801CE01FE
:10B4200001960E94D941BC0183EA9FE00E947A6A9A
:10B43000CE0101960E946D4226960FB6F894DEBFAB
:10B440000FBECDBFDF91CF911F910F910895BF9295
:10B45000CF92DF92EF92FF920F931F93CF93DF93E0
:10B46000CDB7DEB762970FB6F894DEBF0FBECDBF83
:10B470006C018B017A0180918504882309F47CC0DA
:10B4800080918404882309F477C077FF07C0009572
:10B49000109560E0802F0E94096B4DC060E080E055
:10B4A0000E94096B0E941E8528EE33E040E050E0C8
:10B4B0000E948696CA01B90120E831E541E050E0DA
:10B4C0000E948696AB01BC01CE0107960E94346BA8
:10B4D000BE01695F7F4FCE0101960E94A94266E5D9
:10B4E00076E0CE0101960E94C241BC01CE010D96CC
:10B4F0000E94A942CE0101960E946D42CE0107969C
:10B500000E946D42BE01635F7F4F8BE292E10E9419
:10B510000F43B98860E08B2D0E94096B011511055E
:10B5200011F40B2D04C060E0802F0E94096BCE0146
:10B530000D960E946D42B6018BE292E10E940F438C
:10B5400062EC7BE08BE292E10E941D43F601848174
:10B5500060E0800F0E94096B0E941E8560937C0C46
:10B5600070937D0C80937E0C90937F0CB701FF0C41
:10B57000880B990B0E94E68462960FB6F894DEBFA2
:10B580000FBECDBFDF91CF911F910F91FF90EF9034
:10B59000DF90CF90BF900895AF92BF92CF92DF928D
:10B5A000EF92FF920F931F93CF93DF93CDB7DEB748
:10B5B00062970FB6F894DEBF0FBECDBF2091850411
:10B5C000222309F491C020918404222309F48CC021
:10B5D0006A017B015C010E941E8500917C0C109128
:10B5E0007D0C20917E0C30917F0C0C591F4F2F4FFA
:10B5F0003F4F061717072807390708F075C0F7FEF1
:10B6000008C087010095109560E0802F0E94096BAB
:10B610004AC060E080E00E94096B0E941E8528EE0F
:10B6200033E040E050E00E948696CA01B90120E86C
:10B6300031E541E050E00E948696AB01BC01CE01AD
:10B6400001960E94346BBE016F5F7F4FCE0107965B
:10B650000E94A94266E576E0CE0107960E94C241AB
:10B66000BC01CE010D960E94A942CE0107960E9410
:10B670006D42CE0101960E946D42BE01635F7F4F15
:10B680008BE292E10E940F4309891A89E114F104C7
:10B6900031F00E0D1F1D60E0802F0E94096BCE015E
:10B6A0000D960E946D42B5018BE292E10E940F431C
:10B6B00061EB7BE08BE292E10E941D43F501848106
:10B6C00060E0800F0E94096B0E941E8560937C0CD5
:10B6D00070937D0C80937E0C90937F0CB601DD0CF3
:10B6E000880B990B0E94E68462960FB6F894DEBF31
:10B6F0000FBECDBFDF91CF911F910F91FF90EF90C3
:10B70000DF90CF90BF90AF9008950F931F9360E0AC
:10B7100080912E040E94328483E090E00197F1F73B
:10B7200061E080912E040E94328483E290E00197D0
:10B73000F1F760E080912E040E94328480912C0405
:10B7400090912D049927FC01E358F04F6491FC017E
:10B75000E95CF04FE491F0E0EE0FFF1FE35EF04F85
:10B760008591949100E412E42FE030E0462F0E948E
:10B770007485611571058105910549F0DC01CB01E6
:10B780000196A11DB11DBC01CD019F7003C060E0F9
:10B7900070E0CB010E94589520E030E048EC52E484
:10B7A0000E94AA972091860C3091870C4091880CBA
:10B7B0005091890C0E94B99520E030E44CE156E4A8
:10B7C0000E94AA9720E030E040E05FE30E94B99534
:10B7D0001F910F91089523E333E948E853E40E9451
:10B7E000AA9720E030E040E85FE30E94E4960E94E0
:10B7F000A89926E636EA45EA53E40E94B995609393
:10B80000860C7093870C8093880C9093890C089514
:10B81000CF92DF92EF92FF9278DF6B017C0120E004
:10B8200030E040E050E40E94999818161CF46DDF57
:10B830006B017C0120E030E040E050E4C701B6013C
:10B840000E94999818161CF460DF6B017C0120E0BF
:10B8500030E040E050E4C701B6010E949998181604
:10B860001CF453DF6B017C0120E030E040E050E449
:10B87000C701B6010E94999818162CF4FF90EF901A
:10B88000DF90CF9042CFC701B601FF90EF90DF90DD
:10B89000CF900895CF92DF92EF92FF920F931F9374
:10B8A000CF93DF93CDB7DEB762970FB6F894DEBFC4
:10B8B0000FBECDBF81E0809312028AE99CE00E9416
:10B8C000CC31892B09F47AC280918712882319F030
:10B8D00010928712A8C5109287128091800C88233D
:10B8E000D1F16BE67AE0CE0101960E94B142BE0131
:10B8F0006F5F7F4F83EA9FE00E940F43BE016F5F3F
:10B900007F4F8CEC9DE00E940F43CE0101960E9478
:10B910006D4240919E0C50919F0C6091A00C7091D3
:10B92000A10C20E183EA9FE00E94564383EA9FE056
:10B930000E94766A40919E0C50919F0C6091A00CE1
:10B940007091A10C20E18CEC9DE00E9456438CECA0
:10B950009DE00E94766A80919E0C90919F0CA09130
:10B96000A00CB091A10C883025E09207A105B1058B
:10B9700009F4BFC108F08DC0893421E09207A10508
:10B98000B10509F4B9C1E0F5843421E09207A105BD
:10B99000B10509F4A2C1E8F4813421E09207A105C0
:10B9A000B10509F485C138F480349140A105B10591
:10B9B00009F46FC1F1C1823421E09207A105B105FC
:10B9C00009F47FC183349140A105B10509F482C116
:10B9D000E3C1863421E09207A105B10509F483C1D2
:10B9E00008F47EC1873421E09207A105B10509F46E
:10B9F0007DC188349140A105B10509F47AC1CCC15B
:10BA0000823025E09207A105B10509F45AC1E8F496
:10BA1000843721E09207A105B10509F405C138F486
:10BA200082379140A105B10509F409C1B5C181155D
:10BA300025E09207A105B10509F42BC1813095409D
:10BA4000A105B10509F434C1A7C1853025E09207ED
:10BA5000A105B10509F444C170F4833025E09207D3
:10BA6000A105B10509F436C184309540A105B105A1
:10BA700009F433C191C1863025E09207A105B105D3
:10BA800009F431C187309540A105B10509F42EC1F3
:10BA900083C18D3B22E492072FEFA207B10509F481
:10BAA000E9C008F04BC08F3E20E192072FEFA207BC
:10BAB000B10509F41BC118F5823325E09207A105F1
:10BAC000B10509F4BCC038F489309540A105B10531
:10BAD00009F412C161C1843325E09207A105B105C3
:10BAE00009F4A2C08D3F9240AF4FB10509F054C197
:10BAF0006BEA7AE082E491E10E94434290C08D3D7E
:10BB000022E292072FEFA207B10509F48DC038F4A5
:10BB1000873E9841AF4FB10509F4E2C03DC18F3C6B
:10BB200020E392072FEFA207B10509F4D6C0873CA6
:10BB30009843AF4FB10509F4DCC02EC1873928E620
:10BB400092072FEFA207B10509F4B2C040F58D3A74
:10BB500022E592072FEFA207B10509F47CC038F463
:10BB6000853B9A44AF4FB10509F493C015C1853A9E
:10BB70002AE592072FEFA207B10509F4BDC08D3960
:10BB80009246AF4FB10509F007C16BEA7AE082E453
:10BB900091E10E94434281E08093850C40C087354B
:10BBA00028EA92072FEFA207B105F1F078F4853863
:10BBB0002AE792072FEFA207B10509F494C0873650
:10BBC0009849AF4FB10509F47CC0E6C08F3420EB33
:10BBD00092072FEFA207B10509F47CC08D33924C78
:10BBE000AF4FB10561F1D8C06CE271E080E090E048
:10BBF0000E94E68482E080934C1010924F1000E087
:10BC000010E08AE89CE00E94CC31892B09F077C0D3
:10BC10000F5F1F4F0536110509F00EC370C08BEF83
:10BC20009FEF0E94A71DBEC06EEA7AE082E491E118
:10BC30000E9443421092850C8CEF9FEFF2CF61EB94
:10BC40007AE082E491E10E94434281E08093850C96
:10BC50008DEF9FEFE6CF64EB7AE082E491E10E9402
:10BC6000434264EB7AE082E491E10E9443428EEF2A
:10BC70009FEFD7CF67EB7AE082E491E10E944342E5
:10BC800067EB7AE082E491E10E9443428FEF9FEFFD
:10BC9000C8CF6EE07BE086E391E10E9443426EE014
:10BCA0007BE082E491E10E94434280E090E0B9CFE2
:10BCB00068EB7AE086E391E10E94434281E090E004
:10BCC000B0CF65EB7AE086E391E10E94434282E0E7
:10BCD00090E0A7CF83E090E0A4CF84E090E0A1CFF4
:10BCE00085E090E09ECF86E090E09BCF87E090E0FB
:10BCF00098CF88E090E095CF89E090E092CF809156
:10BD0000800C8823B9F063ED7BE083EA9FE00E941A
:10BD10001D4340918E0C50918F0C6091900C70914E
:10BD2000910C2AE083EA9FE00E94564383EA9FE059
:10BD30000E94766A80918E0C90918F0CA091900C4D
:10BD4000B091910C873025E09207A105B10509F467
:10BD500061C208F089C1893421E09207A105B105CB
:10BD600009F45EC208F044C1843421E09207A105C1
:10BD7000B10509F43AC208F024C1813421E09207E8
:10BD8000A105B10509F416C208F00DC18034914037
:10BD9000A105B10509F405C264E670E080E090E019
:10BDA0000E94E6846CE271E080E090E00E94E6840C
:10BDB00082E080934C1010924F104CC064E77BE0FF
:10BDC00082E491E10E9443421092820C64E77BE09E
:10BDD000CE010D960E94B14264E77BE082E491E1DE
:10BDE0000E94434211E083EA9FE00E94733E20914B
:10BDF000820C181619060CF026C2211124C23EC26C
:10BE00000E940153182F882309F49AC28091871247
:10BE100081115ECD64E77BE086E391E10E944342BD
:10BE20008091800C882379F066EE7BE083EA9FE0C6
:10BE30000E941D43612F83EA9FE00E94084383EA2A
:10BE40009FE00E94766A812F0E945C481A3211F0AE
:10BE5000109287120E941E856093E80B7093E90B85
:10BE60008093EA0B9093EB0B92C08CEC9DE00E94C8
:10BE7000513E8A3009F4EEC18D3009F4EBC1909146
:10BE8000820C9111E7C1682FCE010D960E944C548F
:10BE90000F5F1F4F65E070E080E090E00E94E68455
:10BEA0008CEC9DE00E94733E18161906F4F264E1D2
:10BEB00070E080E090E00E94E684012B09F0D2C19E
:10BEC0008091820C882309F4D3C189899A890197CA
:10BED00009F043C066EE78E0CE0101960E94B142BF
:10BEE000BE016F5F7F4FCE010D960E94605481119D
:10BEF00025C267EE7AE0CE0107960E94B142BE01EC
:10BF0000695F7F4FCE010D960E94605411E0811150
:10BF100010E0CE0107960E946D42CE0101960E946C
:10BF20006D421123A1F040E050E0BE01635F7F4FFE
:10BF3000CE0101960E94D96FBE016F5F7F4F86E3ED
:10BF400091E10E943441CE0101960E946D4264E16C
:10BF500070E080E090E00E94E684BE01635F7F4F66
:10BF600082E491E10E945842CE010D960E946D42FA
:10BF70006AE070E080E090E00E94E68480914611E3
:10BF800090914711892B09F43BCF0E943A08809188
:10BF9000850C882309F447C264E670E080E090E0F5
:10BFA0000E94E68440C2823421E09207A105B105D7
:10BFB00009F409C183349140A105B10509F40CC10C
:10BFC000EBCE863421E09207A105B10509F41FC12B
:10BFD00008F414C1873421E09207A105B10509F4E2
:10BFE00019C188349140A105B10509F416C1D4CE18
:10BFF000823025E09207A105B10509F4E4C0E8F418
:10C00000843721E09207A105B10509F40CC138F489
:10C0100082379140A105B10509F4C4CEBDCE81158A
:10C0200025E09207A105B10509F4BBC08130954018
:10C03000A105B10509F4BEC0AFCE843025E092075A
:10C04000A105B10509F4D1C008F4C6C0853025E0CA
:10C050009207A105B10509F4D1C086309540A1052C
:10C06000B10509F4D4C098CE873C28E392072FEF9E
:10C07000A207B10509F4D1C008F03FC08D3F22E00E
:10C0800092072FEFA207B10509F48CCEB8F48930DE
:10C0900025E09207A105B10509F4C2C008F4BDC0AE
:10C0A000823325E09207A105B10509F47BCE8433E4
:10C0B0009540A105B10509F4B6C06ECE873E28E1D2
:10C0C00092072FEFA207B10509F498C038F48F3E0C
:10C0D0009041AF4FB10509F49DC05ECE8D3D22E287
:10C0E00092072FEFA207B10509F49DC08F3C904342
:10C0F000AF4FB10509F479C04FCE8D3922E69207D2
:10C100002FEFA207B10509F44DCE38F5853B2AE49F
:10C1100092072FEFA207B10509F443C078F48D3BD5
:10C120009244AF4FB10509F037CE6BED7AE082E46F
:10C1300091E10E94434284E190E073CD8D3A22E583
:10C1400092072FEFA207B10509F42CCE853A9A4544
:10C15000AF4FB10509F464C01FCE873628E99207B6
:10C160002FEFA207B10579F170F4873928E692071D
:10C170002FEFA207B105F1F085389A47AF4FB1050F
:10C1800009F445C009CE8F3420EB92072FEFA207A8
:10C19000B10511F18D33924CAF4FB10509F402CEC8
:10C1A000FBCD63EC7AE086E391E10E9443428AEFA3
:10C1B0009FEF37CD66EC7AE086E391E10E9443423F
:10C1C00089EF9FEF2ECD69EC7AE086E391E10E9442
:10C1D000434288EF9FEF25CD6CEC7AE086E391E156
:10C1E0000E94434287EF9FEF1CCD6FEC7AE086E31D
:10C1F00091E10E94434286EF9FEF13CD63ED7AE019
:10C2000086E391E10E94434285EF9FEF0ACD84EFE0
:10C210009FEF07CD83EF9FEF04CD82EF9FEF01CD1E
:10C2200081EF9FEFFECC67ED7AE082E491E10E941E
:10C23000434288EE9FEFF5CC6EE170E080E090E045
:10C240000E94E684DECC211140CE00E010E0FF2405
:10C25000F39426CE89899A89892B09F41BCEF09212
:10C26000820C18CE89899A89892B09F03FC028CE83
:10C2700089899A89892B09F028CEACC083EA9FE08E
:10C280000E94513E8A3041F08D3031F0682FCE014E
:10C290000D960E944C5423C089899A89892BF9F004
:10C2A0001093820C6EED7AE0CE0107960E94B142A7
:10C2B000BE01635F7F4FCE0107960E94D941BC014A
:10C2C000CE0101960E94A942CE01019694D8CE01DA
:10C2D00001960E946D42CE0107960E946D426AE06F
:10C2E00070E080E090E00E94E6847DCD69EE7AE027
:10C2F000CE0107960E94B142BE01635F7F4FCE011F
:10C3000007960E94D941BC01CE0101960E94A94224
:10C31000CE01019670D8CE0101960E946D42CE01E9
:10C3200007960E946D428CEC9DE00E94113F64E1F3
:10C3300070E080E090E00E94E684C2CD10E0EDCD98
:10C340008091850C882309F44EC00E941E8528EE3A
:10C35000C22E23E0D22EE12CF12CA70196010E94DF
:10C36000B296CA01B9010E9458952091E40B309110
:10C37000E50B4091E60B5091E70B0E94E39620916C
:10C380001702309118024091190250911A020E942E
:10C390009998181644F50E941E85A70196010E94DF
:10C3A000B296CA01B9010E9458956093E40B70934C
:10C3B000E50B8093E60B9093E70B8091830C9091B3
:10C3C000840C0E94A71D64E170E080E090E00E9470
:10C3D000E684DDCD64E670E080E090E00E94E684D3
:10C3E0000E941E85C1CD0E941E850091E80B109110
:10C3F000E90B2091EA0B3091EB0BDC01CB01801BA8
:10C40000910BA20BB30B88349E4EA105B10508F425
:10C41000BECD1092361260E08BE292E10E94297C40
:10C4200010928404B4CD62960FB6F894DEBF0FBEAE
:10C43000CDBFDF91CF911F910F91FF90EF90DF90D3
:10C44000CF900895EF92FF920F931F93CF93DF93B6
:10C45000CDB7DEB762970FB6F894DEBF0FBECDBF83
:10C460008C018091220D9091230D019731F064E7AA
:10C470007BE0C8010E94B142B3C06FEE7AE0CE010A
:10C480000D960E94B142BE01635F7F4F8CEC9DE030
:10C490000E940F4368EE73E080E090E00E94E68423
:10C4A0000E94A14964EF71E080E090E00E94E68480
:10C4B0006AEF7AE0CE0101960E94B1428091461166
:10C4C00090914711892B81F0E0904211F090431137
:10C4D00069817A81C7010E94C39C009729F09C0161
:10C4E0002E193F09790103C0EE24EA94FE2CCE01F7
:10C4F00001960E946D42A7014F5F5F4F62E471E1B8
:10C50000CE0101960E94D96FBE016F5F7F4FCE01B1
:10C510000D960E943441CE0101960E946D42809199
:10C52000800C8823F1F06BE67AE0CE0101960E9440
:10C53000B142BE01635F7F4FCE0101960E94D94197
:10C54000BC01CE0107960E94A942CE0107960E9427
:10C550007258CE0107960E946D42CE0101960E944C
:10C560006D4289899A89892B61F060E070E0CE0183
:10C570000D960E942341082E000C990BC0970A9734
:10C5800050F064E77BE0C8010E94B142CE010D96F5
:10C590000E946D4225C068E07BE0CE0101960E94BA
:10C5A000B142BE016F5F7F4FCE010D960E94605475
:10C5B000F82ECE0101960E946D42FF2019F06CEF1B
:10C5C0007AE0E1CFF8011182108213821282158283
:10C5D0001482BE01635F7F4FC8010E943441D6CFF1
:10C5E000C80162960FB6F894DEBF0FBECDBFDF91D3
:10C5F000CF911F910F91FF90EF900895AF92BF924E
:10C60000CF92DF92EF92FF920F931F93CF93DF931E
:10C61000CDB7DEB72C970FB6F894DEBF0FBECDBFF7
:10C620008091850C811102C00E942F6F809131048E
:10C6300090913204029751F08091150C9091160C54
:10C64000009709F48DC1039709F48AC16BE17CE07E
:10C6500084E291E10E94FE4164E271E1CE01019623
:10C660000E94A94244E150E060E070E0CE010196F2
:10C670000E94275ACE0101960E946D426CE07CE038
:10C6800084E291E10E94FE4164E271E1CE010196F3
:10C690000E94A94244E150E06FEF7FEFCE01019686
:10C6A0000E945E6FCE0101960E946D4287E00E945B
:10C6B0006F508C0186E00E946F50BC0180E090E0DA
:10C6C0000E9458952AE037ED43EA5CE30E94B99551
:10C6D00023E333E948E853E40E94E3966B017C01CD
:10C6E00084E0A82EB12C20E030E048EC52E4C701F1
:10C6F000B6010E949998181614F581E0A81AB1089D
:10C7000009F4F4C064E670E080E090E00E94E68402
:10C7100086E00E946F50BC0180E090E00E94589536
:10C720002AE037ED43EA5CE30E94B99523E333E95D
:10C7300048E853E40E94E3966B017C01D4CFB80132
:10C7400080E090E00E9458952AE037ED43EA5CE3F0
:10C750000E94B99523E333E948E853E40E94E39645
:10C76000AB01BC0121E0CE0101960E94724262E25F
:10C770007BE0CE0107960E94B142BE016F5F7F4F02
:10C78000CE0107960E94D941BC018AE291E10E9444
:10C790005842CE0107960E946D42CE0101960E943A
:10C7A0006D426AE271E1CE0101960E94A94242E324
:10C7B00050E06FEF7FEFCE0101960E945E6FCE01D9
:10C7C00001960E946D426BEB7AE0CE0101960E94C9
:10C7D000B142CE0101960E94DF54CE0101960E9423
:10C7E0006D426AEB7AE08AE291E10E94EA4121E03F
:10C7F000B701A601CE0101960E9472426EEB7BE06A
:10C80000CE0107960E94B142BE016F5F7F4FCE01FD
:10C8100007960E94D941BC0180E391E10E945842F1
:10C82000CE0107960E946D42CE0101960E946D4294
:10C8300060E27BE0CE0101960E94B14260E371E1CB
:10C84000CE0101960E94D941BC0184E291E10E948F
:10C850005842CE0101960E946D4264E271E1CE0120
:10C8600001960E94A9424AE050E060E070E0CE01EB
:10C8700001960E94CC5ACE0101960E946D426BEB4C
:10C880007AE0CE0101960E94B142CE0101960E944B
:10C89000DF54CE0101960E946D426AEB7AE080E39C
:10C8A00091E10E94EA4160E371E1CE0101960E94AC
:10C8B000A94260E27BE0CE0101960E94C2416AE299
:10C8C00071E10E94D941BC018AE291E10E94584283
:10C8D000CE0101960E946D428091150C9091160C2C
:10C8E000039709F006C184E090E0FFC061E07CE0BE
:10C8F00084E291E10E94FE4164E271E1CE01019681
:10C900000E94A9424AE050E060E070E0CE0101964A
:10C910000E94275ACE0101960E946D4260E17BE0A1
:10C92000CE0101960E94B14264E271E1CE0101960E
:10C930000E94D941BC018AE291E10E945842CE0195
:10C9400001960E946D428091150C9091160C0497EF
:10C9500021F41092160C1092150C81E090E018C191
:10C9600089E69EE00E94FD5464E670E080E090E07D
:10C970000E94E68461E47CE084E291E10E94FE4151
:10C9800064E271E1CE0101960E94A94244E150E0C7
:10C9900060E070E0CE0101960E94275ACE01019618
:10C9A0000E946D4262E37CE084E291E10E94FE41DC
:10C9B00064E271E1CE0101960E94A94244E150E097
:10C9C0006FEF7FEFCE0101960E945E6FCE01019660
:10C9D0000E946D428CE40E941B556B017C0104E0B7
:10C9E00010E0A7019601C701B6010E94E9998111E3
:10C9F00092C021E0B701A601CE0107960E947242C3
:10CA000062E27BE0CE0101960E94B142BE01695F05
:10CA10007F4FCE0101960E94D941BC018AE291E18B
:10CA20000E945842CE0101960E946D42CE010796A7
:10CA30000E946D426AE271E1CE0101960E94A94214
:10CA400042E350E06FEF7FEFCE0101960E945E6FF0
:10CA5000CE0101960E946D426BEB7AE0CE01019609
:10CA60000E94B142CE0101960E94DF54CE01019690
:10CA70000E946D426AEB7AE08AE291E10E94EA410B
:10CA800086E60E941B556B017C0104E010E0A701C3
:10CA90009601C701B6010E94E999882309F47DC077
:10CAA0000150110909F0E2C064E77BE080E391E105
:10CAB0000E94434260E371E1CE0101960E94A942C7
:10CAC00060E27BE0CE0101960E94C2416AE271E120
:10CAD0000E94D941BC018AE291E10E945842CE01F4
:10CAE00001960E946D4283E090E09093160C809333
:10CAF000150C64E670E080E090E00E94E68480918E
:10CB0000850C882309F4BEC060E273E080E090E009
:10CB10000E94E684B7C00150110909F09BC067E28A
:10CB20007CE084E291E10E94FE4164E271E1CE0189
:10CB300001960E94A9424AE050E060E070E0CE0118
:10CB400001960E94275ACE0101960E946D4260E133
:10CB50007BE0CE0101960E94B14264E271E1CE0118
:10CB600001960E94D941BC018AE291E10E9458429B
:10CB7000CE0101960E946D428091150C9091160C89
:10CB8000039721F41092160C1092150C82E090E09D
:10CB90009093320480933104ACCF21E0B701A60119
:10CBA000CE0107960E9472426EEB7BE0CE010196A9
:10CBB0000E94B142BE01695F7F4FCE0101960E9483
:10CBC000D941BC0180E391E10E945842CE01019617
:10CBD0000E946D42CE0107960E946D4260E27BE0AA
:10CBE000CE0101960E94B14260E371E1CE0101964F
:10CBF0000E94D941BC0184E291E10E945842CE01D9
:10CC000001960E946D4264E271E1CE0101960E949C
:10CC1000A9424AE050E06FEF7FEFCE0101960E94FB
:10CC2000CC5ACE0101960E946D426BEB7AE0CE01A8
:10CC300001960E94B142CE0101960E94DF54CE01BE
:10CC400001960E946D426AEB7AE080E391E10E94D6
:10CC5000EA4130CF68EC70E080E090E00E94E6842A
:10CC60008CE40E941B556B017C01BBCE68EC70E02C
:10CC700080E090E00E94E68486E60E941B556B01EE
:10CC80007C0105CF2C960FB6F894DEBF0FBECDBF4A
:10CC9000DF91CF911F910F91FF90EF90DF90CF9098
:10CCA000BF90AF9008952F923F924F925F926F92F4
:10CCB0007F928F929F92AF92BF92CF92DF92EF922C
:10CCC000FF920F931F93CF93DF93CDB7DEB7C55479
:10CCD000D1090FB6F894DEBF0FBECDBF2B013C01CA
:10CCE00069017A010E941E8522966CAF7DAF8EAFDE
:10CCF0009FAF229720E9421621E052066104710499
:10CD000034F090E9492E55245394612C712C30E174
:10CD1000C31637E2D306E104F1042CF4CDA6DEA657
:10CD2000EFA6F8AA08C080E197E2A0E0B0E08DA7E6
:10CD30009EA7AFA7B8AB8091850C882321F0CDA624
:10CD4000DEA6EFA6F8AA22966CAD7DAD8EAD9FADA6
:10CD5000229728EE33E040E050E00E948696269627
:10CD60002CAF3DAF4EAF5FAF269791E09DAB19A6BC
:10CD70001AA61BA61CA68E01035F1F4FCC24DD2420
:10CD80007601C418D508E608F708C9AADAAAEBAAFA
:10CD9000FCAAC9A4DAA4EBA4FCA42DA53EA54FA52A
:10CDA00058A9C216D306E406F5060CF029C3C7013C
:10CDB000B6010E945A9520E030E04AE754E40E9410
:10CDC000AA97AB01BC0123E0C8010E947242B801DE
:10CDD00084E291E10E943441C8010E946D428DA518
:10CDE0009EA5AFA5B8A90A97A105B10584F426961A
:10CDF0004CAD5DAD6EAD7FAD2697C80135D4B801A1
:10CE000084E291E10E943441C8010E946D42CE014A
:10CE100001960E940B5064EF7BE08AE291E10E9450
:10CE2000FE41DE0111961D01C12CD12C7601F101CC
:10CE300081909190A190B1901F01A5019401C5012D
:10CE4000B4010E94B9959B01AC01C701B6010E94D3
:10CE5000E4966B017C0123E0B501A401C8010E94A6
:10CE60007242B801CE0143960E94A94260E27BE083
:10CE7000CE0143960E94C241BC018AE291E10E9428
:10CE8000F841CE0143960E946D42C8010E946D4256
:10CE90000215130561F6C701B6010E94A8996B013E
:10CEA0007C01FDE24F16F1E05F066104710424F09D
:10CEB000D6D760E080E0ADD323E0B701A601CE0174
:10CEC00043960E9472426BE27BE0C8010E94B1422D
:10CED00064E271E1C8010E94D9416EE27BE00E94E8
:10CEE000C241BE016D5E7F4F0E94D94163E37BE08A
:10CEF0000E94C241BC018AE291E10E94F841C8014E
:10CF00000E946D42CE0143960E946D422DEC3CEC96
:10CF10004CE45FE3C701B6010E94999829813A81E8
:10CF20004B815C812DA33EA34FA358A718160CF08C
:10CF3000ABC12AE939E949E95FE3C701B6010E94BB
:10CF4000549587FFA1C1CDA8CC2009F49DC1898447
:10CF50009A84AB84BC8420E030E0A901C501B4010F
:10CF60000E945495CD80DE80EF80F884882309F1FB
:10CF70002DA13EA14FA158A5CA01B9010E94B995A2
:10CF80006EAB7FAB88AF99AFA7019601C701B60121
:10CF90000E94B9959B01AC016EA97FA988AD99AD9E
:10CFA0000E94E4960E94A899A50194010E945797B7
:10CFB00004C06BED7FE089EC9FE320EE3EE245E6A6
:10CFC00052E40E94B9956EAB7FAB88AF99AF20E079
:10CFD00030E0A901C701B6010E945495882309F1E8
:10CFE0002DA13EA14FA158A5CA01B9010E94B99532
:10CFF0006AAF7BAF8CAF9DAFA5019401C501B401B1
:10D000000E94B9959B01AC016AAD7BAD8CAD9DAD25
:10D010000E94E4960E94A899A70196010E94579742
:10D0200004C06BED7FE089EC9FE320EE3EE245E635
:10D0300052E40E94B9956AAF7BAF8CAF9DAF20E000
:10D0400030E0A9016DA17EA18FA198A50E94549501
:10D050008823F9F0A5019401C501B4010E94B99596
:10D060004B015C01A7019601C701B6010E94B99569
:10D070009B01AC01C501B4010E94E4960E94A899ED
:10D080002DA13EA14FA158A50E9457976B017C018D
:10D0900008C08BEDC82E8FE0D82E89ECE82E8FE3E8
:10D0A000F82E6CE27BE0C8010E94B14264E271E1BB
:10D0B000C8010E94D94166E37BE00E94C241BC01E5
:10D0C0008AE291E10E945842C8010E946D426CE2DE
:10D0D0007BE0C8010E94B14264E271E1C8010E9494
:10D0E000D94160E57BE00E94C241BC0184E291E14C
:10D0F0000E945842C8010E946D4221E04EA95FA9DA
:10D1000068AD79ADCE014F960E94724221E04AADE2
:10D110005BAD6CAD7DADCE0149960E94724220EEB2
:10D120003EE245E652E4C701B6010E94B995AB0163
:10D13000BC0121E0C8010E947242B801CE014396B1
:10D140000E94A94260E27BE0CE0143960E94C24168
:10D15000BE01675E7F4F0E94D94160E27BE00E9482
:10D16000C241BE01615E7F4F0E94D941BC018EE188
:10D1700091E10E945842CE0143960E946D42C8013F
:10D180000E946D42CE0149960E946D42CE014F969B
:10D190000E946D422DE2421621E0520661047104A4
:10D1A00074F469A57AA58BA59CA525E030E040E044
:10D1B00050E00E948696672B682B692BB9F564E2D4
:10D1C00071E1C8010E94A94245E050E06FEF7FEF96
:10D1D000C8010E94CC5AC8010E946D4269E57BE0FB
:10D1E000C8010E94B14245E050E061EF7FEFC80105
:10D1F0000E94275AC8010E946D4264E77BE0C80183
:10D200000E94B142C8010E94DF54C8010E946D42D1
:10D210006EE171E1C8010E94A94245E050E060E082
:10D2200070E0C8014BD6C8010E946D426EE171E109
:10D230008AE291E10E94F8413FE143165104610402
:10D24000710434F4C9A4DAA4EBA4FCA4F7FC11C063
:10D250006AE271E1C8010E94A942C8010E947258A5
:10D26000C8010E946D4264E77BE08AE291E10E947E
:10D270004342B201C30177FE04C069A97AA98BA910
:10D280009CA90E94E684A9C023E04DA15EA16FA1E4
:10D2900078A5CE0143960E9472426CE27BE0C80101
:10D2A0000E94B14264E271E1C8010E94D9416BE57C
:10D2B0007BE00E94C241BE016D5E7F4F0E94D9415A
:10D2C00064E37BE00E94C241BC0184E291E10E94E0
:10D2D0005842C8010E946D42CE0143960E946D42A1
:10D2E00049855A856B857C8523E0CE0149960E944D
:10D2F00072424D815E816F81788523E0C8010E9472
:10D300007242B801CE0143960E94A94260E67BE0DA
:10D31000CE0143960E94C241BE01675E7F4F0E94CC
:10D32000D94164E37BE00E94C241BC018EE191E1FE
:10D330000E945842CE0143960E946D42C8010E944D
:10D340006D42CE0149960E946D422DE2421621E0C7
:10D3500052066104710474F469A57AA58BA59CA595
:10D3600025E030E040E050E00E948696672B682B75
:10D37000692BE9F464E271E1C8010E94A9424AE024
:10D3800050E06FEF7FEFC8010E94CC5AC8010E94A5
:10D390006D426EE171E1C8010E94A9424AE050E08D
:10D3A00060E070E0C8018AD5C8010E946D426AE25F
:10D3B00071E1C8010E94A942C8010E947258C801C7
:10D3C0000E946D4264E77BE08AE291E10E94434261
:10D3D000C301B2010E94E6841DAA0E941E856B0152
:10D3E0007C0122962CAD3DAD4EAD5FAD2297C21AA9
:10D3F000D30AE40AF50AC9A6DAA6EBA6FCA6C9CCAC
:10D4000064E271E1CE010D960E94A9424AE050E02B
:10D410006FEF7FEFCE010D960E94275ACE010D9639
:10D420000E946D42CDA8CC20B1F169E57BE0CE0130
:10D430000D960E94B14245E050E061EF7FEFCE01D2
:10D440000D960E94275ACE010D960E946D42809142
:10D45000850C882391F06CEE7BE0CE010D960E9446
:10D46000A14245E050E060E070E0CE010D960E94E0
:10D47000275ACE010D960E946D4264E77BE0CE01F3
:10D480000D960E94B142CE010D960E94DF54CE014E
:10D490000D960E946D426EE171E1CE010D960E94E3
:10D4A000A9424AE050E06FEF7FEFCE010D9606D51E
:10D4B000CE010D960E946D42CB5BDF4F0FB6F89404
:10D4C000DEBF0FBECDBFDF91CF911F910F91FF90B7
:10D4D000EF90DF90CF90BF90AF909F908F907F9014
:10D4E0006F905F904F903F902F90089562E77BE0A0
:10D4F0000C9441430F931F93CF93DF93EC010E9451
:10D500000F438C01CE01F2DF800F911FDF91CF918D
:10D510001F910F910895282F3091CB0D313208F0D3
:10D520004AC08091A80D8111FCCF9091371242E042
:10D530004093A80D2093A70D2FEF2093A60D1092D6
:10D54000A50D3093A40DEBEAFDE0A4E8BDE020E0DA
:10D55000321721F041914D932F5FFACF1092830D36
:10D560002091830D990F922B9093830D9091820DB2
:10D57000913061F41092820D9091830D9093BB00D5
:10D580009091BC0093FDF8CF95EC01C095EE90937F
:10D59000BC009091A80D9230E1F39091A60D9F3FB1
:10D5A00079F08091A60D803241F08091A60D8033F4
:10D5B00031F084E005C081E003C082E001C083E077
:10D5C0001092AA0D1092CB0D1092A90D089581E032
:10D5D000A2CF682F80E490E10C94437B91E090937C
:10D5E000A90D809337121092AA0D1092CB0D0895B9
:10D5F000CF93C82F682F607F8BE292E10E943C7C22
:10D6000080E1C89FB00111248BE292E1CF910C948C
:10D610003C7CCF93DF93CDB7DEB728970FB6F89455
:10D62000DEBF0FBECDBF98E0EDEEF4E0DE01119657
:10D6300001900D929A95E1F790913412961710F49B
:10D640006FEF690FFE013196E60FF11DE60FF11D38
:10D650009081890F806828960FB6F894DEBF0FBEC0
:10D66000CDBFDF91CF91C4CF0F931F93CF93DF93A3
:10D67000CDB7DEB7A2970FB6F894DEBF0FBECDBF11
:10D680008C01CB01BA01F80111821082138212823F
:10D69000158214822AE0AE014F5F5F4F0E942691EF
:10D6A000BE016F5F7F4FC8010E944342A2960FB632
:10D6B000F894DEBF0FBECDBFDF91CF911F910F91C8
:10D6C00008950F931F93CF93DF93EC010E94414382
:10D6D0008C01CE010BDF800F911FDF91CF911F9145
:10D6E0000F910895CF92DF92EF92FF92CF93DF9345
:10D6F0006B017C0197FF15C06DE283EA9FE00E94F9
:10D700000843EC0144275527BA014C195D096E09FD
:10D710007F092AE083EA9FE00E945643C80FD91F81
:10D7200008C02AE0AB01BC0183EA9FE00E94564397
:10D73000EC0183EA9FE0DADE8C0F9D1FDF91CF9131
:10D74000FF90EF90DF90CF9008958F929F92AF92CD
:10D75000BF92CF92DF92EF92FF920F931F93CF93DE
:10D76000DF936B017C01142F9B01AC010E94E999AE
:10D77000882319F065E77BE027C046015701E8944C
:10D78000B7F82FEF3FEF4FE75FE7C501B4010E9405
:10D79000E99981110DC02FEF3FEF4FE75FE7C5011A
:10D7A000B4010E94549518161CF469E77BE00CC084
:10D7B0002FEF3FEF4FE75FE4C701B6010E94999852
:10D7C000181694F46DE77BE083EA9FE0DF91CF9138
:10D7D0001F910F91FF90EF90DF90CF90BF90AF908F
:10D7E0009F908F900C9441432FEF3FEF4FE75FECFA
:10D7F000C701B6010E94549587FDE4CF20E030E0D8
:10D80000A901C701B6010E94549587FF0BC06DE2C4
:10D8100083EA9FE00E940843EC01F7FAF094F7F8DE
:10D82000F09402C0C0E0D0E000E060E070E080E092
:10D830009FE3101741F020E030E040E251E40E9405
:10D84000AA970F5FF6CFA70196010E94E4966B019D
:10D850007C010E9448984B015C012AE0AB01BC01AD
:10D8600083EA9FE00E945643C80FD91F1123C9F1D4
:10D87000C501B4010E9458959B01AC01C701B601D6
:10D880000E94E3966B017C016EE283EA9FE00E94B6
:10D890000843C80FD91F20E030E040E251E4C7013F
:10D8A000B6010E94B9954B015C010E9448986B013A
:10D8B000E12CF12C2AE0B701A60183EA9FE00E9447
:10D8C0005643C80FD91FC701B6010E9458959B0146
:10D8D000AC01C501B4010E94E3966B017C011150BB
:10D8E000D1F6CE01DF91CF911F910F91FF90EF9074
:10D8F000DF90CF90BF90AF909F908F90089525CFED
:10D900002F923F924F925F926F927F928F929F924F
:10D91000AF92BF92CF92DF92EF92FF920F931F933D
:10D92000CF93DF93CDB7DEB728970FB6F894DEBF5D
:10D930000FBECDBFC090320DD090330D4091340D4D
:10D940005091350DC416D5062CF43C2D2D2D6A01B1
:10D95000432F522FE6E3FDE060E070E0CB01019140
:10D9600011910417150754F44A01550FAA08BB0872
:10D97000680D791D8A1D9B1DA80115C0C016D10612
:10D9800054F40D2C000CEE08FF086C0D7D1D8E1D4F
:10D990009F1D680108C0012E000C220B330B600F85
:10D9A000711F821F931F2DE0E238F207C1F60E941B
:10D9B0005A9520E030E048E152E40E94AA978B019A
:10D9C00088879F8382E3E82E8DE0F82E812C912CAE
:10D9D0005401D7016D917D917D01072E000C880BBC
:10D9E000990B0E945A95980148855F810E94E396A1
:10D9F0009B01AC010E94B9959B01AC01C501B4012A
:10DA00000E94E4964B015C01E2E8FDE0EE15FF05A3
:10DA100001F720E030E04CE152E40E94AA970E9416
:10DA2000A8996B017C0120E030E040E85FE30E94B0
:10DA3000999818160CF069C022E33DE03A832983D7
:10DA4000212C312C412C512C3201A981BA818D918C
:10DA50009D91BA83A9839C01990F440B550B2B838D
:10DA60003C834D835E83CA01B9010E945A95980197
:10DA700048855F810E94E3964B015C0120E030E025
:10DA8000A9010E949998181624F0B7FAB094B7F833
:10DA9000B094A7019601C501B4010E94549587FF77
:10DAA0000BC08B819C81AD81BE81480E591E6A1EC0
:10DAB0007B1E9FEF291A390AA2E8BDE0E981FA81AD
:10DAC000AE17BF0711F620E030E040EC5FE3C7017E
:10DAD000B6010E94B9956B017C01F5E02F16310467
:10DAE0000CF4AACFC301B2010E945A956B017C01CC
:10DAF000B101330C880B990B0E945A959B01AC0124
:10DB0000C701B6010E94AA9703C0B80188859F810A
:10DB10006B017C01C701B60128960FB6F894DEBFF1
:10DB20000FBECDBFDF91CF911F910F91FF90EF906E
:10DB3000DF90CF90BF90AF909F908F907F906F902D
:10DB40005F904F903F902F9008954F925F926F9209
:10DB50007F928F929F92AF92BF92CF92DF92EF927D
:10DB6000FF921F93CF93DF93CDB7DEB728970FB601
:10DB7000F894DEBF0FBECDBF4B015C0111E0612EFA
:10DB8000712C9301220F331F220F331F3A832983F5
:10DB9000F901E256FB4FC080D180E280F380A501FD
:10DBA0009401C701B6010E94549587FF02C01F5F10
:10DBB000E6CFA5019401C701B6010E9454954981A1
:10DBC0005A814A575B4F5E834D83811106C0FA012B
:10DBD00060817181828193814DC0F1E06F1AF0EC18
:10DBE0007F0AC301880F991F880F991FFC01E25615
:10DBF000FB4F208131814281538129833A834B83BA
:10DC00005C83FC01EA57FB4F408051806280738047
:10DC1000A3019201ED81FE816081718182819381F6
:10DC20000E94E3966D837E838F83988729813A8152
:10DC30004B815C81C501B4010E94E3969B01AC015C
:10DC40006D817E818F8198850E94B9954B015C0121
:10DC500029813A814B815C81C701B6010E94E3961C
:10DC60009B01AC01C501B4010E94AA97A3019201D6
:10DC70000E94E49628960FB6F894DEBF0FBECDBF83
:10DC8000DF91CF911F91FF90EF90DF90CF90BF90E9
:10DC9000AF909F908F907F906F905F904F9008957E
:10DCA0000F931F930E941E856093710E7093720EE6
:10DCB0008093730E9093740E89E69EE00E94513E0D
:10DCC00097FF1FC00E941E850091710E1091720E69
:10DCD0002091730E3091740EDC01CB01801B910BEF
:10DCE000A20BB30B00916D0E10916E0E20916F0E72
:10DCF0003091700E80179107A207B307E8F28FEFFB
:10DD00009FEF1F910F910895CF92DF92EF92FF92B4
:10DD1000CF93DF93EC016A017B01E889F98982E006
:10DD200080834115514E61057105B1F060E079E0E5
:10DD30008DE390E0A70196010E94B296DA01C90135
:10DD40000197A109B109B695A795979587959C016B
:10DD5000211580E13807A8F0E889F989108260E888
:10DD600074E88EE190E0A70196010E94B296DA0174
:10DD7000C9010197A109B109B695A795979587950E
:10DD80009C01EC85FD853083EE85FF852083188E10
:10DD9000EC89FD8986E08083EA89FB898081806146
:10DDA0008083EA89FB89808188608083EA89FB8996
:10DDB000808180688083EA89FB8980818F7D808370
:10DDC000DF91CF91FF90EF90DF90CF900895CF92A9
:10DDD000DF92FF920F931F93CF93DF93EC010CEA36
:10DDE0001CE06C0186E8C80ED11CF801F1908F018F
:10DDF000CE010E947096F81621F06F2DCE010E9480
:10DE000078962196CC15DD0581F78CEA9CE0DF91B0
:10DE1000CF911F910F91FF90DF90CF900895CF93F6
:10DE2000C091AA0C8EED93E00E947096C81729F05D
:10DE30006C2F8EED93E00E947896C091AB0C8FED25
:10DE400093E00E947096C81729F06C2F8FED93E035
:10DE50000E9478968AEA9CE0CF9108950895809177
:10DE600085048823E1F0809184048823C1F081E057
:10DE7000BFDB8BE39FE10197F1F760E080E0C9DB56
:10DE80006BE37DE08BE292E10E941D4361E080E064
:10DE9000C0DB6BE27DE08BE292E10C941D430895C0
:10DEA00080918504882349F080918404882329F097
:10DEB00060E08BE292E10C94527C08958F929F92E5
:10DEC000AF92BF92EF92FF920F931F93CF93DF9386
:10DED00020918504222309F461C020918404222327
:10DEE00009F45CC08A01EB017C0177FF16C0C09584
:10DEF000D09561E08C2F8DDBB7018BE292E10E941F
:10DF00000F436AE17DE08BE292E10E941D43F7013D
:10DF1000848161E08C0F7DDB31C00E941E85809082
:10DF2000EC0B9090ED0BA090EE0BB090EF0B24E675
:10DF3000820E911CA11CB11C86169706A806B90674
:10DF400068F561E08C2F65DBB7018BE292E10E94FE
:10DF50000F4369E07DE08BE292E10E941D43F701EF
:10DF6000848161E08C0F55DB0E941E856093EC0B71
:10DF70007093ED0B8093EE0B9093EF0BB801110FA4
:10DF8000880B990BDF91CF911F910F91FF90EF902C
:10DF9000BF90AF909F908F900C94E684DF91CF91CB
:10DFA0001F910F91FF90EF90BF90AF909F908F9037
:10DFB0000895CF93DF93EC01FB01248135810E940A
:10DFC000C542CE01DF91CF9108954F925F926F923B
:10DFD0007F928F929F92AF92BF92CF92DF92EF92F9
:10DFE000FF920F931F93CF93DF93CDB7DEB7C65445
:10DFF000D1090FB6F894DEBF0FBECDBF8C0164E728
:10E000007BE0CE01C7960E94B14264E77BE0CE017F
:10E01000CD960E94B142BE016F5F7F4F8FE591E1C7
:10E020000E94BC3F8D889E88AF88B88C498C5A8CE2
:10E030006B8C7C8C8D8D9E8DAF8DB8A127968CAF0F
:10E040009DAFAEAFBFAF2797C8010197039708F008
:10E05000BCC1A3019201C501B40190580E94579719
:10E060002BED3FE049EC5FE30E94E49620916B04C6
:10E0700030916C0440916D0450916E040E94E496BE
:10E080006B017C0120E030E0A9010E94549587FDDE
:10E0900009C0C0924012D0924112E0924212F09216
:10E0A000431210C02BED3FE049EC50E4C701B6012C
:10E0B0000E94E49660934012709341128093421242
:10E0C00090934312C0904012D0904112E0904212BF
:10E0D000F09043122BED3FE049EC50E4C701B6014C
:10E0E0000E949998181684F42BED3FE049EC50E417
:10E0F000C701B6010E94E3966093401270934112EB
:10E10000809342129093431220E030E044E353E4C2
:10E11000609140127091411280914212909143128D
:10E120000E94B9952BED3FE049E450E40E94AA9784
:10E1300060933C1270933D1280933E1290933F1275
:10E140000E944398CE018B960E94BB5861E87BE009
:10E15000CE0185960E94B142BE01655D7F4FCE0122
:10E1600085960E94D9416BE87BE00E94C241BC01C8
:10E1700080E391E10E945842CE0185960E946D4253
:10E18000CE018B960E946D42C0903C12D0903D1201
:10E19000E0903E12F0903F1220E030E044EB52E479
:10E1A000C701B6010E94549518168CF020E030E0AB
:10E1B00040E05FE3C701B6010E94E4960E944398E5
:10E1C000CE018B960E94BB5862E97BE022C020E022
:10E1D00030E044E353E4C701B6010E945495181699
:10E1E0009CF1A701960160E070E884E393E40E944B
:10E1F000E39660933C1270933D1280933E1290938D
:10E200003F120E944398CE018B960E94BB5865E94D
:10E210007BE0CE0185960E94B142BE01655D7F4FD5
:10E22000CE0185960E94D941BC01CE01C7960E94BD
:10E230005842CE0185960E946D42CE018B960E9477
:10E240006D426BED79E061C020E030E047E853E4D7
:10E25000C701B6010E9454951816FCF020E030E08A
:10E2600044E353E4C701B6010E94E39620E030E0A6
:10E2700040E05FE30E94E49660933C1270933D128D
:10E2800080933E1290933F120E944398CE018B964A
:10E290000E94BB5865E97BE01EC0A701960160E0C3
:10E2A00070E084EB93E40E94E39620E030E040E0ED
:10E2B0005FE30E94E49660933C1270933D1280935A
:10E2C0003E1290933F120E944398CE018B960E947B
:10E2D000BB5862E97BE0CE0185960E94B142BE0147
:10E2E000655D7F4FCE0185960E94D941BC01CE016C
:10E2F000C7960E945842CE0185960E946D42CE017B
:10E300008B960E946D4268E97BE0CE01CD960E941B
:10E310004342BE01695C7F4FCE0185960E94A942AF
:10E320004AE050E060E070E0CE0185960E94275AF6
:10E33000CE0185960E946D420E941E85C0907C0C85
:10E34000D0907D0CE0907E0CF0907F0CA4E6CA0E7D
:10E35000D11CE11CF11CC616D706E806F90608F424
:10E3600023C20E941E850E9458956B017C0160911A
:10E370007C0C70917D0C80917E0C90917F0C0E94A2
:10E380005A9520E030E048EC51E40E94E4969B016D
:10E39000AC01C701B6010E94549587FD05C260E239
:10E3A0007BE0CE0185960E94B142BE01635C7F4F47
:10E3B000CE0185960E94D941BC01CE01C7960E942C
:10E3C000F841CE0185960E946D42C80102970297DE
:10E3D00008F0C4C120E030E040E251E4C501B401DE
:10E3E0000E94B9956B017C0120E030E040E251E4ED
:10E3F000C301B2010E94B9954B015C0120E030E0FD
:10E4000040E251E427966CAD7DAD8EAD9FAD279770
:10E410000E94B9952B013C010E941E852091F00BB2
:10E420003091F10B4091F20B5091F30B621B730B87
:10E43000840B950B0E94589520E030E04AE754E4A5
:10E440000E94AA97AB01BC0123E0CE018B960E94EB
:10E4500072426CE27BE0CE0185960E94B142BE0121
:10E46000655D7F4FCE0185960E94D94166E576E0D5
:10E470000E94C241BC018EE191E10E945842CE014E
:10E4800085960E946D42CE018B960E946D426EE190
:10E4900071E1CE0185960E94A94260E371E1CE014F
:10E4A00085960E94D941BE01695C7F4F0E94D94187
:10E4B000BC01CE01C7960E945842CE0185960E94AB
:10E4C0006D426EEF7CE08AE291E10E94FE4121E024
:10E4D000B701A601CE0185960E947242BE016B5D16
:10E4E0007F4F8AE291E10E94F841CE0185960E9419
:10E4F0006D4221E0B301A201CE01C1960E94724299
:10E5000021E0B501A401CE018B960E94724260E227
:10E510007BE0CE0185960E94B142BE01655D7F4FD2
:10E52000CE0185960E94D94160E27BE00E94C24103
:10E53000BE016F5C7F4F0E94D9416AE97BE00E9477
:10E54000C241BC018AE291E10E94F841CE01859668
:10E550000E946D42CE018B960E946D42CE01C19603
:10E560000E946D42A7019601C701B6010E94B995AC
:10E570006B017C01A5019401C501B4010E94B9950C
:10E580009B01AC01C701B6010E94E4966B017C01BE
:10E59000A3019201C301B2010E94B9959B01AC0194
:10E5A000C701B6010E94E4960E94A8996B017C0104
:10E5B000609338127093391280933A1290933B1201
:10E5C0006EE97BE08AE291E10E94EA4121E0B70135
:10E5D000A601CE0185960E947242BE016B5D7F4FFF
:10E5E000CE018B960E94A9426CEA7BE0CE018B960D
:10E5F0000E94C241BC0180E391E10E945842CE01D9
:10E600008B960E946D42CE0185960E946D4260E31A
:10E6100071E18AE291E10E94F841C0903812D090F5
:10E620003912E0903A12F0903B1220E030E04AE7D5
:10E6300054E4C701B6010E94999887FD29C020E0E3
:10E6400030E04AE754E4C701B6010E94AA97AB0143
:10E65000BC0123E0CE0185960E947242BE016B5D33
:10E660007F4FCE018B960E94A9426DEA7BE0CE01DE
:10E670008B960E94C241BC0180E391E10E94584206
:10E68000CE018B960E946D42CE0185960E946D420E
:10E6900020E030E64AE656E4609138127091391273
:10E6A00080913A1290913B120E945495BE01695C90
:10E6B0007F4F87FF4FC0CE0185960E94A9426BE233
:10E6C0007BE0CE0185960E94C2416AE271E10E9420
:10E6D000D941BC018AE291E10E945842CE0185965F
:10E6E0000E946D4203301105A1F46AE271E1CE018E
:10E6F00085960E94A942CE0185960E947258CE014D
:10E7000085960E946D4264E77BE08AE291E10E9477
:10E71000434262EA7BE0CE0185960E94B14260E30B
:10E7200071E1CE0185960E94D941BC01CE018B9644
:10E730000E94A9424AE050E06FEF7FEFCE018B9636
:10E74000BDDBCE018B960E946D42CE0185960E9464
:10E750006D4204C08AE291E10E9458426AE070E092
:10E7600080E090E00E94E684CE01CD960E946D424A
:10E77000CE01C7960E946D42CA5BDF4F0FB6F89478
:10E78000DEBF0FBECDBFDF91CF911F910F91FF90E4
:10E79000EF90DF90CF90BF90AF909F908F907F9041
:10E7A0006F905F904F90089564E77BE0CE0185966F
:10E7B0000E94B142CE0185960E94DF54CE0185961B
:10E7C0000E946D42BE01635C7F4F8BE292E10E942A
:10E7D0000F43E5CD1F93CF93DF93CDB7DEB7A89757
:10E7E0000FB6F894DEBF0FBECDBF182F0E94895818
:10E7F0008EE10E94EE6A62E080E490E144D760E03E
:10E8000080E490E140D70E94E76A8EE10E94EE6AC0
:10E8100061E080E490E137D760E280E490E133D7B3
:10E820000E94E76A80E290E0909363118093621106
:10E8300080E090E8A9E8B4E4809380049093810498
:10E84000A0938204B093830480E090E0A5E7B4E451
:10E8500080937C0490937D04A0937E04B0937F0406
:10E86000BE016F5F7F4F8FE591E10E946F3F1123E3
:10E8700009F486C063ED7CE083EA9FE00E941D43BB
:10E8800083EA9FE00E94766A63EC7CE083EA9FE083
:10E890000E941D43BE016F5F7F4F83EA9FE00E948D
:10E8A000616B63EB7CE083EA9FE00E941D436D8512
:10E8B0007E858F8598890E94726B63EA7CE083EA8B
:10E8C0009FE00E941D4369897A898B899C890E94F7
:10E8D000726B63E97CE083EA9FE00E941D4320E0C5
:10E8E00030E040E251E4698D7A8D8B8D9C8D0E94E1
:10E8F000B99542E050E003D86BEA7BE083EA9FE001
:10E900000E94616B63E87CE083EA9FE00E941D4304
:10E9100020E030E040E251E46D8D7E8D8F8D98A136
:10E920000E94B99542E050E00E947F6C6BEA7BE068
:10E9300083EA9FE00E94616B63E77CE083EA9FE0EB
:10E940000E941D4320E030E040E251E469A17AA139
:10E950008BA19CA10E94B99542E050E00E947F6C7F
:10E960006BEA7BE083EA9FE00E94616B6DE47CE0F0
:10E9700083EA9FE00E941D4383EA9FE00E94766A3B
:10E9800064EF71E080E090E00E94E684A8960FB604
:10E99000F894DEBF0FBECDBFDF91CF911F910895D8
:10E9A00081E08093840480918504882339F088E095
:10E9B0008093361260E08BE292E14BC7089580911C
:10E9C000850481110FC081E08093850480938404C5
:10E9D00080913112982F9460909331128C600E9434
:10E9E000F86A17C080918404882399F01092361237
:10E9F00060E08BE292E12DD7109284048091311275
:10EA00008B7F8093311288600E94F86A109285048F
:10EA10000895C6CF2F923F924F925F926F927F924E
:10EA20008F929F92AF92BF92CF92DF92EF92FF921E
:10EA30000F931F93CF93DF93CDB7DEB766970FB6D3
:10EA4000F894DEBF0FBECDBF1C0186E09FE00E94A0
:10EA5000FD5440E855E260E070E086E09FE054D964
:10EA600064E670E080E090E00E94E6848CED95E042
:10EA7000A0E0B0E080930A0F90930B0FA0930C0FCF
:10EA8000B0930D0F64E670E080E090E00E94E684B1
:10EA90008FEF8A8781E08B8786E88C871D861E86AC
:10EAA0001F86188A198A89E78A8BC101880F991FE6
:10EAB0009E8B8D8BC12CD12CE12CF12C412C512C17
:10EAC000320186E09FE0E214F3046CF5ED89FE89E3
:10EAD000CE16DF0644F50E94423E08974CF049E00E
:10EAE00050E0BE01665F7F4F86E09FE00E94183EC7
:10EAF00065E070E080E090E00E94E68400E010E0D5
:10EB0000812C912C540186E09FE00E94733E892B5A
:10EB100031F4F4E08F169104A104B104ACF5023095
:10EB2000110594F535C00E94FD54E114F10409F477
:10EB30007101C301B2010E945A954B015C01B701FA
:10EB4000FF0C880B990B0E945A959B01AC01C501E3
:10EB5000B4010E94AA9766960FB6F894DEBF0FBE66
:10EB6000CDBFDF91CF911F910F91FF90EF90DF907C
:10EB7000CF90BF90AF909F908F907F906F905F905D
:10EB80004F903F902F9008958FEFC81AD80A99CFD1
:10EB900086E09FE00E94733E892B69F086E09FE04B
:10EBA0000E94513EE1E0F0E0EC0FFD1FE00FF11F8D
:10EBB00080830F5F1F4F65E070E080E090E00E946F
:10EBC000E6840230110569F599818A85981329C078
:10EBD0009A818C85981325C0CE0103969C8B8B8BD4
:10EBE00086E09FE00E94733E892B31F494E0891601
:10EBF0009104A104B1043CF509301105C1F48B81E5
:10EC000090E0982F88272C81820F911D092E000CEF
:10EC1000AA0BBB0B480E591E6A1E7B1EEFEFEE1AA5
:10EC2000FE0AFFEF8F1A9F0AAF0ABF0A6CCF86E079
:10EC30009FE00E94513EEB89FC898193FC8BEB8B1A
:10EC40000F5F1F4FCDCF0430110544F3D8CF2F9263
:10EC50003F924F925F926F927F928F929F92AF926C
:10EC6000BF92CF92DF92EF92FF920F931F93CF93B9
:10EC7000DF936C01C9E5D5E085E3882E84E0982E0A
:10EC80000CEA1CE0EE24E394F12C22E1222E312C3C
:10EC900033E1432E512C40E1642E712C51E1A52E1D
:10ECA000B12C80913304909134048E159F050CF49F
:10ECB000CFC021E0C216D10439F4F80182AD93AD82
:10ECC000F401918380830AC0F2E0CF16D10431F4BD
:10ECD000F40180819181F80193AF82AFF4018081CA
:10ECE0009181009739F48A819B819093DF0480930E
:10ECF000DE0422C08130910539F48A819B81909392
:10ED0000DD048093DC0418C08230910539F48A81D7
:10ED10009B819093DB048093DA040EC0039761F427
:10ED20008A819B819093D9048093D80464E77BE027
:10ED30008EE791E10E944342F401819191914F014C
:10ED40008430910539F42A813B813093110220935C
:10ED5000100221C08530910539F42A813B8130931E
:10ED600007022093060217C08630910539F42A81E4
:10ED70003B813093BF042093BE0417C087309105B8
:10ED800039F42A813B81309305022093040217C095
:10ED90008A309105F1F18531910539F42A813B8161
:10EDA000309303022093020234C08631910539F476
:10EDB0002A813B8130930102209300022AC08731CF
:10EDC000910539F52A813B812830310549F470924B
:10EDD0002F0460922E04B0922D04A0922C0419C02E
:10EDE0002730310549F430922F0420922E0450929E
:10EDF0002D0440922C040DC02630310551F421E041
:10EE000030E030932F0420932E0410922D041092A2
:10EE10002C049C012B5031092A30310590F42A81B1
:10EE20003B813093D9042093D80437E1389FB00157
:10EE3000399F700D1124655E7D4F8EE791E10E9430
:10EE400043428FEFE81AF80A22960E5F1F4F29CF30
:10EE5000DF91CF911F910F91FF90EF90DF90CF90B6
:10EE6000BF90AF909F908F907F906F905F904F90EA
:10EE70003F902F900895FF920F931F93CF93DF93AE
:10EE8000F82E0AE010E0C0E0D0E08F2D0E949C84B4
:10EE9000C80FD91F65E070E080E090E00E94E68432
:10EEA0000150110991F7CE016AE070E00E94119AB9
:10EEB000CB01DF91CF911F910F91FF9008954F9259
:10EEC0005F926F927F92AF92BF92CF92DF92FF924A
:10EED0000F931F93CF93DF9300D000D0CDB7DEB751
:10EEE0005C0186E09FE00E94FD5440E052EC61E04E
:10EEF00070E086E09FE00E94846E8CED95E0A0E0DB
:10EF0000B0E080930A0F90930B0FA0930C0FB09377
:10EF10000D0F64E670E080E090E00E94E684C12C72
:10EF2000D12CF12CCA14DB040CF051C065E070E068
:10EF300080E090E00E94E68400E010E0412C512C3B
:10EF40003201F1100FC086E09FE00E94733E892BD2
:10EF500031F485E148165104610471041CF4033056
:10EF6000110554F08FEFC81AD80A64E670E080E00B
:10EF700090E00E94E684D6CF86E09FE00E94733E38
:10EF8000892B69F086E09FE00E94513EE1E0F0E0CD
:10EF9000EC0FFD1FE00FF11F80830F5F1F4F65E037
:10EFA00070E080E090E00E94E684023011054CF0B1
:10EFB00089818B3B31F4FF24F3948A818A3A09F0EA
:10EFC000F12C8FEF481A580A680A780ABACF8F2DA9
:10EFD00026960FB6F894DEBF0FBECDBFDF91CF915E
:10EFE0001F910F91FF90DF90CF90BF90AF907F90D7
:10EFF0006F905F904F9008951F93CF93DF93182FDA
:10F00000C2E3DDE0812F0E949C84899399936CE395
:10F0100070E080E090E00E94E6848DE0C238D8077E
:10F0200089F70E94806C20E030E040EA50E40E94C2
:10F03000B99520E030E040E85AE30E94B995DF91AD
:10F04000CF911F9108954F925F926F927F92AF92EE
:10F05000BF92CF92DF92EF92FF920F931F93CF93C5
:10F06000DF93CDB7DEB7EA970FB6F894DEBF0FBED9
:10F07000CDBFF82E64E77BE0CE01C5960E94B14279
:10F080008E010B5E1F4F6F2DC801B8D318870F83F9
:10F090001D821E82198289E08A8381E08B838C83A2
:10F0A0001C8A1B8ACE0101960E945052CE01019605
:10F0B0000E94E051CE0101960E9405510E8110E0A0
:10F0C0000330110509F46EC169E67DE0CE01C596F5
:10F0D0000E94FE4164E77BE08AE291E10E944342A4
:10F0E000BE016B5C7F4FCE0183960E94A9424AE02D
:10F0F00050E060E070E0CE0183960E94275ACE0176
:10F1000083960E946D4261E080E00E94096B6EEB85
:10F110007BE0CE01C5960E94434287E1A82E8CE099
:10F12000B82ECC24C394D12CE12CF12CE016F1069E
:10F130000CF0EEC06E2DCE0101960E949550F501A7
:10F1400021913191419151915F010E94E4962B01EF
:10F150003C0120E030E04CEF52EC0E94549587FFD8
:10F1600024C0B601CE0189960E94BB5865E677E0BF
:10F17000CE0183960E94B142BE01675D7F4FCE01F2
:10F1800083960E94D9416FEA7BE00E94C241BC0194
:10F190008AE291E10E94F841CE0183960E946D427D
:10F1A000CE0189960E946D4248C022E0B301A201BF
:10F1B000CE018F960E947242B601CE0189960E94BE
:10F1C000BB5865E677E0CE0183960E94B142BE014E
:10F1D000675D7F4FCE0183960E94D9416FE276E052
:10F1E0000E94C241BE01615D7F4F0E94D941BC01B6
:10F1F0008EE191E10E945842CE0183960E946D42B9
:10F20000CE0189960E946D42CE018F960E946D427A
:10F210006EE171E1CE0183960E94A94260E27BE03B
:10F22000CE0183960E94C241BC018AE291E10E9414
:10F23000F841CE0183960E946D420130110559F4C8
:10F24000E114F10409F05DC06AE271E1CE01C596F6
:10F250000E94584256C00230110511F522E0B30158
:10F26000A201CE0183960E947242BE016D5D7F4F66
:10F27000CE0189960E94A94260E27BE0CE01899688
:10F280000E94C241BC01CE01C5960E94F841CE0148
:10F2900089960E946D42CE0183960E946D4231C0D4
:10F2A0000330110571F16EE171E1CE0183960E9488
:10F2B000A94244E150E06FEF7FEFCE0183960E94B8
:10F2C0005E6FCE0183960E946D426BEB7AE0CE01B9
:10F2D00083960E94B142CE0183960E94DF54CE01F4
:10F2E00083960E946D4280918504882351F080911D
:10F2F0008404882331F060ED77E080E090E00E94A4
:10F30000E684FFEFEF1AFF0A8FEFC81AD80A0ECF74
:10F31000CE01C5960E94C3408AE291E10E94C3409B
:10F3200001151105C9F466E57DE08AE291E10E94CC
:10F33000FE416BE47DE0CE0183960E94A1424AE04B
:10F3400050E06FEF7FEFCE0183960E945E6FCE019B
:10F3500083960E946D42EBC0043011050CF000C191
:10F36000BE016B5C7F4FCE0183960E94A9424AE0AA
:10F3700050E06FEF7FEFCE0183960E945E6FCE016B
:10F3800083960E946D426BEB7AE0CE0183960E94D9
:10F39000B142CE0183960E94DF54CE0183960E9433
:10F3A0006D42DEC06BEB7BE0CE01C5960E9443420E
:10F3B000BE016B5C7F4FCE0183960E94A9424AE05A
:10F3C00050E060E070E0CE0183960E94275ACE01A3
:10F3D00083960E946D4264E77BE08AE291E10E949D
:10F3E00043426AE271E1CE01C5960E94584200E0B4
:10F3F00010E0602FCE0101960E9495506B017C01B8
:10F4000022E0AB01BC01CE0183960115110551F438
:10F410000E947242BE016D5D7F4F8BE292E10E94BD
:10F420000F4318C00E947242BE016D5D7F4FCE0136
:10F4300089960E94A94260E27BE0CE0189960E94F3
:10F44000C241BC01CE01C5960E94F841CE01899609
:10F450000E946D42CE0183960E946D4222E0B70168
:10F46000A601CE0183960E947242BE016D5D7F4F60
:10F47000CE0189960E94A94260E27BE0CE01899686
:10F480000E94C241BC018AE291E10E94F841CE0192
:10F4900089960E946D42CE0183960E946D420F5F55
:10F4A0001F4F0330110509F0A4CFCE01C5960E946D
:10F4B000C340BE016B5C7F4FCE0183960E94A94280
:10F4C0004AE050E06FEF7FEFCE0183960E945E6FBF
:10F4D000CE0183960E946D426BEB7AE0CE0183965B
:10F4E0000E94B142CE0183960E94DF54CE018396E2
:10F4F0000E946D428AE291E10E94C34061EC7BE090
:10F50000CE0183960E94B1426AE271E1CE018396F8
:10F510000E94D9416BEC7BE00E94C241BC018AE2AF
:10F5200091E10E945842CE0183960E946D42CE0125
:10F53000C5960E946D42EA960FB6F894DEBF0FBEE4
:10F54000CDBFDF91CF911F910F91FF90EF90DF9092
:10F55000CF90BF90AF907F906F905F904F90089545
:10F560006BEC7BE08AE291E10E94EA41E0CF85ED1D
:10F570008093BC008091BC0084FDFCCF1092A80D4C
:10F58000089540916412262F30E0240F311D21325E
:10F590003105DCF42091A80D2430C9F4FC0180E091
:10F5A00090E0861758F4309164122191DC01AC5B35
:10F5B000BD4EA30FB11D2C930196F3CF8091641221
:10F5C000680F6093641280E0089581E0089582E0FE
:10F5D0000895089508950895E0915B0C80915A0C68
:10F5E000E81730F4F0E0E45AF34F808190E008959A
:10F5F0008FEF9FEF089590915B0C80915A0C9817B4
:10F6000050F4E92FF0E0E45AF34F208130E09F5F9F
:10F6100090935B0C02C02FEF3FEFC90108958091DA
:10F620005A0C90E020915B0C821B91090895CF92B7
:10F63000DF92EF92FF920F931F93CF93DF937C01A2
:10F64000CB018A012091A90D222389F0EB016B01E6
:10F65000C40ED51ECC15DD0561F06991D701ED9181
:10F66000FC910190F081E02DC7011995F3CF642F33
:10F6700088DFC801DF91CF911F910F91FF90EF902C
:10F68000DF90CF900895CF93DF931F92CDB7DEB771
:10F6900069832091A90D2223D1F02091CB0D203236
:10F6A00040F021E030E0FC013383228380E090E0F1
:10F6B00014C08091AA0DE82FF0E0E555F24F998132
:10F6C00090838F5F8093AA0D8093CB0D04C061E07F
:10F6D000CE01019656DF81E090E00F90DF91CF914F
:10F6E000089580E090E00895FC0190810180F2810E
:10F6F000E02DF8948181892B81832281892F809547
:10F7000028232283A7E0B0E01197F1F7218182231B
:10F710008183A3E2B0E01197F1F780817894EFEC58
:10F72000F0E03197F1F7982381E009F480E0089543
:10F73000FC0190810180F281E02D892F809560FF8E
:10F7400012C0F8942281822382838181892B818354
:10F75000A3E2B0E01197F1F78281982B928378941D
:10F7600087ED90E011C0F894228182238283818109
:10F77000892B8183AFEFB0E01197F1F78281982B4D
:10F78000928378948FE090E00197F1F70895DC017F
:10F790002C911196ED91FC911297F8948181922F02
:10F7A00090958923818378948DE743E050E08150E0
:10F7B00021F1DA011197F1F730813223C1F3F89486
:10F7C0008281892382838181822B81837894ABE734
:10F7D000B7E01197F1F7F89481819823918383E141
:10F7E00091E00197F1F78081282381E009F080E022
:10F7F0007894E3E6F6E03197F1F708951F93CF93FD
:10F80000DF93EC01162F60E0812F0E946084612F4E
:10F8100070E0FB01E358F04FE491E883FB01E95C01
:10F82000F04FE491F0E0EE0FFF1FE35EF04F8591A3
:10F8300094919A8389831B861D861C86FE013B96C4
:10F8400023961292EC17FD07E1F7DF91CF911F91FC
:10F8500008951F93CF93DF93EC01162F8C810E94A4
:10F86000EE6A6B85812F862B90E00E94E96ADF911A
:10F87000CF911F910C94E76A0F931F93CF938C0144
:10F88000C62FE7DF6C2F6460C801E3DF6C2F6B7F4E
:10F89000C801DFDF83EC90E00197F1F7CF911F9172
:10F8A0000F9108950F931F93CF938C01C62F607F04
:10F8B0006160E2DF80E1C89FB00111246160C8018E
:10F8C000DBDF81E090E0CF911F910F9108951F92AF
:10F8D0000F920FB60F9211240BB60F922F933F93F6
:10F8E0004F935F936F937F938F939F93AF93BF9348
:10F8F000EF93FF9380914D108DD720915010309150
:10F9000051102F5F3F4F3093511020935010909122
:10F910004F10953618F096E090934C1090914C1043
:10F920009430C9F128F4923069F09330D1F05EC080
:10F93000953009F451C0963009F058C091E0909389
:10F940001C1151C0811152C02091501030915110A2
:10F950002436310508F442C010921C1110924F1049
:10F960001CC0813009F042C0E0914F1091E09E0F21
:10F9700090934F10F0E02091501030915110EE0F05
:10F98000FF1FEE5AFF4E31832083109251101092C8
:10F99000501094E029C0811117C0E0914F1091E000
:10F9A0009E0F90934F10F0E0209150103091511025
:10F9B000EE0FFF1FEE5AFF4E31832083109251103D
:10F9C0001092501093E010C02091501030915110BF
:10F9D0002536310558F007C0811108C0109251102A
:10F9E0001092501003C095E090934C1090914E10DF
:10F9F000992329F0811102C02F9A01C02F98FF91FD
:10FA0000EF91BF91AF919F918F917F916F915F9196
:10FA10004F913F912F910F900BBE0F900FBE0F9003
:10FA20001F901895CF92DF92EF92FF92CF93DF93C2
:10FA3000EC01072E000C880B990B0E945A956B0164
:10FA40007C0120E030E040E45FE30E94B99520E0D3
:10FA500030E048E452E40E94AA970E944398C617F7
:10FA6000D707D4F020E030E040EA5FE3C701B601F9
:10FA70000E94B99520E030E048E452E40E94AA9741
:10FA800020E030E040E85FE30E94E4960E94439863
:10FA900021E06C177D070CF420E0822F90E0DF91CD
:10FAA000CF91FF90EF90DF90CF9008950F931F9329
:10FAB000CF93DF93082F60E779E083EA9FE00E940D
:10FAC000E843C7E0D0E010E0B8010C2E02C0759505
:10FAD00067950A94E2F76170772742E050E083EA85
:10FAE0009FE00E949E43219778F7DF91CF911F916D
:10FAF0000F9108951F920F920FB60F9211240BB61B
:10FB00000F922F933F934F935F936F937F938F93B6
:10FB10009F93AF93BF93EF93FF938091B900887F3A
:10FB2000803609F49CC068F5883209F45BC090F413
:10FB3000803109F454C038F4882309F4F6C08830C1
:10FB400009F44DC0F5C0883109F44CC0803209F485
:10FB50005DC0EEC0803409F468C048F4803309F415
:10FB600055C0883309F0E4C08093A60DD8C0803515
:10FB700009F44FC0883509F45DC0883409F0D8C055
:10FB8000D6C0883909F4C7C0A8F4883709F467C01B
:10FB900038F4883609F463C0803709F460C0C8C0FF
:10FBA000883809F4B8C0803909F45FC0803809F09A
:10FBB000BFC05BC0803B09F486C038F4803A09F4CA
:10FBC00066C0883A09F47FC0B3C0803C09F4A7C07E
:10FBD000883C09F4A4C0883B09F48AC0A9C080917C
:10FBE000830D10C09091A50D8091A40D981770F50C
:10FBF000E091A50D81E08E0F8093A50DF0E0EC570C
:10FC0000F24F80818093BB0085EC86C08093A60D67
:10FC10008EC0E091A50D81E08E0F8093A50D80919F
:10FC2000BB00F0E0EC57F24F80839091A50D8091DE
:10FC3000A40D6EC0E091A50D81E08E0F8093A50DFF
:10FC40008091BB00F0E0EC57F24F80838091A70DCC
:10FC500081116DC081E08093820D84EA61C083E0F0
:10FC60008093A80D10928612CFCF80918612803299
:10FC700008F051C0E091861281E08E0F80938612C9
:10FC80008091BB00F0E0EA59FD4E8083BDCF85EC4A
:10FC90008093BC001092A80D80918612803230F4BF
:10FCA000E0918612F0E0EA59FD4E108260918612D2
:10FCB00070E0E091560CF091570C86E692E11995B0
:10FCC0001092861235C084E08093A80D10926512C0
:10FCD00010926412E091580CF091590C1995809192
:10FCE0006412811105C081E0809364121092441265
:10FCF000E091651281E08E0F80936512F0E0EC5B7D
:10FD0000FD4E80818093BB009091651280916412BA
:10FD1000981708F479CF85E88093BC0009C085EC7A
:10FD20008093BC001092A80D03C01092A60D1FDC9A
:10FD3000FF91EF91BF91AF919F918F917F916F91C3
:10FD40005F914F913F912F910F900BBE0F900FBE7F
:10FD50000F901F9018950C940F9B08953F924F920F
:10FD60005F926F927F928F929F92AF92BF92CF924B
:10FD7000DF92EF92FF920F931F93CF93DF93CDB754
:10FD8000DEB7A4970FB6F894DEBF0FBECDBF81E0FB
:10FD90008093871200E010E082E0382E0E301105CB
:10FDA00008F0AAC2F8018827E955FF4F8F4F0C943D
:10FDB000389A8091220D9091230D892B09F568ECDA
:10FDC00079E0CE0107960E94B1426FE172E1CE0167
:10FDD00007960E94D941BC01CE0101960E94A9421A
:10FDE00048EC50E06FEF7FEFCE0101960E94275A5A
:10FDF000CE0101960E946D42CE0107960E946D428F
:10FE00008091220D9091230D019709F564EB79E023
:10FE1000CE0107960E94B1426FE172E1CE010796D2
:10FE20000E94D941BC01CE0101960E94A94248EC32
:10FE300050E06FEF7FEFCE0101960E94275ACE016E
:10FE400001960E946D42CE0107960E946D428091FC
:10FE5000220D9091230D029709F56DED79E0CE0109
:10FE600007960E94B1426FE172E1CE0107960E94AF
:10FE7000D941BC01CE0101960E94A94248EC50E054
:10FE80006FEF7FEFCE0101960E94275ACE010196B7
:10FE90000E946D42CE0107960E946D4262EE79E0AB
:10FEA000CE0107960E94B14269E172E1CE01079648
:10FEB0000E94D941BC01CE0101960E94A94240EDA9
:10FEC00057E06FEF7FEFCE0101960E945E6FCE018B
:10FED00001960E946D42CE0107960E946D4280916C
:10FEE000220D9091230D0197E9F5CE0107960E940E
:10FEF00022628B859C85009789F1EF81F8852081AE
:10FF0000222361F1079750F160EE7EE0CE01019669
:10FF10000E94A14248EC50E06FEF7FEFCE010196C6
:10FF20000E94CC5ACE0101960E946D42BE01695FCB
:10FF30007F4FCE0101960E94A94248EC50E06FEF3E
:10FF40007FEFCE0101960E945E6FCE0101960E9466
:10FF50006D4260ED77E080E090E038D5CE01079605
:10FF60000E946D4264E670E080E090E02FD5309210
:10FF70004C1010924F10C0C164ED7EE0CE0101968E
:10FF80000E94A14248EC50E06FEF7FEFCE01019656
:10FF90000E94CC5ACE0101960E946D424FD56B0152
:10FFA0007C014CD528EE33E040E050E00E94B29650
:10FFB000CA01B90120E831E541E050E00E94B29663
:10FFC00020E13EE040E050E00E94869649015A015F
:10FFD0002CE330E040E050E00E94869629013A018F
:10FFE000AB01BC01CE0101960E94346BB301A201AA
:10FFF000CE0107960E94346BB501A401CE010D9687
:020000021000EC
:100000000E94346BC701B60120E03CE546E255E0B2
:100010000E94B296BA01A901CE0149960E94346BA2
:10002000BE01675E7F4FCE0143960E94A9426EEDEE
:100030007BE0CE0143960E94C241BE01635F7F4FC9
:100040000E94D94161EE7BE00E94C241BE01695F1E
:100050007F4F0E94D9416DE179E00E94C241BE010B
:100060006F5F7F4F0E94D94166EE78E00E94C241E7
:10007000BC01CE014F960E94A942CE0143960E9438
:100080006D42CE0149960E946D42CE010D960E94AE
:100090006D42CE0107960E946D42CE0101960E94EC
:1000A0006D4240ED57E06FEF7FEFCE014F960E941B
:1000B0005E6FCE014F961EC18091150C9091160C6B
:1000C000019719F465EC7EE002C067EB7EE0CE019B
:1000D00001960E94A14248EC50E06FEF7FEFCE0105
:1000E00001960E94CC5ACE0101960E946D4267EAA9
:1000F0007EE0F2C067E97EE0CE0101960E94A14257
:1001000048EC50E06FEF7FEFCE0101960E94CC5A91
:10011000CE0101960E946D426AE87EE0DDC06DE787
:100120007EE0CE0101960E94A14248EC50E06FEFC4
:100130007FEFCE0101960E94CC5ACE0101960E941B
:100140006D4262E77EE0C8C066E67EE0CE010196C1
:100150000E94A14248EC50E06FEF7FEFCE01019684
:100160000E94CC5ACE0101960E946D4265E57EE068
:10017000B3C08091150C9091160C039719F46AE4A2
:100180007EE002C060E47EE0CE0101960E94A142C2
:1001900048EC50E06FEF7FEFCE0101960E94CC5A01
:1001A000CE0101960E946D4265E37EE095C068E253
:1001B0007EE0CE0101960E94A14248EC50E06FEF34
:1001C0007FEFCE0101960E94CC5ACE0101960E948B
:1001D0006D4269E17EE080C06EE07EE0CE01019676
:1001E0000E94A14248EC50E06FEF7FEFCE010196F4
:1001F0000E94CC5ACE0101960E946D4261E07EE0E1
:100200006BC08091150C9091160C029719F460EF59
:100210007DE002C060EE7DE0CE0101960E94A14229
:1002200048EC50E06FEF7FEFCE0101960E94CC5A70
:10023000CE0101960E946D4263ED7DE04DC067ECFA
:100240007DE0CE0101960E94A14248EC50E06FEFA4
:100250007FEFCE0101960E94CC5ACE0101960E94FA
:100260006D4267EB7DE038C06CEA7DE0CE0101961F
:100270000E94A14248EC50E06FEF7FEFCE01019663
:100280000E94CC5A35C06CE97DE0CE0101960E94F7
:10029000A14248EC50E06FEF7FEFCE0101960E9443
:1002A000CC5ACE0101960E946D426FE87DE014C0E9
:1002B00063E87DE0CE0101960E94A14248EC50E047
:1002C0006FEF7FEFCE0101960E94CC5ACE010196CE
:1002D0000E946D4263E77DE0CE0101960E94A1423B
:1002E00040ED57E06FEF7FEFCE0101960E945E6F09
:1002F000CE0101960E946D420E940153882319F09D
:10030000109287120CC00E944A5C80918712882349
:1003100031F00F5F1F4F0F30110509F03FCDA4964C
:100320000FB6F894DEBF0FBECDBFDF91CF911F9106
:100330000F91FF90EF90DF90CF90BF90AF909F9084
:100340008F907F906F905F904F903F900895CF93E4
:10035000DF930E94895810923012809134128230BB
:1003600018F098E09093301290913512992339F05B
:10037000813029F48091301284608093301262E3DE
:1003800070E080E090E022D3609136128BE292E13F
:1003900060DA68EE73E080E090E018D360E38BE20F
:1003A00092E16ADACBE4D6E4CE010197F1F760E39B
:1003B0008BE292E161DA2197F1F760E38BE292E15F
:1003C0005BDA83E592E00197F1F760E28BE292E17C
:1003D00053DA8091301280620E94F86A84E0809340
:1003E00031128CE00E94F86A81E00E94F86ACBE347
:1003F000DFE1CE010197F1F782E08093321286E0CF
:100400000E94F86A82E00E94F86A2197F1F7DF9172
:10041000CF910895FF920F931F93CF93DF93CDB7A2
:10042000DEB72B970FB6F894DEBF0FBECDBF86E0C8
:100430009FE00E94FD5440E855E260E070E086E0F5
:100440009FE00E94846E64E670E080E090E0BED29F
:100450008CED95E0A0E0B0E080930A0F90930B0F35
:10046000A0930C0FB0930D0F64E670E080E090E075
:10047000ADD28FEF898381E08A8386E88B831C82EB
:100480001D821E821F82188689E7898786E09FE089
:100490000E94113F62E370E080E090E097D286E036
:1004A0009FE00E94423E08974CF049E050E0BE01B8
:1004B0006F5F7F4F86E09FE00E94183E62E370E02E
:1004C00080E090E083D286E09FE00E94733E892B1B
:1004D00001F186E09FE00E94423E089784F465E0C7
:1004E00070E080E090E072D200E010E0F12C86E055
:1004F0009FE00E94733E02301105A4F50CC049E054
:1005000050E0BE016F5F7F4F86E09FE00E94183E83
:10051000E6CFF12C27C086E09FE00E94733E892B36
:1005200099F465E070E080E090E050D2023011056F
:10053000F1F69A8589819813DACF9B858B81981380
:10054000D6CFFF24F394D3CF86E09FE00E94513EA4
:10055000EAE0F0E0EC0FFD1FE00FF11F80830F5F7A
:100560001F4FDFCF62E370E080E090E02FD286E0A3
:100570009FE00E94FD548F2D2B960FB6F894DEBF9E
:100580000FBECDBFDF91CF911F910F91FF900895C6
:100590008091241190912511009711F00C94E39013
:1005A00060E070E0CB010895AF92BF92CF92DF92EE
:1005B000EF92FF920F931F93CF93DF9320914611F9
:1005C00030914711FC01448155818901041B150BB1
:1005D0004115510559F12115310541F12417350710
:1005E00028F10217130718F08901015011097C0145
:1005F000A0904211B0904311C501DFEFCFEF65012C
:10060000C00ED11EC816D906A0F0F7016081718115
:100610000E94C39C009769F09C012A193B090217AC
:10062000130710F0D22FC32F0196ECCF8FEF9FEF5F
:1006300002C08D2F9C2FDF91CF911F910F91FF90C2
:10064000EF90DF90CF90BF90AF9008958F929F92E0
:10065000AF92BF92CF92DF92EF92FF920F931F93D0
:10066000CF93DF93EB01E881F981DC011C966D915A
:100670007C911D97E617F7070CF04BC0BF01660F82
:10068000771F1A968D919C911B97DB01A80FB91FBC
:10069000AD90BC90E170FF276F01B1E0CB26EF2B4E
:1006A00019F48CE99FEF02C084E690E079018A0199
:1006B0004C01820E931EB401C501B4D9892B89F473
:1006C0008E0C9F1CB401C501ADD9892B69F4B7010B
:1006D000680D791DC501A6D9892BF1F023E030E022
:1006E00005C021E030E002C022E030E0F801808166
:1006F00091810196821793071CF49183808307C030
:100700001182108288819981019699838883C6011C
:1007100005C081E090E002C08FEF9FEFDF91CF91A5
:100720001F910F91FF90EF90DF90CF90BF90AF900F
:100730009F908F90089590E0FC013197E231F10590
:1007400008F04EC08827EB54FF4F8F4F0C94389A17
:10075000809180008F7703C0809180008F7D80938F
:100760008000089580918000877FF9CF84B58F77CE
:1007700002C084B58F7D84BD08958091B0008F77CD
:1007800003C08091B0008F7D8093B0000895809168
:1007900090008F7707C0809190008F7D03C080917B
:1007A0009000877F8093900008958091A0008F77BC
:1007B00007C08091A0008F7D03C08091A000877F3B
:1007C0008093A0000895809120018F7707C08091C9
:1007D00020018F7D03C080912001877F80932001BD
:1007E0000895FC01A089B1898C91A689B78982FD01
:1007F0000FC09C91818D8F5F8F73228D821749F07E
:10080000218DDF01A20FB11D5D969C93818F08950C
:100810008C910895CF93DF93282F30E0F901ED53A9
:10082000F04F8491F901E358F04FD491F901E95C5C
:10083000F04FC491CC2389F081117DDFEC2FF0E0E3
:10084000EE0FFF1FE35EF04FA591B491EC91ED2305
:1008500081E090E021F480E002C080E090E0DF9150
:10086000CF9108951F93CF93DF93282F30E0F901A4
:10087000ED53F04F8491F901E358F04FD491F90111
:10088000E95CF04FC491CC23B9F0162F811153DFEE
:10089000EC2FF0E0EE0FFF1FED5FF04FA591B4914C
:1008A0009FB7F894111104C08C91D095D82302C041
:1008B000EC91DE2BDC939FBFDF91CF911F910895C8
:1008C000CF93DF9390E0FC01E358F04F2491FC01BB
:1008D000E95CF04F8491882361F190E0880F991FC3
:1008E000FC01E751F14FC591D491FC01ED5FF04F50
:1008F000A591B491611109C09FB7F89488812095A2
:1009000082238883EC912E230BC0623061F49FB761
:10091000F8948881322F309583238883EC912E2B95
:100920002C939FBF06C08FB7F894E8812E2B2883A5
:100930008FBFDF91CF910895863308F08653909151
:100940007B00282F2870977F922B90937B0020911B
:10095000E00490E4299F900111248770822B8093FA
:100960007C0080917A00806480937A0080917A0084
:1009700086FDFCCF809178002091790090E0922B49
:1009800008953FB7F89480918D1290918E12A091A6
:100990008F12B091901226B5A89B05C02F3F19F079
:1009A0000196A11DB11D3FBFBA2FA92F982F8827EF
:1009B000820F911DA11DB11DBC01CD0142E0660F4A
:1009C000771F881F991F4A95D1F708958F929F929C
:1009D000AF92BF92CF92DF92EF92FF926B017C01B8
:1009E000D0DF4B015C01C114D104E104F104E9F052
:1009F000C8DFDC01CB0188199909AA09BB09883E27
:100A00009340A105B10578F321E0C21AD108E108AD
:100A1000F10888EE880E83E0981EA11CB11CC11459
:100A2000D104E104F10421F7DECFFF90EF90DF90D5
:100A3000CF90BF90AF909F908F9008952FB7F8946C
:100A40006091891270918A1280918B1290918C1210
:100A50002FBF08951F920F920FB60F9211242F935C
:100A60003F938F939F93AF93BF93809189129091FF
:100A70008A12A0918B12B0918C123091881223E0CF
:100A8000230F2D3720F40196A11DB11D05C026E8C6
:100A9000230F0296A11DB11D209388128093891205
:100AA00090938A12A0938B12B0938C1280918D1226
:100AB00090918E12A0918F12B09190120196A11D6B
:100AC000B11D80938D1290938E12A0938F12B093CC
:100AD0009012BF91AF919F918F913F912F910F9065
:100AE0000FBE0F901F901895CF92DF92EF92FF925A
:100AF0000F931F93E82FF92F05C001501109210909
:100B0000310961F1908196239417B9F305C0015022
:100B100011092109310911F1908196239413F7CF1E
:100B2000C12CD12CE12CF12C0AC08FEFC81AD80AA5
:100B3000E80AF80A0C151D052E053F0579F080819D
:100B40008623841791F36C2D7D2D8E2D9F2D1F9163
:100B50000F91FF90EF90DF90CF90089560E070E0EC
:100B600080E090E01F910F91FF90EF90DF90CF9089
:100B70000895CF93DF93CDB7DEB762970FB6F894A1
:100B8000DEBF0FBECDBF789484B5826084BD84B5CE
:100B9000816084BD85B5826085BD85B5816085BD78
:100BA00080916E00816080936E0010928100809130
:100BB00081008260809381008091810081608093B8
:100BC0008100809180008160809380008091B100DD
:100BD00084608093B1008091B00081608093B00008
:100BE000809191008260809391008091910081605A
:100BF000809391008091900081608093900080911B
:100C0000A10082608093A1008091A1008160809307
:100C1000A1008091A00081608093A00080912101BB
:100C20008260809321018091210181608093210164
:100C30008091200181608093200180917A008460FE
:100C400080937A0080917A00826080937A0080910C
:100C50007A00816080937A0080917A008068809326
:100C60007A001092C10061E089E12ADE61E089E149
:100C7000F9DD0E9489586EEE79E083EA9FE00E94D8
:100C8000616BE12CF12C17E2812F0E94EE6A0E9429
:100C9000E76A811120C06AEF79E083EA9FE00E9451
:100CA000E84340E150E0612F83EA9FE00E94E04F7B
:100CB00010932F1266E17AE083EA9FE00E94E843F6
:100CC00040E150E0612F83EA9FE00E94E04F8FEF08
:100CD000E81AF80A0FC0843069F460E37AE083EA26
:100CE0009FE00E94E84340E150E0612F83EA9FE0EB
:100CF0000E94E04F1F5F103439F6EF2819F46BE4BF
:100D00007AE002C061E67AE083EA9FE00E94616BCC
:100D10001EDB80E40E94F86A04E714E0F8016191A8
:100D20008F018BE292E10E94527CF4E00C371F07A6
:100D3000A9F70E942F6F0E94D0748EED93E09093DC
:100D4000400C80933F0C0E9470968093AA0C8FED0C
:100D500093E00E9470968093AB0C8091AA0C9091C6
:100D6000AB0C1816190654F410927304019731F461
:100D70001092AB0C1092AA0C0E940F6F6DEB7AE0F0
:100D8000CE0101960E94A1424AE050E06FEF7FEF52
:100D9000CE0101960E94275ACE0101960E946D4213
:100DA00040E052EC61E070E083EA9FE00E94846ED4
:100DB00080917304882329F068EE73E080E090E06E
:100DC00005DE83EA9FE00E94513E182F823709F426
:100DD000CEC11092400C10923F0C5CEAC52E5CE034
:100DE000D52EE12CF12CC7010E947096F60181935B
:100DF0006F01FFEFEF1AFF0A86E8E816F10499F792
:100E00008091AC0C9091AD0CA091AE0CB091AF0C58
:100E100085369105A105B1050CF495C180936F0449
:100E200090937004A0937104B09372048091B00CFD
:100E30009091B10CA091B20CB091B30C80936B0463
:100E400090936C04A0936D04B0936E048091B40CE5
:100E50009091B50CA091B60CB091B70C809367043B
:100E600090936804A0936904B0936A0468EC7CE0F2
:100E7000CE0101960E94B142BE016F5F7F4F85E2B5
:100E800092E10E943441CE0101960E946D4266E2D9
:100E90007DE0CE0101960E94B142BE016F5F7F4F9F
:100EA0008FE192E10E943441CE0101960E946D4291
:100EB00023E030E040E050E065E272E1CE010196CF
:100EC0000E94C54223E030E040E050E06FE172E173
:100ED000CE0107960E94C5422B853C858D819E815F
:100EE0002817390719F58F81988569817A810097CC
:100EF00019F061157105A9F46115710551F02115FD
:100F0000310539F0FB01808190E09195819591093F
:100F10000AC0009769F0232B59F0FC01808190E012
:100F200002C00E94969C01E0892B19F000E001C0EC
:100F300001E0CE0107960E946D42CE0101960E940B
:100F40006D42011106C065E272E18FE192E10E94FB
:100F500058428091B80C9091B90CA091BA0CB09104
:100F6000BB0C8093630490936404A0936504B093D6
:100F700066048091BC0C9091BD0CA091BE0CB09108
:100F8000BF0C80935F0490936004A0936104B093BE
:100F900062048091C00C9091C10CA091C20CB091E0
:100FA000C30C80935B0490935C04A0935D04B093A6
:100FB0005E048091C40C9091C50CA091C60CB091B8
:100FC000C70C8093570490935804A0935904B0938E
:100FD0005A048091D00C9091D10CA091D20CB09178
:100FE000D30C8093BA049093BB04A093BC04B09339
:100FF000BD048091D40C9091D50CA091D60CB091E9
:10100000D70C8093B6049093B704A093B804B09320
:10101000B9048091D80C9091D90CA091DA0CB091C0
:10102000DB0C8093530490935404A0935504B09325
:1010300056048091DC0C9091DD0CA091DE0CB091F7
:10104000DF0C80934F0490935004A0935104B0930D
:1010500052048091E00C9091E10CA091E20CB091CF
:10106000E30C80934B0490934C04A0934D04B093F5
:101070004E04C090F60CD090F70CE090F80CF09075
:10108000F90CA7019601C701B6010E94E9998111E7
:1010900008C0C0924704D0924804E0924904F092FC
:1010A0004A046091220D7091230D072E000C880BCD
:1010B000990B0E945A959B01AC010E94E9998823E3
:1010C00021F01092230D1092220DE090240DF0904B
:1010D000250DB7010F2C000C880B990B0E945A9517
:1010E0009B01AC010E94E999811104C0F092460471
:1010F000E09245042AEFE22E2CE0F22E37E1C32ED7
:101100003CE0D32E42E2A42E4DE0B42EF7014190F4
:101110005190619071907F01A3019201C301B201CE
:101120000E94E999811105C0F601408251826282D4
:101130007382F4E0CF0ED11CAE14BF0439F781E006
:1011400090E00E9427760EE8010F013089F01E36EC
:1011500079F08091AC0C9091AD0CA091AE0CB09157
:10116000AF0C85369105A105B10514F055C100E01D
:1011700080916F0490917004A0917104B0917204F9
:101180008093AC0C9093AD0CA093AE0CB093AF0CCD
:1011900080916B0490916C04A0916D04B0916E04E9
:1011A0008093B00C9093B10CA093B20CB093B30C9D
:1011B0008091670490916804A0916904B0916A04D9
:1011C0008093B40C9093B50CA093B60CB093B70C6D
:1011D0001337B1F088EC9CE0009739F048E050E01C
:1011E000BC0185E292E10E947B5486E29DE000977B
:1011F00039F04CE050E0BC018FE192E10E947B5459
:101200008091630490916404A0916504B091660498
:101210008093B80C9093B90CA093BA0CB093BB0C0C
:1012200080915F0490916004A0916104B091620488
:101230008093BC0C9093BD0CA093BE0CB093BF0CDC
:1012400080915B0490915C04A0915D04B0915E0478
:101250008093C00C9093C10CA093C20CB093C30CAC
:101260008091570490915804A0915904B0915A0468
:101270008093C40C9093C50CA093C60CB093C70C7C
:101280008091BA049091BB04A091BC04B091BD04BC
:101290008093D00C9093D10CA093D20CB093D30C2C
:1012A0008091B6049091B704A091B804B091B904AC
:1012B0008093D40C9093D50CA093D60CB093D70CFC
:1012C0008091530490915404A0915504B091560418
:1012D0008093D80C9093D90CA093DA0CB093DB0CCC
:1012E00080914F0490915004A0915104B091520408
:1012F0008093DC0C9093DD0CA093DE0CB093DF0C9C
:1013000080914B0490914C04A0914D04B0914E04F7
:101310008093E00C9093E10CA093E20CB093E30C6B
:101320008091470490914804A0914904B0914A04E7
:101330008093F60C9093F70CA093F80CB093F90CF3
:1013400080914504909146049093250D8093240D3F
:10135000E7E1FCE0AAEFBCE08FE39CE04191519112
:10136000619171914D935D936D937D938E179F075E
:10137000A9F767EA7AE0CE0101960E94A142CE0168
:1013800001960E94FB59CE0101960E946D4283E3B3
:10139000E82E84E0F82E94EEA92E9CE0B92EC12C04
:1013A000D12C80913304909134048C159D0554F117
:1013B000F70180819181F501819391935F01809183
:1013C000800C8823C1F06BE67AE083EA9FE00E94FC
:1013D000E8434AE050E0B60183EA9FE00E949E4362
:1013E00068E67AE083EA9FE00E94E843F7018081A3
:1013F00091810E94B959FFEFCF1ADF0A82E0E80E0F
:10140000F11CCFCF023040F41092400C10923F0CF0
:1014100080E090E00E94E76E8091220D9091230D74
:101420008D7F892B41F440E855E260E070E08CEC60
:101430009DE00E94846E8091220D9091230D019772
:1014400041F440E052EC61E070E08CEC9DE00E94E1
:10145000846E64E670E080E090E0B8DA8091220D5E
:101460009091230D892B09F0B3C01E3671F0809145
:10147000AC0C9091AD0CA091AE0CB091AF0C853638
:101480009105A105B1050CF0A3C064E77BE0CE0196
:1014900007960E94B1426CE577E0CE0101960E946A
:1014A000B1426FE172E1CE0101960E94D941BC01C7
:1014B000CE0107960E945842CE0101960E946D42CD
:1014C000BE01695F7F4F8CEC9DE00E940F4368EB8B
:1014D0007BE080E090E07ADABE01695F7F4FCE0169
:1014E00001960E94A942CE0101960E94FB59CE01AD
:1014F00001960E946D426CE271E080E090E066DA55
:101500004091231250912412425051096FE172E12F
:10151000CE0101960E94D96FBE016F5F7F4FCE0151
:1015200007960E943441CE0101960E946D42BE0191
:10153000695F7F4FCE0101960E94A942BE01695F9B
:101540007F4FCE0101960E94D941BC01CE01079682
:101550000E945842CE0101960E946D426FE977E0E9
:10156000CE0101960E94B142BE01695F7F4FCE015C
:1015700001960E94D941BC01CE0107960E945842B3
:10158000CE0101960E946D42BE01695F7F4F8CECD7
:101590009DE00E940F4368EB7BE080E090E016DA6C
:1015A000BE01695F7F4FCE0101960E94A942CE0124
:1015B00001960E94FB59CE0101960E946D426CE299
:1015C00071E080E090E002DACE0107960E946D4261
:1015D00064E670E080E090E0F9D9F89482E08093CE
:1015E000B0008093B10094E69093B3001092B200E3
:1015F00080937000789480934C1010924F108091DB
:101600004D1060E05DD967E97AE0CE0101960E9455
:10161000A1424AE050E06FEF7FEFCE0101960E94B9
:10162000275ACE0101960E946D428091220D909121
:10163000230D892B09F568EC79E0CE0107960E940D
:10164000B1426FE172E1CE0107960E94D941BC011F
:10165000CE0101960E94A9424AE050E06FEF7FEF71
:10166000CE0101960E945E6FCE0101960E946D42EE
:10167000CE0107960E946D428091220D9091230D1C
:10168000019709F564EB79E0CE0107960E94B1421B
:101690006FE172E1CE0107960E94D941BC01CE01F3
:1016A00001960E94A9424AE050E06FEF7FEFCE0121
:1016B00001960E945E6FCE0101960E946D42CE019E
:1016C00007960E946D428091220D9091230D029702
:1016D00009F56DED79E0CE0107960E94B1426FE108
:1016E00072E1CE0107960E94D941BC01CE0101965C
:1016F0000E94A9424AE050E06FEF7FEFCE010196D1
:101700000E945E6FCE0101960E946D42CE01079647
:101710000E946D428091220D9091230D019709F056
:1017200058C0CE010D960E94226289899A8900973D
:1017300009F44BC0ED85FE852081222309F445C0C4
:10174000079708F442C06DE67AE0CE0107960E9442
:10175000B1426FE172E1CE0107960E94D941BC010E
:10176000CE0101960E94A942CE0101960E947258B4
:10177000CE0101960E946D42CE0107960E946D42F5
:101780006EE87AE0CE0101960E94A14248EC50E05A
:101790006FEF7FEFCE0101960E94CC5ACE010196E9
:1017A0000E946D42BE01635F7F4FCE0101960E9491
:1017B000A94248EC50E06FEF7FEFCE0101960E9406
:1017C0005E6FCE0101960E946D42CE010D960E9481
:1017D0006D426BE67AE0CE0107960E94B1426FE15E
:1017E00072E1CE0107960E94D9416AE77AE00E9431
:1017F000C241BC01CE0101960E94A942CE010196D0
:101800000E947258CE0101960E946D42CE01079649
:101810000E946D4264E670E080E090E0D7D80E94BC
:10182000895864E670E080E090E0D0D883E20E94BE
:10183000EE6A81E090E00E94E96A0E94E76A83E034
:1018400090E09093160C8093150C8CE40E941B552D
:101850006B017C0162E370E080E090E0B7D8A70103
:101860009601C701B6010E94E999882309F44CC08A
:1018700086E60E941B556B017C0162E370E080E00C
:1018800090E0A4D8A7019601C701B6010E94E9998A
:101890008823D1F11092160C1092150C89E69EE067
:1018A0000E94FD5464E670E080E090E08FD840E84C
:1018B00055E260E070E089E69EE00E94846E89E671
:1018C0009EE00E94733E892B71F164E77AE0CE01BD
:1018D00001960E94A142CE0101960E94FB59CE01C1
:1018E00001960E946D4282E090E09093160C8093E6
:1018F000150C64E670E080E090E068D88091150CEB
:101900009091160C039779F46FE57AE0CE01019679
:101910000E94A142CE0101960E94FB59CE01019680
:101920000E946D4222C086E00E946F50BC0180E0A0
:1019300090E00E9458952AE037ED43EA5CE30E946C
:10194000B99523E333E948E853E40E94E39620E0A5
:1019500030E048E453E40E94549587FF06C082E0DB
:1019600090E0909332048093310483E08093481197
:101970000E94895880ED0E94E455853509F02AC1FE
:101980008AEA0E94025690934A11809349118CEA88
:101990000E94025690934C1180934B118EEA0E9444
:1019A000025690934E1180934D1180EB0E94025687
:1019B00090935A118093591182EB0E940256909392
:1019C0005C1180935B1184EB0E94025690935E1130
:1019D00080935D1186EB0E94025690935011809384
:1019E0004F1188EB0E94025690935211809351112F
:1019F0008AEB0E94025690935411809353118CEB02
:101A00000E94025690935611809355118EEB0E94BE
:101A10000256909358118093571166E27AE08AE259
:101A200091E10E94FE410E9441560E945A950E94F7
:101A300043980E945A9520E030E048EC52E40E941E
:101A4000AA97AB01BC0122E0CE0107960E94724228
:101A5000BE01695F7F4FCE0101960E94A94268EFE7
:101A600076E0CE0101960E94C241BC018AE291E17A
:101A70000E94F841CE0101960E946D42CE01079668
:101A80000E946D426AE271E1CE0101960E94A94274
:101A9000CE0101960E94FB59CE0101960E946D4233
:101AA00060E17AE08AE291E10E94FE4160916F0478
:101AB000709170048091710490917204FBD720E0C2
:101AC00030E048EC52E40E94AA97AB01BC0122E04E
:101AD000CE0107960E947242BE01695F7F4FCE0120
:101AE00001960E94A94268EF76E0CE0101960E941D
:101AF000C241BC018AE291E10E94F841CE01019607
:101B00000E946D42CE0107960E946D426AE271E129
:101B1000CE0101960E94A942CE0101960E94FB5976
:101B2000CE0101960E946D42113629F481E00E9497
:101B30007C3881E011C083EA9FE00E94513E182F5B
:101B400064E670E080E090E00E94E684113671F374
:101B500080E00E947C3880E00E94EA7364E670E0D6
:101B600080E090E00E94E6848091150C9091160C24
:101B7000892B91F489E69EE00E94FD5461E08091FA
:101B80002E040E94608460E080912C040E94608496
:101B90000E9413580E94EB5B10917304112331F0E3
:101BA00068EE73E080E090E00E94E68465EB7AE006
:101BB00086E391E10E94434282E090E09093100C12
:101BC00080930F0C11110E942A4A0E944A5C0E94C5
:101BD000323FFBCF69E37AE0CE0101960E94A14239
:101BE000CE0101960E947258CE0101960E946D426C
:101BF00010923004B3CFEF92FF920F931F93CF93C5
:101C0000DF93CDB7DEB7C456D1090FB6F894DEBF67
